:100000000C9445160C9476160C9476160C94761671
:100010000C9476160C9476160C9476160C94761630
:100020000C9476160C9476160C9476160C94761620
:100030000C9476160C9454590C9476160C947616EF
:100040000C9476160C9423C40C9476160C947616A5
:100050000C9476160C9476160C947F760C940A59B0
:100060000C9476160C94BD4B0C9476160C94761664
:100070000C9476160C9476160C9476160C947616D0
:100080000C9476160C9476160C9476160C947616C0
:100090000C9476160C9476160C9476160C947616B0
:1000A0000C9476160C9476160C9476160C947616A0
:1000B0000C9476160C9476160C9476160C94761690
:1000C0000C9476160C9476160C9476160C94761680
:1000D0000C9476160C9476160C946F580C94305839
:1000E0000C9476168631A331D431F13106322F3299
:1000F0009C320233AB33F3370138FA3721382538D5
:100100003F389A3C5438A038C738EE3817396D3923
:100110007E398F39A039B139C2399A3CA53B9A3C16
:10012000B03B203C263C463CD6B0D9B0C8B0CCB0A1
:10013000D2B010B1DDB0E1B0E7B0EBB0EFB0F5B0E8
:10014000F9B0FDB010B103B107B10BB170B675B61F
:100150007AB684B68EB607B798B6A0B6A8B6B2B6C9
:10016000BCB6C6B6D5B6DFB607B7E9B6F3B6FDB6C8
:10017000084AD73B3BCE016E84BCBFFDC12F3D6C0E
:1001800074319ABD56833DDA3D00C77F11BED9E474
:10019000BB4C3E916BAAAABE000000803F05A84C54
:1001A000CDB2D44EB93836A9020C50B99186880820
:1001B0003CA6AAAA2ABE000000803F004E414E493C
:1001C0004E495459494E46CDCCCC3D0AD7233C1715
:1001D000B7D13877CC2B329595E6241FB14F0A0062
:1001E0000020410000C84200401C4620BCBE4CCA52
:1001F0001B0E5AAEC59D74434F4D4D554E4943415C
:1002000054494F4E0044525952554E004552524F98
:10021000525300494E464F004543484F0047322F46
:1002200047332062616420706172616D657465722C
:10023000730A00206F6620004D424C20473239205F
:10024000706F696E74200059206F7574206F66207E
:1002500072616E67652028312D35292E0A005820DD
:100260006F7574206F662072616E67652028312D6E
:1002700035292E0A004D6573682070726F62696EB1
:100280006720646F6E652E0A005374617274206D6E
:100290006573682070726F62696E67207769746831
:1002A0002022473239205331222066697273742E1E
:1002B0000A004732380A47323920533200537461FA
:1002C00074653A20004D65736820626564206C6532
:1002D00076656C696E6720686173206E6F2064615B
:1002E00074612E0A0053206F7574206F662072614E
:1002F0006E67652028302D35292E0A004D657368FC
:1003000020706F696E742063616E6E6F7420626519
:10031000207265736F6C7665640A00456E642066B2
:10032000696C65206C6973740A00426567696E20A8
:1003300066696C65206C6973740A00286E6F2066AC
:10034000696C6529005344207072696E74696E6728
:10035000206279746520004E6F74205344207072BF
:10036000696E74696E670A0043757272656E7420F7
:1003700066696C653A20002569730025696D202542
:100380006973002569682025696D2025697300253A
:100390006964202569682025696D20256973002519
:1003A000697920256964202569682025696D2025E3
:1003B0006973005072696E742074696D653A20002B
:1003C0006F6E2E0A006F66662E0A00473236204492
:1003D000656275672000180213020C020502F7011E
:1003E0006F66660044454255473A004B494C4C45C0
:1003F000442E20004D3131332053006F6B002C20F0
:10040000002C2000544845524D414C5F50524F54EF
:10041000454354494F4E004155544F5245504F5259
:10042000545F53445F53544154555300454D455216
:1004300047454E43595F5041525345520043415343
:10044000455F4C494748545F4252494748544E45DE
:10045000535300544F47474C455F4C49474854530A
:1004600000534F4654574152455F504F5745520035
:100470004255494C445F50455243454E54004C450B
:1004800056454C494E475F44415441005A5F5052D3
:100490004F4245004155544F4C4556454C00505233
:1004A000494E545F4A4F420050524F4752455353B2
:1004B000004155544F5245504F52545F54454D5092
:1004C00000564F4C554D45545249430045455052F6
:1004D0004F4D0053455249414C5F584F4E5F584F66
:1004E0004646004649524D574152455F4E414D45A3
:1004F0003A4D61726C696E20312E312E39202847B9
:1005000069746875622920534F555243455F434FC4
:1005100044455F55524C3A68747470733A2F2F6794
:1005200069746875622E636F6D2F4D61726C696EB0
:100530004669726D776172652F4D61726C696E20CC
:1005400050524F544F434F4C5F56455253494F4EB4
:100550003A312E30204D414348494E455F54595061
:10056000453A3344205072696E7465722045585480
:1005700052554445525F434F554E543A31205555DC
:1005800049443A63656465326132662D34316132C3
:100590002D343734382D396231322D633535633699
:1005A000326633363766660A002F2F20002054004B
:1005B000205200416363656C65726174696F6E3AC5
:1005C0002050005741524E494E4721204C6F772012
:1005D0005A204A65726B206D6179206C65616420D8
:1005E000746F20756E77616E7465642070617573C9
:1005F00065732E0A00546F6F206661722066726FF9
:100600006D207265666572656E636520706F696ED8
:10061000740A0020466C6F773A20000001363726B6
:10062000032BFFFFFF3C3D382AFFFFFFFF2E303E2C
:1006300012FFFFFFFFFFFFFF0809FF2C071A1C181E
:10064000FFFFFF08440A2C4324221E20643A0020A6
:10065000693A0020703A00496E76616C69642065E1
:10066000787472756465720A0043290A0061626CCD
:10067000656420286D696E2074656D702000436F7D
:100680006C6420657874727564657320617265208E
:100690000020643A0020693A0020703A004E6F2032
:1006A00063617365206C696768740A004545505240
:1006B0004F4D204F4B0A00205A004475616C204575
:1006C0006E6473746F702041646A7573746D656EC7
:1006D0007420286D6D293A20003F4B2076616C759F
:1006E00065206F7574206F662072616E67652028C3
:1006F000302D3130292E0A00416476616E63652009
:100700004B3D004163746976652045787472756469
:1007100065723A2000496E76616C69642065787470
:1007200072756465720A0043616E6E6F7420656E47
:10073000746572207375626469723A2000473931BA
:100740000A4731205A2D302E30320A4739300053B3
:1007500070656369616C204D656E753A205A20445E
:100760006F776E20302E310A004739310A47312029
:100770005A2D302E30320A47393000537065636984
:10078000616C204D656E753A205A20446F776E205B
:10079000302E30320A004739310A4731205A2B3087
:1007A0002E30320A473930005370656369616C201E
:1007B0004D656E753A205A20557020302E30320A21
:1007C000004739310A4731205A2B302E310A473938
:1007D00030005370656369616C204D656E753A2019
:1007E0005A20557020302E310A00473239205332BA
:1007F000005370656369616C204D656E753A204EDB
:10080000657874204D65736820506F696E740A00B6
:10081000473239205331005370656369616C204D54
:10082000656E753A205374617274204D657368204B
:100830004C6576656C696E670A004D313430205323
:100840003630005370656369616C204D656E753A92
:100850002050726568656174204265640A004D35F8
:100860003031005370656369616C204D656E753A77
:10087000205265616420454550524F4D0A004D3568
:100880003030005370656369616C204D656E753A58
:10089000205361766520454550524F4D0A004D3337
:1008A000303320452D31205336302043362055310A
:1008B000005370656369616C204D656E753A204127
:1008C00075746F2054756E6520486F74626564207E
:1008D0005069640A004D31303620533137380A4DA3
:1008E00033303320453020533231302043362055C9
:1008F00031005370656369616C204D656E753A20F7
:100900004175746F2054756E6520486F74656E6410
:10091000205049440A003C5370656369616C5F4D27
:10092000656E753E003C5370656369616C5F4D6533
:100930006E753E002F002F002F002F2E2E0A002F45
:100940002E2E002F2E2E003C5370656369616C5F64
:100950004D656E753E0A003C5370656369616C209D
:100960004D656E753E003C5370656369616C204D4A
:10097000656E753E003C5265616420454550524F9E
:100980004D3E003C5265616420454550524F4D3EFE
:10099000003C4175746F2054756E6520486F746219
:1009A0006564205049443E003C4175746F20547585
:1009B0006E6520486F74626564205049443E003C77
:1009C0004175746F2054756E6520486F74656E6450
:1009D000205049443E003C4175746F2054756E654B
:1009E00020486F74656E64205049443E003C457851
:1009F00069743E003C457869743E003C53617665FD
:100A000020454550524F4D3E003C53617665204590
:100A10004550524F4D3E003C4E657874204D6573F5
:100A20006820506F696E743E003C4E657874204DAE
:100A300065736820506F696E743E003C5374617238
:100A400074204D657368204C6576656C696E673EF1
:100A5000003C5374617274204D657368204C657658
:100A6000656C696E673E003C507265686561742014
:100A70006265643E003C5072656865617420626521
:100A8000643E003C5A20446F776E20302E313E0089
:100A90003C5A20446F776E20302E313E003C5A2065
:100AA000446F776E20302E30323E003C5A20446F27
:100AB000776E20302E30323E003C5A205570203068
:100AC0002E30323E003C5A20557020302E30323EBF
:100AD000003C5A20557020302E313E003C5A2055A3
:100AE0007020302E313E0056313136004A333320EB
:100AF000004D3530300A4D3432302053310A473101
:100B0000205A313020463234300A473120583020C4
:100B10005930204636303030004A3232004A3232C4
:100B2000004731205A3520463234300A47312058A8
:100B3000313930205932302046363030300A473192
:100B4000205A302046323430004731205A35204672
:100B50003234300A47312058313930205931393058
:100B60002046363030300A4731205A302046323461
:100B700030004731205A3520463234300A47312080
:100B800058313930205932302046363030300A471B
:100B900031205A302046323430004739310A47314B
:100BA000205A313020463234300A4739300A473231
:100BB000380A4732390A473120583230205932300A
:100BC0002046363030300A4731205A302046323401
:100BD00030004A3032004A3132004731205A313039
:100BE000004F4B004731205A313000473930004721
:100BF00031204525694635303000473120452D30BC
:100C00002E314625690047312045302E3146256971
:100C1000004731205A2569462569004731205A2D61
:100C2000302E31462569004731205A302E31462575
:100C30006900473120592569462569004731205907
:100C40002D302E314625690047312059302E31464E
:100C5000256900473120582569462569004731201C
:100C6000582D302E314625690047312058302E311D
:100C7000462569004739310047323800473238206D
:100C80005A00473238205900473238205800413244
:100C9000305620004731205A3130004A3034004A63
:100CA0003231004A3230004B494C4C45442E200032
:100CB0004A303400454E4400464E20004A3032004F
:100CC0003939393A393939004D0048004137562011
:100CD00000413656202D2D2D004A30320041365627
:100CE00020005A3A2000593A2000583A2000413555
:100CF00056004134562000413356200041325620E0
:100D000000413156200041305620004D3834004A11
:100D10003136004A3138004739310A4731205A31DB
:100D20003020463234300A473930004A3134004AE4
:100D30003030004A3031004A31300024F4D4305091
:100D4000C38E20C2A24017828B7011127A910D813E
:100D50006CD90AA861E108C7586607615143061EAD
:100D60004B5D05C145A7041A411104093D98037163
:100D70003931034036DB0265339102D430540280AE
:100D80002E1D02632CEE01752AC501B028A00110AA
:100D90002781018F2564012B244B01E0223401AC13
:100DA000211F018D200D01801FFC00841EED009786
:100DB0001DDF00B81CD200E61BC600201BBC00646F
:100DC0001AB200B219A8000A19A0006A189900D135
:100DD00017910040178B00B516840031167E00B3C2
:100DE0001579003A157300C7146F0058146A00EEA5
:100DF0001366008813630025135E00C7125B006C46
:100E000012570015125400C111510070114F0021EA
:100E1000114B00D61049008D1047004610440002C7
:100E2000104200C00F4000800F3E00420F3C000601
:100E30000F3B00CB0E3800930E37005C0E350027B9
:100E40000E3400F30D3200C10D3100900D30006002
:100E50000D2E00320D2D00050D2C00D90C2B00AEEF
:100E60000C2900850C29005C0C2700350C27000E8E
:100E70000C2600E80B2400C40B2400A00B23007DEB
:100E80000B23005A0B2100390B2100180B2000F80E
:100E90000A1F00D90A1E00BB0A1E009D0A1D008001
:100EA0000A1D00630A1C00470A1B002C0A1B0011C4
:100EB0000A1A00F7091A00DD091900C4091900AB64
:100EC000091900920917007B091800630917004CE3
:100ED00009160036091600200916000A091500F542
:100EE000081500E0081400CC081400B8081400A489
:100EF000081400900813007D0812006B08130058B6
:100F000008120046081200340811002308110012CC
:100F100008110001081100F0071000E0071000D0D0
:100F2000071000C0071000B0070F00A107100091C4
:100F3000070E0083070F0074070F0065070E0057A8
:100F4000070E0049070E003B070D002E070E00207C
:100F5000070D0013070D0006070D00F9060C00ED44
:100F6000060D00E0060C00D4060C00C8060C00BC00
:100F7000060C00B0060C00A4060B0099060C008DB0
:100F8000060B0082060B0077060B006C060B006157
:100F9000060A0057060B004C060A0042060A0038F3
:100FA000060A002E060A0024060A001A060A001085
:100FB00006090007060A00FD050900F4050900EB13
:100FC000050900E2050900D9050900D0050900C797
:100FD000050900BE050900B5050800AD050800A516
:100FE0000509009C050800940508008C050800848C
:100FF0000508007C050800740508006C05070065FD
:101000000508005D050700560508004E0507004766
:101010000507004005080038050700310507002ACC
:10102000050700230507001C050600160507000F2D
:101030000507000805060002050700FB040600F589
:10104000040700EE040600E8040600E2040700DBE3
:10105000040600D5040600CF040600C9040600C338
:10106000040600BD040600B7040600B1040500AC88
:10107000040600A6040600A00405009B04060095D3
:10108000040500900406008A04050085040500801C
:101090000406007A04050075040500700405006B61
:1010A00004050066040500610405005C04050057A2
:1010B000040500520405004D0405004804050043E2
:1010C0000405003E0404003A040500350405003020
:1010D0000404002C04050027040400230405001E5A
:1010E0000404001A04040016040500110404000D91
:1010F000040400090405000404040000040400FCC6
:10110000030400F8030400F4030400F0030400ECFB
:10111000030400E8030400E4030400E0030400DC2B
:10112000030400D8030400D4030400D0030400CC5B
:10113000030400C8030300C503030024F404D920FA
:101140001BC40C5C0E9804C4095F0265077101F4AE
:1011500005F900FB04B30048048700C10369005887
:1011600003550003034500BE023A008402310053D8
:10117000022A002902250004022000E4011C00C804
:10118000011900AF011700980114008401130071C8
:101190000110006101100051010E0043010D0036E5
:1011A000010B002B010B0020010B00150109000CA5
:1011B00001090003010800FB000800F3000800EB30
:1011C000000700E4000600DE000600D8000600D29A
:1011D000000600CC000500C7000500C2000500BDE8
:1011E000000400B9000400B5000400B1000400AD23
:1011F000000400A9000400A5000300A20003009F52
:101200000004009B00030098000300950002009377
:10121000000300900003008D0002008B0003008893
:101220000002008600020084000300810002007FAB
:101230000002007D0002007B0002007900020077BE
:1012400000010076000200740002007200010071CB
:101250000002006F0002006D0001006C0002006AD5
:1012600000010069000200670001006600010065DE
:1012700000010064000200620001006100010060E2
:101280000001005F0002005D0001005C0001005BE6
:101290000001005A000100590001005800010057E8
:1012A00000010056000100550001005400010053E8
:1012B00000000053000100520001005100010050E5
:1012C0000001004F0001004E0000004E0001004DE3
:1012D0000001004C0001004B0000004B0001004ADF
:1012E00000010049000100480000004800010047DB
:1012F00000010046000000460001004500000045D6
:1013000000010044000100430000004300010042CE
:1013100000000042000100410000004100010040C7
:101320000001003F0000003F0001003E0000003EC1
:101330000001003D0000003D0001003C0000003CB9
:101340000000003C0001003B0000003B0001003AAF
:101350000000003A000100390000003900010038A7
:10136000000000380000003800010037000000379E
:101370000001003600000036000000360001003594
:10138000000000350000003500010034000000348A
:10139000000000340001003300000033000000337F
:1013A0000001003200000032000000320001003174
:1013B000000000310000003100010030000000306A
:1013C000000000300001002F0000002F0000002F5F
:1013D0000000002F0001002E0000002E0000002E53
:1013E0000001002D0000002D0000002D0000002D48
:1013F0000001002C0000002C0000002C0000002C3C
:101400000001002B0000002B0000002B0000002B2F
:101410000001002A0000002A0000002A0000002A23
:101420000001002900000029000000290000002917
:10143000000000290001002800000028000000280A
:1014400000000028000000280001002700000027FD
:1014500000000027000000270000002700010026F0
:1014600000000026000000260000002600000026E4
:1014700000010025000000250000002500000025D7
:1014800000000025000000250001002400000024C9
:1014900000000024000000240000002400010023BC
:1014A00000000023000000230000002300000023B0
:1014B00000000023000000230001002200000022A1
:1014C0000000002200000022000000220000002294
:1014D0000001002100000021000000210000002187
:1014E0000000002100000021000000210001002078
:1014F000000000200000002000000020000000206C
:101500000000002000000020000000200001001F5B
:101510000000001F0000001F0000001F0000001F4F
:101520000000001F0000001F0001001E0000001E40
:101530000000001E0000001E000000232C0000B868
:10154000220000561800003A0F0000B8080000B151
:10155000040000710200003E010000696E206D6F02
:1015600076655F746F282920666565645F76616CB7
:10157000756520666F722058593A002C2065793DB8
:101580000029202D3E202865783D002C2073793DD0
:101590000020436F6E6E656374696E6720776974AF
:1015A0006820766572746963616C206C696E652071
:1015B0002873783D002C2065793D0029202D3E20A0
:1015C0002865783D002C2073793D0020436F6E6EB6
:1015D000656374696E67207769746820686F7269E3
:1015E0007A6F6E74616C206C696E65202873783D2B
:1015F000003F53706563696669656420582C592003
:10160000636F6F7264696E617465206F7574206FAB
:101610006620626F756E64732E0A003F285229653A
:10162000706561742076616C7565206E6F742070D2
:101630006C61757369626C653B206D7573742062B3
:1016400065206174206C6561737420312E0A003F3F
:101650002852296570656174206D75737420626508
:1016600020737065636966696564207768656E20BC
:101670006E6F74207573696E6720616E204C4344F1
:101680002E0A003F537065636966696564206E6F5A
:101690007A7A6C652074656D7065726174757265B7
:1016A000206E6F7420706C61757369626C652E0AB0
:1016B000003F5370656369666965642066696C61A3
:1016C0006D656E742073697A65206E6F7420706C1E
:1016D00061757369626C652E0A003F5370656369BA
:1016E00066696564207072696D65206C656E6774EB
:1016F00068206E6F7420706C61757369626C652E02
:101700000A003F5072696D65206C656E67746820D1
:101710006D757374206265207370656369666965B1
:1017200064207768656E206E6F74207573696E67CC
:1017300020616E204C43442E0A003F53706563695C
:1017400066696564206E6F7A7A6C652073697A6564
:10175000206E6F7420706C61757369626C652E0AFF
:10176000003F5370656369666965642052657472F1
:10177000616374696F6E204D756C7469706C696516
:1017800072206E6F7420706C61757369626C652E67
:101790000A003F52657472616374696F6E204D7503
:1017A0006C7469706C696572206D75737420626504
:1017B000207370656369666965642E0A003F537023
:1017C00065636966696564206C6179657220686526
:1017D00069676874206E6F7420706C6175736962DC
:1017E0006C652E0A003F5370656369666965642005
:1017F0006265642074656D706572617475726520D0
:101800006E6F7420706C61757369626C652028342A
:10181000302D31343043292E0A0047323620636F91
:101820006D6D616E6420737461727465642E2057EF
:10183000616974696E6720666F722068656174659E
:10184000722873292E0A00024A3135004A313200CB
:101850004A3137002020506C616E6E6572427566A9
:1018600066657242797465733A2000204672656538
:10187000204D656D6F72793A2000436F6D70696C11
:1018800065643A2044656320323420323031380AAE
:1018900000207C20417574686F723A20286461765C
:1018A000696472616D69726F2C20666F7220416E7F
:1018B000796375626963206933204D656761290A20
:1018C00000323031382D31322D323400204C6173EA
:1018D0007420557064617465643A2000312E312E95
:1018E000390A004D61726C696E0020536F6674771F
:1018F0006172652052657365740A002057617463D4
:1019000068646F672052657365740A002042726FC5
:10191000776E206F75742052657365740A002045D8
:10192000787465726E616C2052657365740A00503C
:101930006F77657255700A0073746172740A004D96
:101940003234004D3233202573006175746F256980
:101950002E67006572726F722077726974696E67A4
:1019600020746F2066696C650A00205A3A0020597D
:101970003A0020583A00656E6473746F7073206883
:1019800069743A2000446F6E6520736176696E67F2
:101990002066696C652E0A004D32390020746F6F25
:1019A000206C6F6E6720657874727573696F6E2036
:1019B00070726576656E7465640A0020636F6C648E
:1019C00020657874727573696F6E207072657665C4
:1019D0006E7465640A00454550524F4D2064617431
:1019E0006173697A65206572726F722E0A00290A26
:1019F000002062797465733B206372632000536535
:101A00007474696E67732053746F72656420280064
:101A1000290A002062797465733B20637263200099
:101A20002073746F7265642073657474696E677374
:101A300020726574726965766564202800202863C9
:101A4000616C63756C6174656429210A0020213D15
:101A50002000454550524F4D20435243206D69733D
:101A60006D61746368202D202873746F726564291A
:101A700020002053697A653A2000496E6465783AFF
:101A80002000204D61726C696E3D563535290A0083
:101A900028454550524F4D3D00454550524F4D2031
:101AA00076657273696F6E206D69736D61746368BA
:101AB00020001000C90210012C0140012201700118
:101AC0001801B0010E01F00104015002FA00B00249
:101AD000F0003003E600D003DC009004D200700573
:101AE000C800A006BE000008B400B009AA00D00BD0
:101AF000A000600E960060118C0000158200201975
:101B00007800C01D6E00A0226400B0275A00902CFF
:101B1000500000314600E0343C0010383200903A6A
:101B20002800603C1E00A03D1400803E0A00203FBB
:101B300000002CFFFFFFFFFF0001010101016265B2
:101B4000640A002C2073797374656D2073746F7050
:101B500070656421204865617465725F49443A206C
:101B6000004265642068656174696E67206661691A
:101B70006C65640048656174696E67206661696CB4
:101B800065640045312048656174696E672066614F
:101B9000696C65640048656174696E672066616997
:101BA0006C65640070012C0190012701B0012201D5
:101BB000C0011D01F00118011002130130020E01D5
:101BC0006002090190020401C002FF000003FA0054
:101BD0004003F5008003F000D003EB002004E60092
:101BE0007004E100E004DC004005D700C005D2002D
:101BF0004006CD00D006C8008007C3003008BE00F4
:101C0000F008B900C009B400B00AAF00B00BAA00D8
:101C1000D00CA500000EA000500F9B00C010960035
:101C20005012910000148C00C0158700B01782007C
:101C3000B0197D00D01B7800001E730040206E009C
:101C400090226900F024640040275F0090295A0028
:101C5000E02B5500102E500020304B001032460073
:101C6000E033410090353C001037370070383200C7
:101C7000A0392D00B03A2800A03B2300603C1E0094
:101C8000103D1900903D1400103E0F00703E0A00F8
:101C9000C03E0500003F0000403FFBFF803FF6FFD5
:101CA000C03FF1FF453120544845524D414C205230
:101CB000554E415741590042454420544845524DE4
:101CC000414C2052554E4157415900546865726D40
:101CD000616C2052756E61776179004531204572E3
:101CE000723A204D415854454D50004572723A2089
:101CF0004D415854454D5020424544004D415854A3
:101D0000454D50207472696767657265640045319E
:101D1000204572723A204D494E54454D500045724F
:101D2000723A204D494E54454D5020424544004D95
:101D3000494E54454D5020747269676765726564F9
:101D4000004D383420582059205A204500202F00BB
:101D50002042403A0020403A006F70656E20666174
:101D6000696C65642C2046696C653A200043616E9D
:101D70006E6F74206F70656E207375626469722077
:101D8000004A3035004A3233004739310A473120A2
:101D90005A2D313020463234300A4739300053440E
:101DA0002063617264206F6B0A006F70656E526F02
:101DB0006F74206661696C65640A00766F6C756D7E
:101DC000652E696E6974206661696C65640A0045F8
:101DD00072726F723A00534420696E6974206661B2
:101DE000696C0A006563686F3A00656E71756575A8
:101DF00065696E672022004B494C4C45442E2000FB
:101E00005072696E7465722073746F7070656420AF
:101E100064756520746F206572726F72732E204630
:101E2000697820746865206572726F7220616E64D3
:101E300020757365204D39393920746F20726573B0
:101E4000746172742E202854656D706572617475AA
:101E500072652069732072657365742E20536574F2
:101E60002069742061667465722072657374617292
:101E700074696E67290A004E6F20436865636B734F
:101E8000756D2077697468206C696E65206E756D5C
:101E90006265722C204C617374204C696E653A2027
:101EA000004E6F20436865636B73756D20776974AE
:101EB00068206C696E65206E756D6265722C204CB1
:101EC000617374204C696E653A2000636865636BCA
:101ED00073756D206D69736D617463682C204C613E
:101EE0007374204C696E653A20004C696E65204E13
:101EF000756D626572206973206E6F74204C61731A
:101F000074204C696E65204E756D6265722B312CA4
:101F1000204C617374204C696E653A20004D31315C
:101F200030004D3331005344207265616420657286
:101F3000726F720A00446F6E65207072696E746908
:101F40006E672066696C650A00205A3A0020593A8B
:101F50000020436F756E7420583A0020453A0020E7
:101F60005A3A0020593A00583A003A004361703A10
:101F700000205A00205900580020204D61783A2056
:101F800000205A00205900580020204D696E3A2048
:101F9000004F6E20004F666600536F667420656EBA
:101FA0006473746F70733A20004B6420002364657F
:101FB00066696E652044454641554C545F004B6947
:101FC000200023646566696E652044454641554C92
:101FD000545F004B70200023646566696E65204481
:101FE000454641554C545F00504944204175746F3B
:101FF00074756E652066696E69736865642120502A
:10200000757420746865206C617374204B702C208B
:102010004B6920616E64204B6420636F6E73746142
:102020006E74732066726F6D2062656C6F772069C5
:102030006E746F20436F6E66696775726174696F45
:102040006E2E680A00504944204175746F74756E95
:1020500065206661696C6564212074696D656F75C2
:10206000740A00453120544845524D414C20525588
:102070004E415741590042454420544845524D4134
:102080004C2052554E4157415900546865726D615C
:102090006C2052756E617761790045312048656129
:1020A00074696E67206661696C65640042656420CE
:1020B00068656174696E67206661696C6564004873
:1020C000656174696E67206661696C65640050497A
:1020D00044204175746F74756E65206661696C6526
:1020E00064212054656D7065726174757265207429
:1020F0006F6F20686967680A00204B643A200020EF
:102100004B693A2000204B703A20000A20436C6152
:102110007373696320504944200A002054753A20A3
:1021200000204B753A2000206D61783A2000206D28
:10213000696E3A200020643A200020626961733A97
:102140002000504944204175746F74756E65206697
:1021500061696C65642120426164206578747275E0
:10216000646572206E756D6265720A005049442084
:102170004175746F74756E652073746172740A00B2
:102180004F66660A00466164652048656967687441
:102190002000426564204C6576656C696E6720009E
:1021A0004661696C656420746F20656E61626C6560
:1021B00020426564204C6576656C696E670A004D47
:1021C00065736820426564204C6576656C206461A7
:1021D00074613A0A004D65736820706F696E7420EF
:1021E00063616E6E6F74206265207265736F6C76CA
:1021F00065640A004D34323120696E636F72726516
:10220000637420706172616D6574657220757361AD
:1022100067650A007C3C3E5E2B3D3F2F5B5D3B2C9F
:102220002A225C00627573793A2070617573656467
:1022300020666F7220696E7075740A00627573791A
:102240003A2070617573656420666F7220757365DE
:10225000720A00627573793A2070726F63657373E6
:10226000696E670A004A3135004B494C4C45442E93
:1022700020004B494C4C2063617573656420627982
:10228000204B494C4C20627574746F6E2F70696ED0
:102290000A004B494C4C45442E20004B494C4C20E5
:1022A00063617573656420627920746F6F206D754A
:1022B000636820696E6163746976652074696D6511
:1022C000202D2063757272656E7420636F6D6D6171
:1022D0006E643A20004A3131005072696E74657242
:1022E0002068616C7465642E206B696C6C282920F1
:1022F00063616C6C6564210A000000A0C0000000EE
:1023000000000000005761726E696E673A20486FE6
:102310006D696E672042756D702044697669736FD0
:1023200072203C20310A000202040000A04000009C
:10233000A040000000400000614300005C4300003A
:102340004D43FFFFFF20496E76616C69642065781C
:1023500074727564657220000000A0C00000000067
:102360000000000000005C4300005C4300004D439F
:10237000486F6D696E67206661696C656400206EE8
:102380006F7420656E74657265642E0A0046696C10
:10239000652064656C657465643A0044656C6574B9
:1023A000696F6E206661696C65642C2046696C6596
:1023B0003A200050726F7465637465642050696ED2
:1023C0000A004A3036004A3034004A30370020577D
:1023D0003A004A3038004A30390020573A000000AD
:1023E0002100240027002A002D00300033000101C5
:1023F0000000040107010A01000022002500280056
:102400002B002E00310034000201000005010801FC
:102410000B01000020002300260029002C002F00C3
:102420003200000100000301060109010505050550
:10243000070508080808020202020A0A080804043C
:10244000040401010101010101010303030303036A
:102450000303040707070C0C0C0C0C0C0C0C0202F9
:10246000020206060606060606060B0B0B0B0B0BF6
:102470000B0B010210202008081020401020408083
:102480000201020108040201010204081020408038
:1024900080402010080402018004020180402010C6
:1024A000080402010804020101020408102040800F
:1024B000010204081020408000000A0B02090C0DE4
:1024C0000E080703040100000000000000000000E7
:1024D00000000000000000000000000000000000FC
:1024E00000000000121110000000000000000000B9
:1024F0000000000000000000000000000000556E19
:102500006B6E6F776E20636F6D6D616E643A202223
:10251000002066697273740A005A00590058004816
:102520006F6D6520000000484200004842000080B6
:102530004000000000545249474745524544006F4F
:1025400070656E003A20007A325F6D696E007A5FC6
:102550006D696E00795F6D696E00785F6D696E0000
:102560005265706F7274696E6720656E6473746F04
:1025700070207374617475730A000A4D6561737518
:1025800072656420706F696E74733A0A005A206F26
:1025900066667365743A20004E756D20582C593A62
:1025A00020352C350A000000000100000001000069
:1025B0008000555555000000400033333300AAAA6F
:1025C0002A004992240000002000C7711C0099993C
:1025D0001900D1451700555515003BB1130024498A
:1025E000120011111100000010000F0F0F00E3384E
:1025F0000E0043790D00CCCC0C00C3300C00E8A2D7
:102600000B0064210B00AAAA0A00703D0A009DD8A5
:102610000900427B090092240900DCD30800888865
:1026200008001042080000000800F0C1070087877A
:10263000070075500700711C07003EEB0600A1BCA7
:1026400006006990060066660600703E0600611886
:10265000060017F4050074D105005BB00500B290C8
:102660000500627205005555050078390500B81E51
:102670000500050505004EEC040087D40400A1BD4B
:10268000040090A7040049920400C17D0400EE6993
:102690000400C7560400444404005C3204000821CE
:1026A000040041100400000004003FF00300F8E0C3
:1026B000030026D20300C3C30300CCB503003AA82D
:1026C00003000A9B0300388E0300C08103009F753E
:1026D0000300D0690300505E03001D53030034481B
:1026E0000300913D03003333030016290300381F14
:1026F000030097150300300C0300030303000BFADB
:10270000020049F10200BAE802005CE002002DD8A4
:1027100002002DD0020059C80200B0C0020031B939
:102720000200DAB10200AAAA0200A0A30200BC9C27
:102730000200FA9502005C8F0200DF8802008282AC
:102740000200457C02002776020027700200436ADF
:1027500002007C640200D05E02003F590200C853B0
:10276000020048617264636F646564204465666159
:10277000756C742053657474696E6773204C6F6157
:102780006465640A00B80B0000B80B00003C000050
:1027900000102700000000FA430000FA430000C0C8
:1027A00040000070420000A0420000A0420000C8AB
:1027B000433333B94220286D6D290020204D393034
:1027C00030204B004C696E65617220416476616E09
:1027D00063653A0A0020440020490020204D333030
:1027E0003420500020440020490020204D33303157
:1027F0002050005049442073657474696E67733AC1
:102800000A00205A0020204D36363600456E64738B
:10281000746F702061646A7573746D656E743A0AC2
:1028200000205A00205900202047323920533320FD
:102830005800205A0020204D3432302053004D657E
:10284000736820426564204C6576656C696E673AF2
:102850000A00205A0020590020204D3230362058DE
:1028600000486F6D65206F66667365743A0A0020D4
:102870004500205A002059002058002054002053C1
:102880000020204D32303520510020453C6D6178CC
:102890005F655F6A65726B3E0020583C6D61785FD2
:1028A000785F6A65726B3E20593C6D61785F795F35
:1028B0006A65726B3E205A3C6D61785F7A5F6A652B
:1028C000726B3E00416476616E6365643A20513CF0
:1028D0006D696E5F7365676D656E745F74696D6554
:1028E0005F75733E20533C6D696E5F66656564720B
:1028F0006174653E20543C6D696E5F7472617665EB
:102900006C5F66656564726174653E0020540020EA
:10291000520020204D323034205000416363656CFA
:1029200065726174696F6E2028756E6974732F7398
:1029300032293A20503C7072696E745F616363653E
:102940006C3E20523C726574726163745F616363B4
:10295000656C3E20543C74726176656C5F616363A4
:10296000656C3E0A00204500205A002059002020B6
:102970004D3230312058004D6178696D756D2041C0
:102980006363656C65726174696F6E2028756E692A
:1029900074732F7332293A0A00204500205A002010
:1029A000590020204D3230332058004D6178696D38
:1029B000756D206665656472617465732028756E37
:1029C0006974732F73293A0A00204500205A0020A9
:1029D000590020204D3932205800537465707320FF
:1029E00070657220756E69743A0A0020204D32308D
:1029F000302044300A0020204D3230302044002066
:102A000044697361626C65640A0046696C616D6556
:102A10006E742073657474696E67733A0020204782
:102A20003231202020203B00FFFDFCFAF8F6F4F2C2
:102A3000F0EEECEAE9E7E5E3E1E0DEDCDAD9D7D570
:102A4000D4D2D0CFCDCBCAC8C7C5C3C2C0BFBDBC0E
:102A5000BAB9B7B6B4B3B2B0AFADACAAA9A8A6A57F
:102A6000A4A2A1A09E9D9C9A9998979594939290C8
:102A70008F8E8D8B8A8988878684838281807F7EF2
:102A80007D7B7A797877767574737271706F6E6DFD
:102A90006C6B6A696867666564636261605F5E5DEE
:102AA0005C5B5A5958585756555453525150504FD1
:102AB0004E4D4C4B4A4A494847464645444342429C
:102AC00041403F3E3E3D3C3B3B3A39383837363556
:102AD00035343332323130302F2E2E2D2C2B2B2A01
:102AE00029292827272625252423232221212020A0
:102AF0001F1E1E1D1C1C1B1B1A1919181817161631
:102B0000151514131312121111100F0F0E0E0D0DB7
:102B10000C0C0B0A0A090908080707060605050434
:102B20000403030202010000526573656E643A20DB
:102B3000006F6B0020746F6F206C6F6E672065787C
:102B400074727573696F6E2070726576656E7465E8
:102B5000640A0020636F6C64206578747275736911
:102B60006F6E2070726576656E7465640A004572DA
:102B7000726F722077726974696E6720746F204576
:102B80004550524F4D210A0057726974696E672093
:102B9000746F2066696C653A20006F70656E206600
:102BA00061696C65642C2046696C653A20006F7021
:102BB000656E206661696C65642C2046696C653AB7
:102BC000200046696C652073656C65637465640AF2
:102BD000002053697A653A200046696C65206F7061
:102BE000656E65643A20002066696C653A20006471
:102BF0006F696E67006672657368004E6F772000BC
:102C0000454E4420535542524F5554494E450A00B3
:102C10002220706F73002220706172656E743A22F8
:102C200000535542524F5554494E452043414C4C58
:102C3000207461726765743A22004B494C4C4544DC
:102C40002E2000747279696E6720746F2063616C46
:102C50006C207375622D67636F64652066696C65AF
:102C600073207769746820746F6F206D616E7920AE
:102C70006C6576656C732E204D4158206C657665C9
:102C80006C2069733A009ADF50E111241FBECFEF28
:102C9000D1E2DEBFCDBF00E00CBF14E0A0E0B2E0A7
:102CA000EAE5FCED01E00BBF02C007900D92A431F4
:102CB000B107D9F728E1A4E1B4E001C01D92A83C16
:102CC000B207E1F716E1C4E4D6E100E006C02197BF
:102CD0000109802FFE010E9485EDC334D10780E0F9
:102CE0000807A9F70E94FAD90C941CEE0C94000076
:102CF0002F923F924F925F926F927F928F929F920C
:102D0000AF92BF92CF92DF92EF92FF920F931F93F9
:102D1000CF93DF93CDB7DEB7CA58D1090FB6F89479
:102D2000DEBF0FBECDBF21E020933F10809115186C
:102D30008D3411F40C947621843511F40C949E2E6C
:102D4000873411F00C94EA2E809113189091141886
:102D50008A31910509F4BEC79CF4843091053CF496
:102D600082309105B4F597FF2DC00C947221843008
:102D7000910509F4D2C1059709F40EC20C94722191
:102D80008A32910511F40C9469204CF48C31910530
:102D900009F4A4C74D9709F4A6C70C9472218B358A
:102DA000910511F40C94F4208C35910511F40C94D8
:102DB000F8208A35910511F00C94722110922704A5
:102DC0000C94EC2E8091270281110C94F12E0C941E
:102DD000EC2E20912702222311F40C94EC2E11E00A
:102DE000029709F010E00E94ACAA19821A821B8295
:102DF0001C821D821E821F82188682E50E94974CCB
:102E0000882309F43AC10E94174C4B015C0120E071
:102E100030E0A9010E943DE6882309F444C1C09036
:102E20003204D0903304E0903404F0903504CCAAFE
:102E3000DDAAEEAAFFAAC0903604D0903704E09035
:102E40003804F0903904C8AED9AEEAAEFBAEC090FB
:102E5000AE10D090AF10E090B010F090B110CCAEAA
:102E6000DDAEEEAEFFAEC090B210D090B310E090E9
:102E7000B410F090B5102496CCAEDDAEEEAEFFAE41
:102E800024972CAD3DAD4EAD5FAD6CA97DA98EA94B
:102E90009FA90E943DE681110BC0A701960168AD74
:102EA00079AD8AAD9BAD0E943DE6882309F4FBC055
:102EB00020E030E0A901C501B4010E943DE6881F71
:102EC0008827881F181739F0C12CD12C80E8E82EEC
:102ED0008FEBF82E06C0C12CD12C00E8E02E0FE3BA
:102EE000F02E2C96CCAEDDAEEEAEFFAE2C972CA91C
:102EF0003DA94EA95FA96CAD7DAD8EAD9FAD0E9481
:102F000088EA28966CAF7DAF8EAF9FAF289728AD2B
:102F100039AD4AAD5BAD24966CAD7DAD8EAD9FAD48
:102F200024970E9488EA6B017C0128962CAD3DAD68
:102F30004EAD5FAD2897CA01B9010E94A2E62B01F0
:102F40003C01A7019601C701B6010E94A2E69B01C0
:102F5000AC01C301B2010E9489EA0E94F4EC2B018A
:102F60003C0120E030E040E05FE30E94A2E6609692
:102F70006CAF7DAF8EAF9FAF6097A5019401C50187
:102F8000B4010E94A2E64B015C0160962CAD3DAD00
:102F90004EAD5FAD6097CA01B9010E94A2E69B01E8
:102FA000AC01C501B4010E9488EA0E94F4EC2C96A1
:102FB0002CAD3DAD4EAD5FAD2C970E94A2E64B010E
:102FC0005C01C701B6019058A30192010E9465EB14
:102FD000A50194010E94A2E66B017C012CAD3DADE0
:102FE0004EAD5FAD6CA97DA98EA99FA90E9489EA0B
:102FF00020E030E040E05FE30E94A2E69B01AC01EC
:10300000C701B6010E9489EA2CA93DA94EA95FA972
:103010000E9488EA69837A838B839C8324962CADF3
:103020003DAD4EAD5FAD249768AD79AD8AAD9BAD3A
:103030000E9489EA20E030E040E05FE30E94A2E6DF
:103040006B017C01A301920128966CAD7DAD8EAD24
:103050009FAD28970E9465EBA50194010E94A2E60E
:103060009B01AC01C701B6010E9489EA28AD39ADC8
:103070004AAD5BAD0E9488EA12C089E40E94974C79
:10308000882331F00E94174C69837A838B839C8359
:103090008AE40E94974C882331F00E94174C6D837C
:1030A0007E838F83988720E030E0A90169817A814F
:1030B0008B819C810E943DE681110EC020E030E0B2
:1030C000A9016D817E818F8198850E943DE68111E5
:1030D00003C0EFECFDE10DC0412FBE016F5F7F4FDC
:1030E0008EEA90E10E94CEA40C94EC2E0E94CC8932
:1030F000F80184918F010F5F1F4F8111F7CFEDE130
:10310000F2E084918F010F5F1F4F882311F40C941C
:10311000EC2E0E94CC89F801F4CF80E50E94974CF8
:10312000882379F08091210490912204009749F03E
:103130004AE050E060E070E00E94BCE46B017C017A
:1031400003C0C12CD12C760183E50E94974C8823C3
:1031500061F00E94174C20E030E04AE754E40E94FE
:10316000A2E60E94D2EB6B017C010E941E6A0E94C3
:10317000FE58C60ED71EE81EF91E0E94FE58DC013E
:10318000CB018C199D09AE09BF09B7FD02C00C9493
:10319000EC2E0E9402A1F1CF80912702882311F426
:1031A0000C94EC2E0E94ACAA89E40E94974C8823D0
:1031B00029F00E94174C2B013C0103C0412C512CDB
:1031C00032018AE40E94974C882329F00E94174C10
:1031D0004B015C0103C0812C912C540180E50E94BD
:1031E000974C882329F00E94174C6B017C0103C087
:1031F000C12CD12C760181E50E94974C882339F0AF
:103200000E94174C6CAB7DAB8EAB9FAB04C01CAA6D
:103210001DAA1EAA1FAA20913E10C657DF4F288361
:10322000CA58D0406091020270910302072E000C30
:10323000880B990B0E9443E62091300230913102B5
:1032400040913202509133020E94A2E62AE037ED0B
:1032500043E25CE30E94A2E668AB79AB8AAB9BAB2E
:1032600040913204509133046091340470913504DC
:1032700048AF59AF6AAF7BAF9A01AB01C301B2014E
:103280000E9489EAA1966CAF7DAF8EAF9FAFA197E8
:1032900040903604509037046090380470903904A0
:1032A000A3019201C501B4010E9489EAA5966CAF01
:1032B0007DAF8EAF9FAFA5972091AE103091AF102C
:1032C0004091B0105091B110C701B6010E9489EA37
:1032D000A9966CAF7DAF8EAF9FAFA9972091B2102A
:1032E0003091B3104091B4105091B5106CA97DA9E4
:1032F0008EA99FA90E9489EAAD966CAF7DAF8EAF73
:103300009FAFAD97C8ACD9ACEAACFBACC982DA824E
:10331000EB82FC824D825E826F8278860E94FE582C
:103320009B01AC0128533F4F4F4F5F4FCB57DF4FAF
:10333000288339834A835B83C558D040BDEC8B2EEC
:10334000BCEC9B2EA92CBDE3BB2E25961FAE25976A
:1033500029961FAE29972D961FAE2D9761961FAE09
:1033600061970E94CF7B0E94FE588B019C01CB5736
:10337000DF4FC880D980EA80FB80C558D0400C1947
:103380001D092E093F0937FD10C09B01AC012853D0
:103390003F4F4F4F5F4FCB57DF4F288339834A83CF
:1033A0005B83C558D0400E9402A125967FAD25972A
:1033B00029966FAD29972D969FAD2D9761968FAD6C
:1033C0006197272F362F492F582FC501B4010E942E
:1033D00089EA6CAB78AF8CAF21969FAF219720E044
:1033E00030E040E85FE30E94AFEC181644F41CAAFA
:1033F00018AE30E83CAF4FE321964FAF2197609174
:10340000AE107091AF108091B0109091B110E19614
:103410006CAF7DAF8EAF9FAFE197809132049091FA
:103420003304A0913404B0913504E5968CAF9DAF80
:10343000AEAFBFAFE59721969FAD21979F93ACADFF
:10344000AF93B8ADBF93ECA9EF93E196ACACBDAC34
:10345000CEACDFACE197A996ECACFDAC0EAD1FADE8
:10346000A997A1962CAD3DAD4EAD5FADA197E59668
:103470006CAD7DAD8EAD9FADE5970E9488C50F9078
:103480000F900F900F9062966FAF629763967FAF29
:10349000639764968FAF649765969FAF6597C0906A
:1034A000B210D090B310E090B410F090B510E9963F
:1034B000CCAEDDAEEEAEFFAEE99720913604309192
:1034C00037044091380450913904ED962CAF3DAF4C
:1034D0004EAF5FAFED9721963FAD21973F934CAD37
:1034E0004F9358AD5F936CA96F93E996ACACBDACAC
:1034F000CEACDFACE997AD96ECACFDAC0EAD1FAD3C
:10350000AD97A5962CAD3DAD4EAD5FADA597ED96B3
:103510006CAD7DAD8EAD9FADED970E9488C50F90CF
:103520000F900F900F9066966FAF669767967FAF7C
:10353000679768968FAF689769969FAF69978981FB
:103540009A81AB81BC81C358DF4F88839983AA835A
:10355000BB83CD57D040CD80DE80EF80F884CF573D
:10356000DF4FC882D982EA82FB82C158D0406A9676
:103570001FAE6A9725967FAD259729966FAD29973F
:103580002D969FAD2D9761968FAD6197272F362F82
:10359000492F582FBCA9A8ADFCAD2196EFAD2197BE
:1035A0006B2F7A2F8F2F9E2F0E9488EA2FE632E111
:1035B00043E05BE30E943DE687FD29C125967FAD90
:1035C000259729966FAD29972D969FAD2D976196DA
:1035D0008FAD6197272F362F492F582FBCA9A8AD43
:1035E000FCAD2196EFAD21976B2F7A2F8F2F9E2F59
:1035F0000E9489EA20E030E040E05FE30E94A2E61A
:10360000662E972E882E792E9F938F937F936F939C
:10361000E196ACACBDACCEACDFACE197A996ECAC1E
:10362000FDAC0EAD1FADA997A1962CAD3DAD4EAD35
:103630005FADA197E5966CAD7DAD8EAD9FADE59785
:103640000E9488C50F900F900F900F906B966FAFF0
:103650006B976C967FAF6C976D968FAF6D97C757D2
:10366000DF4F9883C958D0407F928F929F926F927C
:10367000E996ACACBDACCEACDFACE997AD96ECACAA
:10368000FDAC0EAD1FADAD97A5962CAD3DAD4EADCD
:103690005FADA597ED966CAD7DAD8EAD9FADED9711
:1036A0000E9488C50F900F900F900F90162F072F34
:1036B000B82EA92E66962FAD669767963FAD679791
:1036C00068964FAD689769965FAD6997CF57DF4FA2
:1036D000688179818A819B81C158D0400E9489EAA2
:1036E00020E030E040E05FE30E94A2E61B012C01F5
:1036F00062962FAD629763963FAD639764964FAD28
:10370000649765965FAD6597C358DF4F688179818F
:103710008A819B81CD57D0400E9489EA20E030E029
:1037200040E05FE30E94A2E69B01AC016B966FADA7
:103730006B976C967FAD6C976D968FAD6D97C757F5
:10374000DF4F9881C958D0400E9488EA6B017C0104
:1037500020E030E0A9010E94AFEC87FF04C0F7FA37
:10376000F094F7F8F094A2019101612F702F8B2D46
:103770009A2D0E9488EA1B012C0120E030E0A9016B
:103780000E94AFEC87FF04C057FA509457F850944A
:10379000A2019101C701B6010E9489EA2DEC3CEC1F
:1037A0004CEC5DE30E943DE618168CF566961FAF63
:1037B000669767960FAF67976896BFAE68976996EA
:1037C000AFAE69976B96DFAC6B976296DFAE629790
:1037D0006C96EFAC6C976396EFAE63976D96FFAC0B
:1037E0006D976496FFAE6497C757DF4F2881C9581D
:1037F000D04065962FAF65976CAA98AE8CAE219697
:103800007FAE219731E06A963FAF6A97B3CE6A9652
:103810004FAD6A97411144C125967FAD25972996F2
:103820006FAD29972D969FAD2D9761968FAD6197BE
:10383000272F362F492F582FBCA9A8ADFCAD2196B4
:10384000EFAD21976B2F7A2F8F2F9E2F0E9488EA42
:103850006B017C012DEC3CEC4CEC5DE30E94AFEC89
:1038600018160CF41DC1A7019601C701B6010E94EC
:1038700089EA2596EFAD25972996BFAD29972D9614
:10388000AFAD2D976196FFAD61972E2F3B2F4A2F3D
:103890005F2F0E9489EA662E972E882E792E20E0CF
:1038A00030E040E85FE30E94AFEC87FFF9C07F9211
:1038B0008F929F926F92E196ACACBDACCEACDFAC78
:1038C000E197A996ECACFDAC0EAD1FADA997A19602
:1038D0002CAD3DAD4EAD5FADA197E5966CAD7DAD28
:1038E0008EAD9FADE5970E9488C50F900F900F9009
:1038F0000F906A966FAF6A976B967FAF6B976C96D7
:103900008FAF6C976D969FAF6D977F928F929F92BE
:103910006F92E996ACACBDACCEACDFACE997AD969E
:10392000ECACFDAC0EAD1FADAD97A5962CAD3DAD8D
:103930004EAD5FADA597ED966CAD7DAD8EAD9FADF7
:10394000ED970E9488C50F900F900F900F90162F43
:10395000072FB82EA92E262F372F482F592FCF5794
:10396000DF4F688179818A819B81C158D0400E9454
:1039700089EA20E030E040E05FE30E94A2E66B01CC
:103980007C016A962FAD6A976B963FAD6B976C96EC
:103990004FAD6C976D965FAD6D97C358DF4F6881E3
:1039A00079818A819B81CD57D0400E9489EA20E0AD
:1039B00030E040E05FE30E94A2E69B01AC0162962A
:1039C0006FAD629763967FAD639764968FAD649792
:1039D00065969FAD65970E9488EA1B012C0120E047
:1039E00030E0A9010E94AFEC87FF04C057FA509461
:1039F00057F85094A701960166966FAD6697679643
:103A00007FAD679768968FAD689769969FAD699708
:103A10000E9488EA6B017C0120E030E0A9010E944D
:103A2000AFEC87FF04C0F7FAF094F7F8F094A20126
:103A30009101C701B6010E9489EA2DEC3CEC4CECE7
:103A40005DE30E94AFEC18165CF166961FAF6697B7
:103A500067960FAF67976896BFAE68976996AFAEE7
:103A600069976A965FAD6A9762965FAF62976B9649
:103A70006FAD6B9763966FAF63976C967FAD6C97E6
:103A800064967FAF64976D968FAD6D9765968FAF97
:103A900065976CAA98AE8CAE21967FAE2197BCCE6E
:103AA00025967FAD259729966FAD29972D969FADC9
:103AB0002D9761968FAD6197272F362F492F582F5D
:103AC000BCA9A8ADFCAD2196EFAD21976B2F7A2F45
:103AD0008F2F9E2F0E9488EA4B015C0162968FAD6A
:103AE000629763969FAD63976496AFAD6497659652
:103AF000BFAD659789839A83AB83BC8366968FAD90
:103B0000669767969FAD67976896AFAD6897699619
:103B1000BFAD69978D839E83AF83B8877CA968AD5D
:103B20009CAD21968FAD2197272F362F492F582FE7
:103B300060E070E080E89FE30E9488EA6B017C010E
:103B400020913A0430913B0440913C0450913D0453
:103B50000E94A2E62B013C012091B6103091B710D3
:103B60004091B8105091B910BCA9A8ADFCAD2196F8
:103B7000EFAD21976B2F7A2F8F2F9E2F0E94A2E6F9
:103B80009B01AC01C301B2010E9489EA69877A876F
:103B90008B879C8720913E0430913F0440914004E4
:103BA00050914104C701B6010E94A2E66B017C015D
:103BB0002091BA103091BB104091BC105091BD10B3
:103BC000BCA9A8ADFCAD2196EFAD21976B2F7A2F44
:103BD0008F2F9E2F0E94A2E69B01AC01C701B60168
:103BE0000E9489EA6D877E878F87988BCE01019628
:103BF0000E94C5C91CA61DA61EA61FA689819A8162
:103C0000AB81BC8188A399A3AAA3BBA38D819E810C
:103C1000AF81B8858CA39DA3AEA3BFA389859A85E8
:103C2000AB85BC8588A799A7AAA7BBA7AE01485DAD
:103C30005F4FBE016C5D7F4FCE0180960E94C8BC75
:103C4000DE019C966D01C657DF4FE880CA58D04010
:103C50008E01005D1F4F9E01235F3F4FAE01485D07
:103C60005F4FBE016C5D7F4FCE0180960E94FA5976
:103C7000882329F120E030E040E85FE3BCA9A8AD4B
:103C8000FCAD2196EFAD21976B2F7A2F8F2F9E2FB2
:103C90000E943DE687FF13C03CA925963FAF2597BC
:103CA00048AD29964FAF29975CAD2D965FAF2D9704
:103CB00021966FAD219761966FAF619752CB80E1EE
:103CC000EEEAF0E1A2E3B4E001900D928A95E1F70B
:103CD0000C94EC2E0E94344E0C94EC2E80E00E944A
:103CE0004CAC0C94EC2E83E50E94974C882321F178
:103CF0000E94F74B182F863070F0E5EEF2E08491C9
:103D00008F010F5F1F4F882311F40C94EC2E0E943B
:103D1000CC89F801F4CF833009F44AC130F4813002
:103D200091F1823009F43FC008C0843009F49FC18A
:103D3000853009F4ACC101C010E00E94FFAB8111D5
:103D400003C0E5ECF2E013C080917C10882319F0E9
:103D500063E173E002C067E173E08DEB92E00E94E3
:103D60006DC58AE00E94CC890E9402BD96C18491F3
:103D70007F01BFEFEB1AFB0A882309F48EC10E9472
:103D8000CC89F701F4CF0E94B5BD109201021092C8
:103D9000000282EB92E09093A4078093A3070E9415
:103DA000F8890C94EC2E809100029091010297FF0B
:103DB0000EC0E9E8F2E084918F010F5F1F4F882366
:103DC00011F40C94EC2E0E94CC89F801F4CF0097EA
:103DD000A1F4809152028093280419821A821B82D6
:103DE0001C8218A219A21AA21BA2BE016F5F7F4FEC
:103DF000CE0180960E944BB427C0815065E00E949E
:103E000051ED80FF03C024E0291B922F25E0920290
:103E1000F0011124E80FF11D87FDFA95EE0FFF1F49
:103E2000EE0FFF1FEA53FF4E80913A0490913B043E
:103E3000A0913C04B0913D0480839183A283B3831D
:103E40008091280480935202809100029091010297
:103E5000893191050CF067C0109252029C012F5FCE
:103E60003F4F309301022093000265E00E9451ED24
:103E700080FF03C024E0291B922F40913A04509107
:103E80003B0460913C0470913D0448A359A36AA38C
:103E90007BA319821A821B821C8244E08402900157
:103EA0001124B9016751764F4B01DB012D913D91F2
:103EB0004D915C91B4E09B02C0011124FC01E350E0
:103EC000F64F5F016081718182819381DE011196DD
:103ED0006D01E12CF12C00EA10E40E947EB31982FE
:103EE0001A821B821C82B601CE0180960E944BB4BE
:103EF000F50180819181A281B381809332049093F6
:103F00003304A0933404B0933504F401808191818B
:103F1000A281B3818093360490933704A093380430
:103F2000B0933904BCC080E090E0A0EAB0E4809394
:103F30003A0490933B04A0933C04B0933D040E9448
:103F40003FAD0E941E6A8FEF9FEF90930102809316
:103F50000002E5E7F2E084918F010F5F1F4F882395
:103F600021F00E94CC89F801F6CF83E992E09A8390
:103F7000898304E610E019A308A3BE016F5F7F4F99
:103F8000CE0180960E9466B58AEB92E09A8389837F
:103F900019A308A3BE016F5F7F4FCE0180960E94D8
:103FA00066B581E00E944CAC81E00E942CAC77C0E9
:103FB00088E50E94974C8823A1F00E94E74B1FEFF1
:103FC000160F1530A8F0EEE5F2E084918F010F5F37
:103FD0001F4F882311F40C94EC2E0E94CC89F80119
:103FE000F4CF88E50E94CC890E948CE10C94EC2EE1
:103FF00089E50E94974C8823A1F00E94E74B0FEFC0
:10400000060F0530A8F0E7E4F2E084918F010F5F1E
:104010001F4F882311F40C94EC2E0E94CC89F801D8
:10402000F4CF89E50E94CC890E948CE10C94EC2E9F
:104030008AE50E94974C882399F00E94174C25E04E
:10404000129FF0011124E00FF11DEE0FFF1FEE0F84
:10405000FF1FEA53FF4E608371838283938335C0D1
:104060008AE50E94CC890E948CE10C94EC2E8AE5B2
:104070000E94974C8823A1F30E94174C6093C210B2
:104080007093C3108093C4109093C5101EC080E03D
:104090000E942CAC0E94B5BD18C01230B1F46091E2
:1040A0000002709101026931710514F069E170E05C
:1040B00088E392E00E9454C569E170E083E392E0F6
:1040C0000E9454C58AE00E94CC890E944B950C94B2
:1040D000EC2E80912702882311F40C94EC2E89E4B5
:1040E0000E94974CE82E882321F00E94E74B062F70
:1040F00001C000E08AE40E94974CF82E882321F04A
:104100000E94E74B162F01C010E0EE2011F00530A1
:1041100020F4FF2081F0153070F0ECEFF2E0849194
:104120008F010F5F1F4F882311F40C94EC2E0E9417
:10413000CC89F801F4CF0E94A34CEE2091F034E03A
:104140000302F0011124E350F64F80819181A28196
:10415000B3818093AE109093AF10A093B010B09342
:10416000B110FF2091F044E01402F0011124E75156
:10417000F64F80819181A281B3818093B210909398
:10418000B310A093B410B093B51080E50E94974C83
:10419000882319F00E94084C03C080E50E944E4C11
:1041A00086E40E94974C8823D9F00E94174C6B013B
:1041B0007C0120E030E0A9010E94AFEC181684F4E5
:1041C00020E030E040E752E4C701B6010E9465EB11
:1041D00060933002709331028093320290933302E5
:1041E0000E945CCA0C94EC2E209327040C94EC2EB5
:1041F00097E5292E92E0392E2DE4E22E20E1F22ED1
:1042000062E374E07DAB6CAB34E1C32E34E0D32EBB
:1042100000E010E0D1018D911D010E94974C882390
:1042200009F44BC00E94174C2B013C01133049F09C
:10423000F60120813181428153810E9488EA2B015D
:104240003C01ACA9BDA92D913D914D915C91C3015B
:10425000B2010E9488EA4B015C012DEB37E346E88E
:1042600055EB0E94AFEC87FD0AC02DEB37E346E823
:1042700055E3C501B4010E943DE61816F4F413306D
:1042800051F440923E0450923F0460924004709278
:10429000410401E012C0A5019401F7016081718120
:1042A000828193810E9489EAD7016D937D938D93DA
:1042B0009C931397812F0E9496AD1F5FB4E0EB0E85
:1042C000F11CECA9FDA93496FDABECABF4E0CF0EEC
:1042D000D11C143009F09ECF002309F4F6CE0E94C1
:1042E0001AB3F3CE0E949AB50C94EC2E8091131859
:1042F000909114188537910511F40C94EC2E0CF064
:10430000C0C08C34910509F43CC40CF058C08A310B
:10431000910509F42EC224F58531910509F4E7C110
:1043200084F48231910509F4A9C58431910509F419
:104330009EC1419711F00C949B2E0E94C3A40C9433
:10434000EC2E8731910509F4DCC10CF4D4C188311D
:10435000910509F4ECC1499709F4F4C10C949B2E22
:104360008F31910509F401C39CF48C31910509F456
:10437000A6C20CF40CC28D31910511F40C94EC2EF4
:104380004E9711F00C949B2E0E9415B00C94EC2EBD
:104390008A32910509F49CC32CF4809709F499C2E0
:1043A0000C949B2E8133910509F4C6C38B3491057F
:1043B00011F00C949B2E0E94C3780C94EC2E8A363C
:1043C000910509F40AC5B4F58435910509F456C57B
:1043D000E4F48135910509F42CC54CF48D34910534
:1043E00011F00C949B2E0E94FA780C94EC2E8235DE
:1043F000910509F440C58335910511F00C949B2E6D
:1044000081E0809326040C94EC2E8C35910509F400
:104410007BC534F48535910509F45DC50C949B2E5C
:104420008836910509F4B1C38936910509F475C43C
:104430000C949B2E8F36910509F4E3C384F48C36DB
:10444000910509F431C40CF4E4C48D36910509F4E6
:10445000A6C48E36910509F4C1C30C949B2E8137F6
:10446000910509F42DC40CF423C48237910509F495
:10447000D3C58337910511F00C949B2EE3EEF4E045
:1044800008C68E3221E0920711F40C94D72C0CF060
:1044900071C08B3C910509F416C7CCF58C38910599
:1044A00009F481C4ACF48737910509F49AC60CF479
:1044B0004BC68837910509F497C68937910511F0E5
:1044C0000C949B2E10923705109236050C94EC2E0E
:1044D0008E3B910509F47DC434F48B39910509F4C0
:1044E00037C40C949B2E883C910509F483C6893C03
:1044F000910511F00C949B2EF7E5EF2EF2E0FF2EC4
:104500000FE411E1AFE5CA2EA1E1DA2EC3C68C3D5E
:10451000910511F40C946A2B9CF48D3C910509F4DF
:1045200063C70CF4ECC68E3C910509F4EAC7833DE1
:10453000910511F00C949B2E0E9437940C94EC2E54
:10454000823E910511F40C94E52B3CF48D3D9105D0
:1045500011F40C94772B0C949B2E8C3241E0940731
:1045600011F40C940E2C8D32914011F40C94372CD4
:104570000C949B2E853F61E0960711F40C94C42D9A
:10458000DCF58A39A1E09A0709F496C3BCF48033BC
:10459000E1E09E0711F40C942E2D14F40C942B2DB5
:1045A000833621E0920709F45EC08039914011F012
:1045B0000C949B2E0E941E6A0C94EC2E853A41E0CE
:1045C000940711F40C94C12D4CF4843A914011F0ED
:1045D0000C949B2E0E9415960C94EC2E8C3A71E054
:1045E000970709F4B1C7843F914011F00C949B2EBA
:1045F0000E9465700C94EC2E8A39B2E09B0711F48E
:104600000C94032EB4F4873FF1E09F0711F40C944F
:10461000CA2D14F40C94C72D883F31E0930711F490
:104620000C94D62D8C30924011F40C94FA2D0C94ED
:104630009B2E8B3853E0950711F40C94EC2E3CF430
:104640008438934011F40C94302E0C949B2E803AB5
:10465000A3E09A0709F47CC1873E934011F40C94BF
:10466000882E0C949B2EEFECFDE10C94AE2DEAE22B
:10467000F3E084918F010F5F1F4F882321F00E9488
:10468000CC89F801F6CF1092AF0C82E69AE00E9436
:104690003C9A8BE1E2E6FAE0DE01159601900D927C
:1046A0008A95E1F78091600A9091610A9C838B83DF
:1046B0008DEE92E09A83898340E050E0BE016F5F07
:1046C0007F4F80E090E00E94E982CE0101960E9437
:1046D00098A0EBE1F3E084918F010F5F1F4F8823D7
:1046E00011F40C94EC2E0E94CC89F801F4CF0E94B6
:1046F000BB800C94EC2E1092310A1092320A0C946A
:10470000EC2EE0911118F09112188081882329F085
:10471000803209F410823196F8CF40E061E0809158
:104720001118909112180E948BD50C94EC2E809148
:10473000320A882319F081E08093310A0E94C378FD
:104740000C94EC2E1092310A80912B07813011F0DD
:104750000C94EC2E82E080932B070E94FE5860930D
:104760002707709328078093290790932A070C94B2
:10477000EC2E8091320A882311F40C94EC2E83E500
:104780000E94974C81110C94F62E0C94EC2E83E42D
:104790000E944E4C882309F450C0E8E6F3E084916F
:1047A0008F010F5F1F4F882321F00E94CC89F801F1
:1047B000F6CF8091FD0B811103C0EBE3F3E012C053
:1047C000BE016F5F7F4F8AEF9BE00E9404998E01CC
:1047D0000F5F1F4FF80181918F01882349F10E94DB
:1047E000CC89F8CF84918F010F5F1F4F882301F18F
:1047F0000E94CC89F801F6CF06EDC02E03E0D02E42
:10480000E12CF12C20E08091100790E00E2C02C0EA
:10481000959587950A94E2F780FD23C2BFEFEB1AC6
:10482000FB0AE2E0CE0ED11CF5E0EF16F10459F7D9
:104830008AE00E94CC890C94EC2E8091320A882365
:1048400039F08091310A882319F0E5E4F3E003C0E0
:10485000E7E5F3E028C084918F010F5F1F4F8823A5
:1048600021F00E94CC89F801F6CF6091AB0C7091D9
:10487000AC0C8091AD0C9091AE0C4AE00E94EF8C94
:104880008FE20E94CC896091A70C7091A80C809156
:10489000A90C9091AA0C4AE00E94EF8C8AE00E9439
:1048A000CC890C94EC2E84918F010F5F1F4F8823CD
:1048B00011F40C94EC2E0E94CC89F801F4CF40E066
:1048C00060E080911118909112180E948BD50C9481
:1048D000EC2E8091310A81110E941E6A8091320A69
:1048E000882311F40C94EC2E80E50E94974C8823C9
:1048F00019F00E94084C03C080E50E944E4C182F0E
:10490000482F61E080911118909112180E948BD568
:1049100083E50E94974C882381F00E94E74BAB010E
:10492000BC014093AB0C5093AC0C6093AD0C7093F6
:10493000AE0C8AEF9BE00E94F5978091320A8823A3
:1049400019F081E08093310A11110C94EC2EF6CE0F
:10495000809111189091121821E02093300A40E0C4
:1049600060E00E948BD50C94EC2E0E9474787B0141
:104970008C0120E831E541E050E00E942BEAC901BA
:104980006DE671E00E945EED4B015C01C801B7016C
:1049900020E13EE040E050E00E942BEACA01B9016C
:1049A00028E130E040E050E00E942BEA762E672EAE
:1049B000C62ED72E8CE3282E312C412C512CC80129
:1049C000B701A20191010E942BEAF62EE72ECA013F
:1049D000B901A20191010E942BEACB018E010F5F68
:1049E0001F4F81149104D1F0EF92FF927F936F9348
:1049F0006F927F92BF92AF929F928F928FE993E0D6
:104A00009F938F931F930F930E940FE60FB6F89416
:104A1000DEBF0FBECDBFE4EEFDE145C0A114B10481
:104A200089F0EF92FF927F936F936F927F92BF9284
:104A3000AF928FE893E09F938F931F930F930E9401
:104A40000FE6E4CFCD2879F0EF92FF927F936F933A
:104A50006F927F9283E893E09F938F931F930F93BE
:104A60000E940FE6D3CF892B69F0EF92FF927F93DC
:104A70006F938BE793E09F938F931F930F930E9405
:104A80000FE6C4CFEF92FF9287E793E09F938F9357
:104A90001F930F930E940FE60F900F900F900F90AF
:104AA0000F900F90B8CF84917F019FEFE91AF90A18
:104AB000882321F00E94CC89F701F5CFB80183EB60
:104AC00093E00E946DC58AE00E94CC890C94EC2E84
:104AD00083E50E94974C882311F40C94EC2E0E94DD
:104AE000F74BE82E80E50E94974C882339F00E940E
:104AF000F74B182F87FF03C00C94EC2E1DE089E4C0
:104B00000E94974C882341F00E94084C81110C941C
:104B1000722FEBE1F6E00BC089E40E944E4CF6CF19
:104B20003196A6E0EB34FA0711F40C94722F8491BD
:104B30001813F6CF0C94472FF090200481E0F8264C
:104B4000F0922004EBECF3E084918F010F5F1F4F94
:104B5000882321F00E94CC89F801F6CFFF2019F0BC
:104B6000E0ECF3E002C0E5ECF3E084918F010F5F2D
:104B70001F4F882311F40C94EC2E0E94CC89F8016D
:104B8000F4CF0E94E5780C94EC2E88E690E00E9429
:104B9000D6AD81110C94EC2E8091100783FF02C0DA
:104BA0000C94EC2E83E50E94974C882399F00E9488
:104BB000174C0E94CDEBCB010E94F3590E94174C79
:104BC00020E030E044EB52E40E943DE6181614F079
:104BD0000E94FA780E9497C70C94EC2E8EE40E94F3
:104BE000974C882311F40C94EC2E0E94E74B6093B1
:104BF000BE187093BF188093C0189093C1180C947E
:104C0000EC2E83E50E944E4C882359F083E50E94E8
:104C1000974C882319F00E94F74B01C080E08093E5
:104C20001007E4EEFDE184918F010F5F1F4F8111AA
:104C300003C0E4EEF3E004C00E94CC89F801F3CF96
:104C400084918F010F5F1F4F882321F00E94CC8930
:104C5000F801F6CF809110078111CECDE0EEF3E0A0
:104C600018C0BB24B394B20E222319F08CE20E9428
:104C7000CC89F60185919491FC0184918F010F5F9D
:104C80001F4F882321F00E94CC89F801F6CF2B2DED
:104C9000C5CD84918F010F5F1F4F882309F4C8CDC4
:104CA0000E94CC89F801F5CF109220020C94EC2ED2
:104CB0008BEE93E00E94BBA00E94CC8E0C94EC2E55
:104CC00083E50E94974C811103C0E4EEFDE10DC025
:104CD0000E94F74B8D3320F480932B020C94EC2E22
:104CE0008CE380932B020C94EC2E84918F010F5F48
:104CF0001F4F882321F00E94CC89F801F6CF409104
:104D00002B0250E060E070E084EF93E00E941AC54F
:104D10008AE00E94CC890C94EC2E89E690E00E94F7
:104D2000D6AD811111C0EBEFF3E084918F010F5FDD
:104D30001F4F882321F00E94CC89F801F6CF0E94F2
:104D4000FC758AE00E94CC8910923F100C94872F4A
:104D500083E50E94974C882311F40C94EC2E0E945A
:104D6000F74B182F8D3308F01CE310934C100E9462
:104D7000FE586B017C01212F30E0A8EEB3E00E94C9
:104D800079EAC60ED71EE81EF91EC0924810D092CE
:104D90004910E0924A10F0924B100C94EC2E0E94B5
:104DA00018AE0C94EC2E8091100783FF02C00C9477
:104DB000EC2E83E50E94974C882311F40C94EC2E82
:104DC0000E94174C0E94CDEBCB010E94264E0C9402
:104DD000EC2E0E94DCA80C94EC2E80E50E94974CEF
:104DE000811106C083E50E94974C882359F005C0C5
:104DF0000E94F74B8111F0C7F5CF0E94E74B6F3F40
:104E0000710510F06FEF70E07093430460934204FB
:104E1000E3C780E50E94974C811105C010924304BE
:104E200010924204D9C70E94E74B672B09F0D4C700
:104E3000F5CF0E940F790E94AAB7109243041092F6
:104E4000420400E010E062E370E080E090E00E9445
:104E500010B70E94CF7B0F5F1F4F0331110599F7E9
:104E600062E370E080E090E00E9410B70E94CF7B88
:104E70000E94A12FB1C710922604AEC783E50E94FD
:104E8000974C882399F00E94174C20E030E04AE7C5
:104E900054E40E94A2E60E94D2EB60932C0270932D
:104EA0002D0280932E0290932F0296C788E50E94D0
:104EB0004E4C8111ACC789E50E944E4C8111A7C7A9
:104EC0008AE50E944E4C8111A2C785E40E944E4C97
:104ED00081119DC7CEC783E50E944E4C882309F4FB
:104EE0007BC70E94174C20E030E04AE754E40E9460
:104EF000A2E60E94D2EB6093441070934510809319
:104F000046109093471068C7B7E5CB2EB2E0DB2E72
:104F100012E9E12E10E1F12E10E0D6018D916D0124
:104F20000E944E4C882309F46DC0133009F063C011
:104F30000E94174C4B015C0120E030E040EA51E454
:104F40000E943DE687FF4EC0A501940160919E102E
:104F500070919F108091A0109091A1100E9465EB1C
:104F60002B013C019B01AC016091DF067091E006D2
:104F70008091E1069091E2060E94A2E66093DF062E
:104F80007093E0068093E1069093E206A3019201FC
:104F90006091FF06709100078091010790910207D0
:104FA0000E94A2E66093FF067093000780930107BA
:104FB0009093020760914B1170914C1180914D11AB
:104FC00090914E110E9441E6A30192010E94A2E637
:104FD0000E94D2EB60934B1170934C1180934D1152
:104FE00090934E1180929E1090929F10A092A010CC
:104FF000B092A11007C00E94174CF7016083718323
:10500000828393831F5FF4E0EF0EF11C143009F0EC
:1050100084CF0E9438C9E0C60E941E6A83E50E94C0
:10502000974C882309F451C80E94E74B6230710500
:1050300009F04BC80E94A9C98BE50E94CC896091F8
:10504000A4187091A5188091A6189091A71842E015
:105050000E94748D4091A8185091A9186091AA18C7
:105060007091AB1881E094E00E9437C54091AC1874
:105070005091AD186091AE187091AF188EEF93E01B
:105080000E9437C58DE50E94CC898AE00E94CC89B8
:10509000A3C684918F010F5F1F4F882321F00E94C8
:1050A000CC89F801F6CF60E083ED94E00E9415957D
:1050B00061E08CEC94E00E94159561E081EC94E055
:1050C0000E94159561E081EB94E00E94159560E0E7
:1050D00088EA94E00E94159561E08EE994E00E94D0
:1050E000159560E084E994E00E94159560E08CE8F5
:1050F00094E00E94159561E08EE794E00E9415957A
:1051000060E080E794E00E94159560E081E694E01D
:105110000E94159560E083E594E00E94159560E09B
:105120008DE394E00E94159560E08CE294E00E948B
:10513000159560E087E194E00E94159561E084E0B8
:1051400094E00E94159548C600911118109112180C
:1051500083E0D12C40E08150E9F0D8019C91292FC7
:105160002B7F2134C1F711962C912133A1F7913473
:1051700021F0953421F441E002C0DD24D39498015C
:105180002E5F3F4F89012F5F3F4FF8019081903292
:10519000C9F3E1CF442369F0E4EEFDE184917F019E
:1051A0002FEFE21AF20A882321F00E94CC89F7013E
:1051B000F5CFDD2069F0E9EAF5E084917F013FEF6A
:1051C000E31AF30A882321F00E94CC89F701F5CF76
:1051D000D8018D918D01882309F42ACB0E94CC89B6
:1051E000F7CF0E944DBEF8C581E0809337058093CC
:1051F0003605F2C588EC90E00E94D6AD8111ECC571
:1052000084E40E944E4C882309F441C00E94174C4C
:105210006B017C0111E020E030E0A9010E943DE635
:10522000811101C010E010932A1120E030E0A901A3
:10523000C701B6010E943DE6882349F10E94174C40
:10524000E0914E07B4E0EB9FF0011124E15DFE4ECA
:10525000608371838283938320E030E0A9016091B1
:105260002F117091301180913111909132110E9463
:105270003DE681110CC080E090E0A0EEBFE380939A
:105280002F1190933011A0933111B09332110E94DD
:10529000E8B7A2C5F70181917F010E944E4C882397
:1052A00051F00E94174C0E94D2EBD8016D937D9370
:1052B0008D939C9313970C5F1F4FC016D10651F727
:1052C0000E94C7C789C5E7E5EE2EE2E0FE2E03EF98
:1052D00016E0F70181917F010E944E4C882341F036
:1052E0000E94174CD8016D937D938D939C931397D7
:1052F0000C5F1F4FB7E003301B0759F76DC583E5FF
:105300000E94974C8823A1F00E94174C6093EB06F3
:105310007093EC068093ED069093EE066093E7069B
:105320007093E8068093E9069093EA0610E001C0C6
:1053300011E080E50E94974C882359F00E94174C99
:105340006093EB067093EC068093ED069093EE0667
:1053500010E082E50E94974C882359F00E94174C78
:105360006093EF067093F0068093F1069093F20637
:1053700010E084E50E94974C882359F00E94174C56
:105380006093E7067093E8068093E9069093EA0637
:1053900023C5112309F420C54091EB065091EC067A
:1053A0006091ED067091EE0683EB95E00E9437C5A3
:1053B0004091EF065091F0066091F1067091F2066F
:1053C00080EB95E00E9437C54091E7065091E806D2
:1053D0006091E9067091EA068DEA95E00E9437C572
:1053E0008AE00E94CC89F8C481E50E944E4C882353
:1053F000C1F08091210490912204009739F04AE095
:1054000050E060E070E00E94BCE403C060E070E047
:10541000CB01609303077093040780930507909373
:10542000060783E50E944E4C882351F00E94174CDA
:1054300060930B0770930C0780930D0790930E07F2
:1054400084E50E944E4C882351F00E94174C6093D3
:105450000707709308078093090790930A0788E568
:105460000E944E4C882351F00E94174C6093D30643
:105470007093D4068093D5069093D60689E50E9452
:105480004E4C882351F00E94174C6093D7067093BE
:10549000D8068093D9069093DA068AE50E944E4C8E
:1054A0008823F1F00E94174C6093DB067093DC06B2
:1054B0008093DD069093DE062DEC3CEC4CEC5DE336
:1054C0000E943DE6181664F0E3ECF5E084918F014C
:1054D0000F5F1F4F882321F00E94CC89F801F6CF7F
:1054E00085E40E944E4C882309F476C40E94174C30
:1054F0006093DF067093E0068093E1069093E206E6
:105500006BC467E5C62E62E0D62E78E3E72E75E021
:10551000F72E10E0F60181916F010E944E4C882316
:1055200059F00E94174CD7016D937D938D939C93F6
:105530001397812F0E9496AD1F5FB4E0EB0EF11C14
:10554000133041F70C9465200E9469B4811144C462
:1055500009EF12E2E2E3F4E0FDABECAB9E012F5F5A
:105560003F4F590152E4852E53E2952E1901F8015F
:105570006591759185919491ACA9BDA9CD90DD906F
:10558000ED90FD90BDABACABA70196010E9488EAFF
:105590002B013C01F101608371838283938320E0BE
:1055A00030E040EA51EC0E94AFEC87FD0AC020E0F9
:1055B00030E040EA51E4C301B2010E943DE6181612
:1055C0002CF4F401849118160CF456C4D101CD903A
:1055D000DD90ED90FD901D0120E030E040EA51ECBF
:1055E000C701B6010E94AFEC87FD0AC020E030E0A1
:1055F00040EA51E4C701B6010E943DE618164CF599
:10560000EFECFDE184918F010F5F1F4F811103C00B
:10561000E5EFF5E004C00E94CC89F801F3CF849156
:105620008F010F5F1F4F882321F00E94CC89F80162
:10563000F6CF88E290E099A388A388EC90E09DA73C
:105640008CA7BE01605E7F4FCE018C960E9466B52E
:10565000C3C30C5F1F4FBFEF8B1A9B0AE5E0F3E259
:10566000E017F10709F083CF48E3E42E45E0F42E7C
:1056700010E0F50181919191A191B1915F01F70144
:1056800081939193A193B1937F01812F0E9496AD55
:105690001F5F133071F70E944B9583E992E09DA73D
:1056A0008CA704E610E019A308A3BE01645D7F4F38
:1056B000CE0180960E9466B58AEB92E09DA78CA7EA
:1056C00019A308A3BE01645D7F4FCE0180960E949E
:1056D00066B582C383E50E94974C882309F47CC396
:1056E0000E94E74B709303026093020275C38DED35
:1056F00090E00E94D6AD81116FC383E50E94974C64
:10570000811103C0E4EEFDE13AC000914E0710E0C4
:105710000E94E74B000F111FF801E85CFD4F7183F9
:10572000608380914E0790E07C01EE0CFF1CEE0C34
:10573000FF1C87010F5D1D4F880F991FFC01E85C5E
:10574000FD4F60817181072E000C880B990B0E9420
:1057500043E62AE037ED43E25CE30E94A2E6F7016C
:10576000E55DFE4E20813181428153810E94A2E697
:10577000D8016D937D938D939C9313972DC3849142
:105780008F010F5F1F4F882321F00E94CC89F80101
:10579000F6CF85E40E94CC8980914E07805D0E94FF
:1057A000CC89E0914E07F0E0EE0FFF1FE85CFD4F63
:1057B0006081718183E196E00E9454C585E20E9478
:1057C000CC898AE00E94CC8907C380E50E944E4CB8
:1057D000882309F401C30E94E74B6B017C0183E538
:1057E0000E94974C882321F00E94E74B8B0102C056
:1057F0000FEF1FEFC8010196039708F0EDC2D7FC29
:10580000EBC28C2DEBE1F6E09491891709F43FC3CC
:105810003196B6E0EB34FB07B9F73CC383E50E9451
:10582000974C882319F00E94E74B02C064E071E0B6
:1058300079A368A380E50E94974C882339F00E94E1
:10584000E74B6938E3E17E0730F402C068EE73E0AD
:105850007A83698304C088E893E19A838983BE01CF
:10586000605E7F4FCE0101960E9466B5B5C285E4A9
:105870000E94974C811110C080E50E944E4C8823F5
:1058800091F00E94174C60933C0770933D07809302
:105890003E0790933F0707C00E94F74B882361F3B0
:1058A000EFECFDE171C089E40E944E4C882381F049
:1058B0000E94174C2CEA35EC47E25EE30E94A2E618
:1058C000609338077093390780933A0790933B07AA
:1058D00084E40E944E4C882381F00E94174C2CEAED
:1058E00035EC47E25EE30E9465EB609340077093FE
:1058F00041078093420790934307E4EEFDE18491D2
:105900008F010F5F1F4F882321F00E94CC89F8017F
:10591000F6CF40913C0750913D0760913E07709152
:105920003F0783E596E00E9437C52CEA35EC47E255
:105930005EE3609138077091390780913A07909142
:105940003B070E9465EBAB01BC018FE496E00E942F
:1059500037C52CEA35EC47E25EE360914007709171
:10596000410780914207909143070E94A2E6AB0154
:10597000BC018BE496E00E9437C58AE00E94CC8986
:105980002BC20E94CC89F80184918F010F5F1F4FB9
:105990008111F7CFE7E5F6E084918F010F5F1F4F8C
:1059A000882309F419C20E94CC89F801F5CF83E558
:1059B0000E944E4C182F882371F00E94174C0E94B1
:1059C000CDEB709326026093250221E0672B09F04E
:1059D00020E020930F0780E50E944E4C882359F069
:1059E0002091250230912602232B11F00E94084CB1
:1059F00080930F07F1C11111EFC1E4EEFDE1849135
:105A00008F010F5F1F4F882321F00E94CC89F8017E
:105A1000F6CF80910F07882319F06BE173E002C085
:105A20006EE173E08EE796E00E946DC560912502FD
:105A3000709126028DE696E00E9454C5E9E6F6E0F4
:105A400084918F010F5F1F4F882309F4C5C10E9405
:105A5000CC89F801F5CF0E94088FBEC180E50E9475
:105A60004E4C882351F00E94174C6093340770937A
:105A70003507809336079093370789E40E944E4C90
:105A8000882381F00E94174C2CEA35EC47E25EE354
:105A90000E94A2E66093300770933107809332072B
:105AA0009093330784E40E944E4C882381F00E9437
:105AB000174C2CEA35EC47E25EE30E9465EB6093FD
:105AC0002C0770932D0780932E0790932F07E4EEF9
:105AD000FDE184918F010F5F1F4F882321F00E9409
:105AE000CC89F801F6CF4091340750913507609189
:105AF00036077091370789E996E00E9437C52CEA8E
:105B000035EC47E25EE36091300770913107809198
:105B10003207909133070E9465EBAB01BC0185E928
:105B200096E00E9437C52CEA35EC47E25EE36091CF
:105B30002C0770912D0780912E0790912F070E94BE
:105B4000A2E6AB01BC0181E996E00E9437C58AE07C
:105B50000E94CC8941C10E94CC89F80184918F01B7
:105B60000F5F1F4F8111F7CFEDE9F6E084918F01B0
:105B70000F5F1F4F882309F42FC10E94CC89F801C1
:105B8000F5CF0E94E58D28C10E94597025C10E9461
:105B9000F1C222C183E50E944E4C882321F00E946D
:105BA000084C91E089270E9482BE16C181E0809353
:105BB00017070E944F6A10921707882309F40CC137
:105BC000E4EEFDE184918F010F5F1F4F811103C04F
:105BD000ECEAF6E004C00E94CC89F801F3CF84918E
:105BE0008F010F5F1F4F882309F4F6C00E94CC89F4
:105BF000F801F5CF8091310A882309F4EDC081E0E6
:105C00008093340AE9C08AE50E94974C811103C051
:105C1000EAEBF6E00BC00E94174C609337117093CB
:105C200038118093391190933A11D6C084918F0125
:105C30000F5F1F4F882321F00E94CC89F801F6CF17
:105C400040913711509138116091391170913A118A
:105C500087EB96E00E9437C58AE00E94CC89BCC0E1
:105C60008BE40E94974C811103C0E4EEFDE136C045
:105C70008BE40E94974C8823C1F00E94174C6B0163
:105C80007C0120E030E0A9010E94AFEC87FD0AC052
:105C900020E030E040E251E4C701B6010E943DE659
:105CA000181634F4E9EDF6E00EC0C12CD12C7601C3
:105CB0000E941E6AC092E306D092E406E092E506D6
:105CC000F092E60689C084918F010F5F1F4F8823F1
:105CD00009F482C00E94CC89F801F5CF84918F012C
:105CE0000F5F1F4F882321F00E94CC89F801F6CF67
:105CF0004091E3065091E4066091E5067091E60656
:105D000088EF96E00E9437C58AE00E94CC8964C083
:105D100081E08093270283E50E94974C882339F025
:105D20000E94084C811158C00E944DCE55C083E599
:105D30000E944E4CF7CF0E949AB54EC0F0901318B7
:105D40000E941E6A10917C1080E00E942CACFF2003
:105D500029F1E4EEFDE184918F010F5F1F4F88234D
:105D600021F00E94CC89F801F6CF84E50E94CC890D
:105D70006F2D70E080E090E04AE00E94EF8C80E2BE
:105D80000E94CC89E5E1F7E084918F010F5F1F4FFE
:105D9000882311F10E94CC89F801F6CF10923E10B1
:105DA000812F0E942CACE4EEFDE184918F010F5F06
:105DB0001F4F882321F00E94CC89F801F6CF609113
:105DC0003E1070E083E097E00E9454C58AE00E9494
:105DD000CC8902C00E949AB510923F100E9430CE2A
:105DE00096C00E94ACAA0E945CCAF6CF0E94E74B04
:105DF000AB01BC014093AB0C5093AC0C6093AD0C69
:105E00007093AE0C8AEF9BE00E94F597E5CF0E945D
:105E10001E6A88E50E944E4C882331F05F9A80917B
:105E200031048E7F8093310489E50E944E4C882393
:105E300039F08A9A479A809131048D7F809331049A
:105E40008AE50E944E4C882361F08091080180957C
:105E5000817080930601479A809131048B7F8093F3
:105E6000310485E40E944E4C882309F4B5CF129A80
:105E7000B3CF0E94AAB7B0CFF7FAF094F7F8F09436
:105E8000D101CD92DD92ED92FC9213979FCB0E94AF
:105E900071E1A2CF0E941E6ABC2C60E08C2D0E9492
:105EA0000DB60F3FBFEF1B0759F48C2D0E94B7B5FD
:105EB00031E020E0892B09F030E0032F122F05C0DC
:105EC0000130110561F401E010E08B2D0E94B7B59F
:105ED0008017910709F480CF0E9402A1F6CF00E05D
:105EE00010E0F3CF61E0812F0E940DB66E2D812F5F
:105EF0000E94DFB5F12CB701812F0E9449B61930FD
:105F000009F06ACFF0924304E092420465CFC6578D
:105F1000DF4F0FB6F894DEBF0FBECDBFDF91CF913C
:105F20001F910F91FF90EF90DF90CF90BF90AF90B7
:105F30009F908F907F906F905F904F903F902F90A9
:105F400008952F923F924F925F926F927F928F921D
:105F50009F92AF92BF92CF92DF92EF92FF920F93F8
:105F60001F93CF93DF93CDB7DEB76F970FB6F8943B
:105F7000DEBF0FBECDBFC0904C04D0904D04E0906A
:105F80004E04F0904F0420E030E040EA50E4C701B6
:105F9000B6010E943DE687FD19C120E030E041E9ED
:105FA00053E4C701B6010E94AFEC18160CF40EC101
:105FB00010924E0E10924D0E8091090140914C0EA0
:105FC000042E000C550B817021E0822790E04817C9
:105FD000590709F433C08091090181702827209363
:105FE0004C0E81111BC00E94BB80EFE2FDE084914A
:105FF0008F01882351F0082E000C990B0E94B68067
:106000000F5F1F4FF8018491F4CF8DE090E00E9464
:10601000B6808AE090E00E94B68010C0E3E3FDE025
:1060200084918F01882389F3082E000C990B0E941C
:10603000B6800F5F1F4FF8018491F4CF80913F0E1F
:10604000833009F44CC02CF4882351F08130D9F00E
:1060500072C0843009F43EC0853009F44DC06BC075
:106060008091310A882309F466C081E080933F0E55
:106070000E94FE586093430E7093440E8093450E29
:106080009093460E58C08091310A811154C080917E
:10609000FD0B882321F082E080933F0E4CC01092CC
:1060A0003F0EEBE2FDE084918F01882351F0082E32
:1060B000000C990B0E94B6800F5F1F4FF80184916E
:1060C000F4CF8DE090E00E94B6808AE090E00E94DC
:1060D000B68031C080918C0E8823E9F22CC080916B
:1060E000310A811128C08091B3099091B409891BAC
:1060F0008F7009F496C01FC08091310A81111BC0B6
:106100008091B3099091B409891B8F7009F4ABC0D9
:1061100012C08DE090E00E94B6808AE090E00E947C
:10612000B68010923F0E8BE09DE09093A407809381
:10613000A3070E94F8898091340E9091350E039741
:106140004CF57FE3272E79E0372EE0E68E2EEAEE3F
:106150009E2EA12CB12C8AE99FE00E94694B181653
:106160001906C4F48091340E9091350E049794F47E
:106170008AE99FE00E942D4B80933A0EE0913B0EFE
:10618000F0913C0E8A3019F08D3009F07DC03097C7
:1061900009F083C08091340E9091350E009711F470
:1061A0000C94223F01979093350E8093340E80918A
:1061B000360E9091370E019664E070E00E9472ED09
:1061C0009093370E8093360E0C94223F80914D0EA3
:1061D00090914E0E8136FAEE9F07E8F010924E0E27
:1061E00010924D0EE7E3FDE084918F01882351F07A
:1061F000082E000C990B0E94B6800F5F1F4FF8010C
:106200008491F4CF8DE090E00E94B6808AE090E027
:106210000E94B680D1CE019690934E0E80934D0E83
:10622000CBCE87E19DE09093A4078093A3070E94C3
:10623000F88980918C0E882311F082E001C084E0FF
:1062400080933F0EE3E1FDE084918F01882309F400
:1062500038CF082E000C990B0E94B6800F5F1F4F9D
:10626000F8018491F3CFEFE0FDE084918F01882362
:1062700009F44FCF082E000C990B0E94B6800F5FD7
:106280001F4FF8018491F3CF8A3309F480CFEF35A3
:10629000F10514F40C94B63C7ACF8091380E9091AD
:1062A000390E20E6289F7001299FF00C11248701E8
:1062B0000C54134FE00FF11F108261E470E0C8012D
:1062C0000E94D9ED009711F40C949A3C90933E0EE5
:1062D00080933D0E801B910B8E0D9F1D60E070E042
:1062E0008B54934F0E943EE20E94CDEBCB01770F7F
:1062F000AA0BBB0B8232910510F00C949A3CFC0166
:106300008827EE58FF4F8F4F0C9485EDE6E0FDE0B7
:1063100084918F01882351F0082E000C990B0E9464
:10632000B6800F5F1F4FF8018491F4CF20E030E07A
:1063300040E05FE360914C0470914D0480914E0405
:1063400090914F041EC0E1E0FDE084918F0188230D
:1063500051F0082E000C990B0E94B6800F5F1F4F62
:10636000F8018491F4CF60914A0470914B04072E98
:10637000000C880B990B0E9443E620E030E040E0DF
:106380005FE30E9489EA0E94CDEBCB010E94F04DB1
:106390000E94C1D78DE090E00E94B6808AE090E034
:1063A0000E94B6800C949A3CECEFFCE084918F0143
:1063B000882351F0082E000C990B0E94B6800F5FC5
:1063C0001F4FF8018491F4CF20E030E040E05FE31C
:1063D000609146047091470480914804909149046B
:1063E000D0CFE7EFFCE084918F01882351F0082E95
:1063F000000C990B0E94B6800F5F1F4FF80184912B
:10640000F4CF6091440470914504B1CF20914204CF
:106410003091430444E6429FC001439F900D1124F4
:106420006FEF70E00E9472ED8B016536710510F020
:1064300004E610E0E2EFFCE084917F01882359F04C
:10644000082E000C990B0E94B680FFEFEF1AFF0A8E
:10645000F7018491F3CFB80180E090E036C7EEEE0B
:10646000FCE084918F01882351F0082E000C990BD9
:106470000E94B6800F5F1F4FF8018491F4CF80E235
:1064800090E00E94B680EAEEFCE084918F018823C0
:1064900051F0082E000C990B0E94B6800F5F1F4F21
:1064A000F8018491F4CF60913204709133048091AB
:1064B0003404909135040E94C2D780E290E00E949B
:1064C000B680E6EEFCE084918F01882351F0082E1F
:1064D000000C990B0E94B6800F5F1F4FF80184914A
:1064E000F4CF609136047091370480913804909114
:1064F00039040E94C2D780E290E00E94B680E2EEAA
:10650000FCE084918F01882351F0082E000C990B38
:106510000E94B6800F5F1F4FF8018491F4CF609105
:106520003A0470913B0480913C0490913D040E9498
:10653000C2D780E290E0A0C58091310A882309F497
:1065400050C0EDEDFCE084918F01882351F0082EBE
:10655000000C990B0E94B6800F5F1F4FF8018491C9
:10656000F4CF8091320A882359F18091FD0B882362
:1065700029F18091A70C9091A80CA091A90CB09141
:10658000AA0C0097A105B105C1F0BC01CD016D5960
:106590007F4F8F4F9F4F24E630E040E050E00E9455
:1065A0002BEA6091AB0C7091AC0C8091AD0C90918A
:1065B000AE0C0E942BEA822F01C080E090E0E6CE74
:1065C000E9EDFCE084918F01882309F4E3CE082EE5
:1065D000000C990B0E94B6800F5F1F4FF801849149
:1065E000F3CFE1EDFCE084918F01882309F4D2CE52
:1065F000082E000C990B0E94B6800F5F1F4FF80108
:106600008491F3CFECECFCE084918F01882351F06E
:10661000082E000C990B0E94B6800F5F1F4FF801E7
:106620008491F4CF8091430E9091440EA091450E39
:10663000B091460E892B8A2B8B2B09F477C00E94D0
:10664000FE58A50194010E942BEA69017A0160912C
:10665000430E7091440E8091450E9091460EA50117
:1066600094010E942BEA8601021B130BC8016CE304
:1066700070E00E945EEDCB019927EAE0F0E0BF01F7
:106680000E9472ED282FCB01BF010E9472ED805D48
:1066900080932904205D20932A0410922B0489E220
:1066A00094E00E94C1D780E290E00E94B680EAECBC
:1066B000FCE084917F01882359F0082E000C990B8F
:1066C0000E94B680FFEFEF1AFF0AF7018491F3CF23
:1066D00080E290E00E94B680C8016CE370E00E9406
:1066E0005EED6AE070E00E9472ED605D60932904E7
:1066F000805D80932A0410922B0489E294E00E942A
:10670000C1D780E290E00E94B680E8ECFCE0849182
:106710008F01882309F43ECE082E000C990B0E94AD
:10672000B6800F5F1F4FF8018491F3CF80E290E0B5
:106730000E94B680E0ECFCE084918F01882309F48C
:1067400029CE082E000C990B0E94B6800F5F1F4FB8
:10675000F8018491F3CF10926D0E8091090180FFB2
:1067600011C0ECEBFCE084918F01882309F412CE78
:10677000082E000C990B0E94B6800F5F1F4FF80186
:106780008491F3CF83E50E945DD7882341F00E9476
:1067900078D70E94D2EB7093420E6093410EE8EBE3
:1067A000FCE084918F01882351F0082E000C990B96
:1067B0000E94B6800F5F1F4FF8018491F4CF8DE0E7
:1067C00090E00E94B6808AE090E00E94B6808091BE
:1067D0008B0E882309F442C28091410E9091420EA3
:1067E0008430910509F4C8C08830910509F47DC151
:1067F000892B09F0E7C3ECEDFAE084918F0188233F
:1068000051F0082E000C990B0E94B6800F5F1F4FAD
:10681000F8018491F4CF8DE090E00E94B6808AE088
:1068200090E00E94B680E1EDFAE084918F01882328
:1068300051F0082E000C990B0E94B6800F5F1F4F7D
:10684000F8018491F4CF8DE090E00E94B6808AE058
:1068500090E00E94B680E5ECFAE084918F018823F5
:1068600051F0082E000C990B0E94B6800F5F1F4F4D
:10687000F8018491F4CF8DE090E00E94B6808AE028
:1068800090E00E94B680E9EBFAE084918F018823C2
:1068900051F0082E000C990B0E94B6800F5F1F4F1D
:1068A000F8018491F4CF8DE090E00E94B6808AE0F8
:1068B00090E00E94B680EBEAFAE084918F01882391
:1068C00051F0082E000C990B0E94B6800F5F1F4FED
:1068D000F8018491F4CF8DE090E00E94B6808AE0C8
:1068E00090E00E94B680EDE9FAE084918F01882360
:1068F00051F0082E000C990B0E94B6800F5F1F4FBD
:10690000F8018491F4CF8DE090E00E94B6808AE097
:1069100090E00E94B680E0E9FAE084918F0188233C
:1069200051F0082E000C990B0E94B6800F5F1F4F8C
:10693000F8018491F4CF8DE090E00E94B6808AE067
:1069400090E00E94B680E3E8FAE084918F0188230A
:1069500051F0082E000C990B0E94B6800F5F1F4F5C
:10696000F8018491F4CF8DE090E00E94B6808AE037
:1069700090E00E94B68026C3E5E7FAE084918F019B
:10698000882351F0082E000C990B0E94B6800F5FEF
:106990001F4FF8018491F4CF8DE090E00E94B68003
:1069A0008AE090E00E94B680E7E6FAE084918F01E9
:1069B000882351F0082E000C990B0E94B6800F5FBF
:1069C0001F4FF8018491F4CF8DE090E00E94B680D3
:1069D0008AE090E00E94B680E1E5FAE084918F01C0
:1069E000882351F0082E000C990B0E94B6800F5F8F
:1069F0001F4FF8018491F4CF8DE090E00E94B680A3
:106A00008AE090E00E94B680EBE3FAE084918F0187
:106A1000882351F0082E000C990B0E94B6800F5F5E
:106A20001F4FF8018491F4CF8DE090E00E94B68072
:106A30008AE090E00E94B680E9E2FAE084918F015A
:106A4000882351F0082E000C990B0E94B6800F5F2E
:106A50001F4FF8018491F4CF8DE090E00E94B68042
:106A60008AE090E00E94B680E7E1FAE084918F012D
:106A7000882351F0082E000C990B0E94B6800F5FFE
:106A80001F4FF8018491F4CF8DE090E00E94B68012
:106A90008AE090E00E94B680E9E0FAE084918F01FC
:106AA000882351F0082E000C990B0E94B6800F5FCE
:106AB0001F4FF8018491F4CF8DE090E00E94B680E2
:106AC0008AE090E00E94B680EBEFF9E084918F01BC
:106AD000882309F448CF082E000C990B0E94B68039
:106AE0000F5F1F4FF8018491F3CFE4EFF9E0849139
:106AF0008F01882351F0082E000C990B0E94B6805C
:106B00000F5F1F4FF8018491F4CF8DE090E00E9459
:106B1000B6808AE090E00E94B680EDEEF9E08491C4
:106B20008F01882351F0082E000C990B0E94B6802B
:106B30000F5F1F4FF8018491F4CF8DE090E00E9429
:106B4000B6808AE090E00E94B680E6EDF9E084919C
:106B50008F01882351F0082E000C990B0E94B680FB
:106B60000F5F1F4FF8018491F4CF8DE090E00E94F9
:106B7000B6808AE090E00E94B680EFEBF9E0849165
:106B80008F01882351F0082E000C990B0E94B680CB
:106B90000F5F1F4FF8018491F4CF8DE090E00E94C9
:106BA000B6808AE090E00E94B680E8EAF9E084913D
:106BB0008F01882351F0082E000C990B0E94B6809B
:106BC0000F5F1F4FF8018491F4CF8DE090E00E9499
:106BD000B6808AE090E00E94B680E1E9F9E0849115
:106BE0008F01882351F0082E000C990B0E94B6806B
:106BF0000F5F1F4FF8018491F4CF8DE090E00E9469
:106C0000B6808AE090E00E94B680E3E8F9E08491E3
:106C10008F01882351F0082E000C990B0E94B6803A
:106C20000F5F1F4FF8018491F4CF8DE090E00E9438
:106C3000B6808AE090E00E94B680E5E7F9E08491B2
:106C40008F01882309F48FCE082E000C990B0E9427
:106C5000B6800F5F1F4FF8018491F3CF8091320A05
:106C6000882309F486C181E08093AF0C1092B10CA7
:106C70001092B00C81E89AE00E943C9A8BE1E1E826
:106C8000FAE0DE01159601900D928A95E1F7809168
:106C90007F0A9091800A9C838B838DEE92E09A8389
:106CA000898340E050E0BE016F5F7F4F80E090E05D
:106CB0000E94E982CE0101960E9498A0C090B00C7B
:106CC000D090B10C0091410E1091420EC601801B74
:106CD000910B049720F06801F3E0CF0ED11C56E62B
:106CE000452E59E0552E67E5662E69E0762EC016D2
:106CF000D10608F467C10115110509F0A1C065E3CB
:106D00007AE081E89AE00E94049962E273E085E308
:106D10009AE00E94E4ED892B09F04AC0F2018491C7
:106D200046E6E42E49E0F42E882359F0082E000CA4
:106D3000990B0E94B680FFEFEF1AFF0AF7018491CA
:106D4000F3CF8DE090E00E94B6808AE090E00E9450
:106D5000B680F301849137E5E32E39E0F32E8823E2
:106D600059F0082E000C990B0E94B680FFEFEF1A25
:106D7000FF0AF7018491F3CF8DE090E00E94B68086
:106D80008AE090E00E94B6804AE060E070E0CB01CB
:106D90000E94EF8CE7E4F9E084917F012FEFE21A83
:106DA000F20A882309F4E2C00E94CC89F701F4CFEB
:106DB000E3E4F9E084917F01882359F0082E000C68
:106DC000990B0E94B680FFEFEF1AFF0AF70184913A
:106DD000F3CF8DE090E00E94B6808AE090E00E94C0
:106DE000B680F10184912FE3E22E29E0F22E882370
:106DF00059F0082E000C990B0E94B680FFEFEF1A95
:106E0000FF0AF7018491F3CF8DE090E00E94B680F5
:106E10008AE090E00E94B6804AE060E070E0CB013A
:106E20000E94EF8CEAE3F9E084917F012FEFE21AF0
:106E3000F20A882309F49AC00E94CC89F701F4CFA2
:106E400060E070E0C80101970E94A7848091330A36
:106E5000882309F45FC0E8E3F9E084917F01882387
:106E600059F0082E000C990B0E94B680FFEFEF1A24
:106E7000FF0AF7018491F3CF85E39AE00E94C1D71E
:106E80008DE090E00E94B6808AE090E00E94B6809B
:106E9000E6E3F9E084917F01882359F0082E000C85
:106EA000990B0E94B680FFEFEF1AFF0AF701849159
:106EB000F3CF82E49AE00E94C1D78DE090E00E9477
:106EC000B6808AE090E00E94B680C801A0E0B0E001
:106ED0004AE0BC01CD010E94EF8CE4E3F9E084912B
:106EE0007F012FEFE21AF20A882321F00E94CC8959
:106EF000F701F5CF92E4E92E9AE0F92EF70181919E
:106F00007F01882319F00E94CC89F8CF8AE00E9483
:106F1000CC892CC085E39AE00E94C1D78DE090E037
:106F20000E94B6808AE090E00E94B68082E49AE0F7
:106F30000E94C1D78DE090E00E94B6808AE090E088
:106F40000E94B680C801A0E0B0E04AE0BC01CD01DB
:106F50000E94EF8C82E4E82E8AE0F82EF7018191FE
:106F60007F01882399F20E94CC89F8CF0F5F1F4FD1
:106F7000BECEE5E2F9E084918F01882351F0082E1E
:106F8000000C990B0E94B6800F5F1F4FF80184918F
:106F9000F4CF8DE090E00E94B6808AE090E00E94FD
:106FA000B680E6E1F9E084918F01882309F4DBCC17
:106FB000082E000C990B0E94B6800F5F1F4FF8013E
:106FC0008491F3CFE4EBFCE084918F01882309F4F2
:106FD000E1C9082E000C990B0E94B6800F5F1F4F6D
:106FE000F8018491F3CF8091310A882339F00E940F
:106FF0001B82A0C48091310A8823E9F00E9411B15C
:1070000099C480913F0E823019F0833609F092C402
:107010000E94FB81E0EBFCE084918F01882309F45E
:10702000B9C9082E000C990B0E94B6800F5F1F4F44
:10703000F8018491F3CF80913F0E833609F07AC432
:10704000DDCF87EA9CE00E94BBA08091B3099091BC
:10705000B409891B8F7009F06DC480913F0E823096
:1070600009F468C4833609F099C464C48DE090E0E3
:107070000E94B6808AE090E00E94B6808BC9809121
:10708000B3099091B409891B8F7009F053C48091A2
:107090003F0E823009F44EC4833609F44BC480910C
:1070A000FD0B8111CFC446C483E50E945DD78111D9
:1070B00026C083E40E945DD7882309F43BC48091F5
:1070C000B3099091B409891B8F7009F033C420E093
:1070D00030E040E251E460913A0470913B048091C9
:1070E0003C0490913D040E943DE687FF08C084E97E
:1070F0009CE09093A4078093A3070E94F8890E94C4
:1071000078D720E030E0A9010E943DE687FD10C05D
:107110000E9478D720E030E849E853E40E94AFECC1
:1071200018164CF00E9478D70E94D2EBCB0105C014
:1071300080E090E002C083E191E00E94F359FAC33D
:1071400083E50E945DD7882309F4F4C30E9478D7B1
:1071500020E030E0A9010E943DE687FD10C00E94BA
:1071600078D720E030E046E153E40E94AFEC1816F7
:107170004CF00E9478D70E94D2EBCB0105C080E092
:1071800090E002C086E990E00E94264ED3C383E5DA
:107190000E945DD78823D9F00E9478D720E030E0A4
:1071A0004FE753E40E94A2E620E030E048EC52E4CE
:1071B0000E9465EB0E94D2EB6F3F710519F010F051
:1071C0006FEF70E07093430460934204E3C88FEF65
:1071D00090E09093430480934204DCC88091B3090B
:1071E0009091B409891B8F7009F0D4C88091310A3D
:1071F0008111D0C80E94CC8E5F9A809131048E7F1D
:10720000809331048A9A479A809131048D7F8093CC
:107210003104809108018095817080930601479A1E
:10722000809131048B7F80933104129AB3C883E537
:107230000E945DD7882319F10E9478D720E030E0C2
:1072400040E252E40E943DE687FD0FC00E9478D7DD
:1072500020E030EC49E754E40E94AFEC181644F00B
:107260000E9478D70E94CDEB05C068E270E002C0B2
:1072700067EE73E070930302609302025BC3EEE873
:10728000FCE084918F01882351F0082E000C990BAB
:107290000E94B6800F5F1F4FF8018491F4CFC09019
:1072A0000202D09003020D2C000CEE08FF08F7FE3E
:1072B0000EC06DE28AE99FE00E94E04A66277727C8
:1072C000CB016C197D098E099F094AE003C04AE091
:1072D000C701B6010E9481D75DC88091B309909122
:1072E000B409891B8F7009F025C380913F0E82304D
:1072F00009F420C3833609F0EBC21CC38091B309A3
:107300009091B409891B8F7009F044C880913F0E99
:10731000823009F43FC8833609F0B6C33BC8809178
:10732000B3099091B409891B8F7009F003C3809150
:107330003F0E823009F4FEC2833609F0FBC4FAC264
:107340008091B3099091B409891B8F7009F0F2C242
:1073500080913F0E823009F4EDC2833609F020C5DA
:10736000E9C28091B3099091B409891B8F7009F02B
:10737000E1C280913F0E823009F4DCC2833609F00D
:1073800045C5D8C280916D0E811103C00E94BB809B
:10739000C4C18E3271F580916E0E8E3209F046C1F5
:1073A0008091D20B882309F4B8C181508093D20B0D
:1073B000882361F090E001974FE1489F9001499F39
:1073C000300D1124C9018456954F02C08EE59AE014
:1073D0002BE1FC013496A1E8BAE001900D922A95C8
:1073E000E1F7FC01828193819093800A80937F0A68
:1073F00094C18C3309F01AC164E273E08DE69EE01B
:107400000E94E4ED892B21F481E080938B0E85C1ED
:1074100063E373E08DE69EE00E94E4ED892B79F44E
:10742000E2EFF8E084918F010F5F1F4F882321F076
:107430000E94CC89F801F6CF85ED98E0E4C06AE4BB
:1074400073E08DE69EE00E94E4ED892B79F4E1EB98
:10745000F8E084918F010F5F1F4F882321F00E9475
:10746000CC89F801F6CF8EE998E0CDC061E673E0F3
:107470008DE69EE00E94E4ED892B79F4E3E8F8E0E4
:1074800084918F010F5F1F4F882321F00E94CC89C8
:10749000F801F6CF8EE798E0B6C06FE673E08DE6B0
:1074A0009EE00E94E4ED892B79F4E3E6F8E0849114
:1074B0008F010F5F1F4F882321F00E94CC89F801B4
:1074C000F6CF8EE598E09FC06DE773E08DE69EE015
:1074D0000E94E4ED892B79F4E3E4F8E084918F01D4
:1074E0000F5F1F4F882321F00E94CC89F801F6CF4F
:1074F0008AE398E088C06BE873E08DE69EE00E9426
:10750000E4ED892B71F407E118E0F80184918823F8
:1075100029F00F5F1F4F0E94CC89F7CF80E198E0E0
:1075200072C061EA73E08DE69EE00E94E4ED892B73
:1075300079F4E1EFF7E084918F010F5F1F4F88230B
:1075400021F00E94CC89F801F6CF8AEE97E05BC06B
:1075500063EB73E08DE69EE00E94E4ED892B79F405
:10756000E2EDF7E084918F010F5F1F4F882321F038
:107570000E94CC89F801F6CF81EC97E044C06EEB15
:1075800073E08DE69EE00E94E4ED892B79F4E8EA51
:10759000F7E084918F010F5F1F4F882321F00E9435
:1075A000CC89F801F6CF86E997E02DC06AEC73E04C
:1075B0008DE69EE00E94E4ED892B79F4EBE7F7E09D
:1075C00084918F010F5F1F4F882321F00E94CC8987
:1075D000F801F6CF89E697E016C068ED73E08DE616
:1075E0009EE00E94E4ED892BA9F4EFE4F7E084919A
:1075F0008F010F5F1F4F882321F00E94CC89F80173
:10760000F6CF8DE397E09093A4078093A3070E94A1
:10761000F88983C065EE73E08DE69EE00E94E4ED9C
:10762000892B09F07AC010928B0E77C01D821886C4
:107630001C821B828DEE92E09A8389838091840A5A
:10764000811103C06EE57AE002C06DE77AE0611552
:10765000710519F06C5F7F4F02C060E070E021E0BF
:107660004DE65EE0CE0105960E946B9E882361F197
:107670008BE1FE013596A1E8BAE001900D928A9562
:10768000E1F72B813C813093800A20937F0A80911F
:10769000D20B8A3008F03DC091E0980F9093D20B46
:1076A000FFE18F9FC0011124DC01A056B54F4BE1D3
:1076B000E1E8FAE001900D924A95E1F7FC01E45609
:1076C000F54F3383228325C0E4EEFDE184918F01E1
:1076D0000F5F1F4F882321F00E94CC89F801F6CF5D
:1076E000E7E2F7E084918F010F5F1F4F882321F0BD
:1076F0000E94CC89F801F6CF0DE61EE0F8018191D9
:107700008F01882319F00E94CC89F8CF8AE00E946B
:10771000CC89CE0101960E9498A010926D0E8091A6
:10772000090180FF07C1E2EDFBE084918F0188230E
:1077300011F40C94CA31082E000C990B0E94B680EB
:107740000F5F1F4FF8018491F2CF8FE40E945DD745
:1077500081110C94CA3183E40E945DD70C94CA3124
:1077600083E50E945DD7811159C08FE40E945DD7E7
:10777000882319F08AE99BE007C084E50E945DD761
:10778000882349F082E79BE09093A4078093A307A6
:107790000E94F88943C083E40E945DD7882319F0D2
:1077A00089E49BE0F1CF81E50E945DD7882319F041
:1077B00081E29BE0E9CF88E40E945DD78823C9F08D
:1077C000EDE1FBE084918F01882351F0082E000C3D
:1077D000990B0E94B6800F5F1F4FF8018491F4CF80
:1077E0008DE090E00E94B6808AE090E00E94B68032
:1077F00015C08CE40E945DD7882381F0E9E1FBE0AD
:1078000084918F01882361F3082E000C990B0E944C
:10781000B6800F5F1F4FF8018491F4CFE1EEFBE0DB
:1078200084918F01882311F40C94CA31082E000C26
:10783000990B0E94B6800F5F1F4FF8018491F2CF21
:107840008091B3098091B4090C94CA3183E50E94F8
:107850005DD7882309F46EC081EF9AE09093A40766
:107860008093A3070E94F889E1EEFBE084918F01E9
:10787000882311F40C94CA31082E000C990B0E9435
:10788000B6800F5F1F4FF8018491F2CFECEEFAE063
:1078900084918F01882351F0082E000C990B0E94CF
:1078A000B6800F5F1F4FF8018491F4CFE7EEFAE046
:1078B00084918F01882311F40C94CA31082E000C96
:1078C000990B0E94B6800F5F1F4FF8018491F2CF91
:1078D00088E50E945DD7811106C089E50E945DD7C9
:1078E000882309F4C3C088E50E945DD7882341F04E
:1078F00088E89CE09093A4078093A3070E94F889EE
:1079000089E50E945DD7882341F082E89CE090934E
:10791000A4078093A3070E94F8898AE50E945DD797
:10792000882341F08CE79CE09093A4078093A30701
:107930000E94F8898091380E9091390E019664E08A
:1079400070E00E9472ED9093390E8093380E809112
:10795000340E9091350E01969093350E8093340E2F
:1079600010923C0E10923B0E0C94AB304091380EAE
:107970005091390E9F012F5F3F4F30933C0E209363
:107980003B0E90E6949F9001959F300D11242C544E
:10799000334FE20FF31F80830C94AB3000913D0E08
:1079A00010913E0E780124E0E20EF11C6AE270E0D4
:1079B000C7010E94D9EDF80124812F3221F4B801CA
:1079C0006B5F7F4F03C02C3339F4B7018DE69EE027
:1079D0000E94EDED0C94CA3110926D0E009719F0D3
:1079E000FC013197108280913D0E90913E0E40E057
:1079F00061E004960E948BD58091FD0B882389F06D
:107A0000E3EAFCE084918F01882309F42FCB082E50
:107A1000000C990B0E94B6800F5F1F4FF8018491F4
:107A2000F3CFEFE9FCE084918F01882309F41ECBAA
:107A3000082E000C990B0E94B6800F5F1F4FF801B3
:107A40008491F3CF0E94FB81EBE9FCE084918F01EC
:107A5000882311F40C94CA31082E000C990B0E9453
:107A6000B6800F5F1F4FF8018491F2CF8AE50E9424
:107A70005DD7811138CF83E40E945DD7882309F454
:107A800059CF88E79CE050CF86E40E945DD78823D9
:107A900009F44DC10E9478D70E94D2EB8B0184E794
:107AA0009CE09093A4078093A3070E94F88988E53F
:107AB0000E945DD7882309F451C00E9478D72B011A
:107AC0003C012DEC3CEC4CE45EE30E943DE69E0163
:107AD0002F5F3F4F7901181674F020E030E0A901C4
:107AE000C301B2010E94AFEC18162CF41F930F9340
:107AF00089E69CE005C12DEC3CEC4CEC5DEBC30150
:107B0000B2010E943DE618167CF020E030E040E82B
:107B10005FEBC301B2010E94AFEC18162CF41F9367
:107B20000F938DE59CE0ECC01F930F93C301B2014E
:107B30000E94CDEB7F936F9383E59CE09F938F939F
:107B4000FF92EF920E940FE60FB6F894DEBF0FBED1
:107B5000CDBFCE0101960E94D389DFC089E50E9486
:107B60005DD7882309F441C00E9478D72B013C01DE
:107B70002DEC3CEC4CE45EE30E943DE6FE013196C8
:107B80007F01181674F020E030E0A901C301B201B2
:107B90000E94AFEC18162CF41F930F9388E49CE01E
:107BA000AFC02DEC3CEC4CEC5DEBC301B2010E948C
:107BB0003DE618167CF020E030E040E85FEBC301C2
:107BC000B2010E94AFEC18162CF41F930F938CE3B4
:107BD0009CE096C01F930F93C301B2010E94CDEBAE
:107BE0007F936F9382E39CE0A9CF8AE50E945DD7E3
:107BF000882309F441C00E9478D72B013C012DEC69
:107C00003CEC4CE45EE30E943DE6FE0131967F01D0
:107C1000181674F020E030E0A901C301B2010E94FF
:107C2000AFEC18162CF41F930F9387E29CE068C00A
:107C30002DEC3CEC4CEC5DEBC301B2010E943DE647
:107C400018167CF020E030E040E85FEBC301B201A1
:107C50000E94AFEC18162CF41F930F938BE19CE05D
:107C60004FC01F930F93C301B2010E94CDEB7F93CE
:107C70006F9381E19CE062CF85E40E945DD7882309
:107C800009F44BC00E9478D72B013C012DEC3CEC51
:107C90004CE45EE30E943DE6FE0131967F0118163A
:107CA00074F020E030E0A901C301B2010E94AFEC02
:107CB00018162CF41F930F9386E09CE021C02DEC46
:107CC0003CEC4CEC5DEBC301B2010E943DE61816A2
:107CD0007CF020E030E040E85FEBC301B2010E949D
:107CE000AFEC18162CF41F930F938AEF9BE008C09B
:107CF000C301B2010E94CDEB7F936F938FEE9BE0A7
:107D00009F938F93FF92EF920E940FE60F900F9038
:107D10000F900F900F900F901CCF8BEE9BE09093E5
:107D2000A4078093A3070E94F8890C94CA3100E04D
:107D300010E0B5CE20E030E040E251E460913A043A
:107D400070913B0480913C0490913D040E943DE67B
:107D500087FF08C084EE9BE09093A4078093A3075D
:107D60000E94F88982E390E0909345048093440454
:107D70000E94B67688EC90E00E94F359E1EEFBE0B9
:107D800084918F01882311F40C94CA31082E000CC1
:107D9000990B0E94B6800F5F1F4FF8018491F2CFBC
:107DA00020E030E040E251E460913A0470913B04FD
:107DB00080913C0490913D040E943DE687FF08C0FD
:107DC0008AED9BE09093A4078093A3070E94F88913
:107DD00080E590E090934504809344040E94B67639
:107DE00080EF90E00E94F359E1EEFBE084918F0177
:107DF000882311F40C94CA31082E000C990B0E94B0
:107E0000B6800F5F1F4FF8018491F2CF80E090E0C1
:107E10000E94F35910924504109244040E94B676D1
:107E2000E6EDFBE084918F01882311F40C94CA31B4
:107E3000082E000C990B0E94B6800F5F1F4FF801AF
:107E40008491F2CF6F960FB6F894DEBF0FBECDBF10
:107E5000DF91CF911F910F91FF90EF90DF90CF9026
:107E6000BF90AF909F908F907F906F905F904F905A
:107E70003F902F9008952F923F924F925F926F9272
:107E80007F928F929F92AF92BF92CF92DF92EF92AA
:107E9000FF920F931F93CF93DF93CDB7DEB7629717
:107EA0000FB6F894DEBF0FBECDBFF8948FEF9FEFF3
:107EB00090938900809388002AE02A8B212C312C12
:107EC00078948091A2049091A304A091A404B0910D
:107ED000A504892B8A2B8B2B09F016C280911A07D7
:107EE0008823E1F010921A078091180790911907E2
:107EF000892B09F409C210925A04109219071092A2
:107F000018079091B3098091B409981709F4FCC13E
:107F10008091B4098F5F8F708093B40980911807A6
:107F200090911907892B09F4EFC140919E0450915B
:107F30009F046091A0047091A10480919A04909193
:107F40009B04A0919C04B0919D040091910410E0C9
:107F500020E030E0841B950BA60BB70B0817190720
:107F60002A073B0710F4D901C801E82F840F951F99
:107F7000A61FB71F80939E0490939F04A093A00414
:107F8000B093A1042091840030918500225E3F4F80
:107F9000409176045091770460917804709179044F
:107FA0008091660490916704A0916804B09169047F
:107FB000840F951FA61FB71F8093760490937704B4
:107FC000A0937804B0937904B7FD1CC0889A80917F
:107FD000821090918310A0918410B09185104091EF
:107FE0000402042E000C550B660B770B840F951FB3
:107FF000A61FB71F8093821090938310A0938410C4
:10800000B093851040917A0450917B0460917C0478
:1080100070917D0480916A0490916B04A0916C042E
:10802000B0916D04840F951FA61FB71F80937A042B
:1080300090937B04A0937C04B0937D04B7FD1CC097
:108040008E9A8091861090918710A0918810B0919F
:10805000891040910502042E000C550B660B770B1E
:10806000840F951FA61FB71F8093861090938710CB
:10807000A0938810B093891040917E0450917F04A2
:10808000609180047091810480916E0490916F04DE
:10809000A0917004B0917104840F951FA61FB71FA3
:1080A00080937E0490937F04A0938004B093810416
:1080B000B7FD3FC080915404F09106028823C9F0B7
:1080C0008091520482FF02C0F7FD06C080915104E6
:1080D000882311F40C94F348809152049091530436
:1080E00093FF02C0F7FD0CC080915004811108C0BD
:1080F00006C080910B018095887080930901419A98
:1081000040918A1050918B1060918C1070918D105D
:108110008F2FFF0F990BAA0BBB0B840F951FA61F68
:10812000B71F80938A1090938B10A0938C10B093FC
:108130008D10409182045091830460918404709169
:1081400085048091720490917304A0917404B0919D
:108150007504840F951FA61FB71F80938204909308
:108160008304A0938404B0938504B7FD3AC0409182
:108170008E1050918F106091901070919110C0905E
:1081800007020C2C000CDD08EE08FF084C0D5D1DED
:108190006E1D7F1D40938E1050938F106093901032
:1081A0007093911040916204509163046091640453
:1081B00070916504841B950BA60BB70B809382040A
:1081C00090938304A0938404B09385049091550404
:1081D00080918F0493FF02C0815001C08F5F809314
:1081E0008F04809184009091850082179307C8F3D3
:1081F0008091760490917704A0917804B0917904ED
:10820000B7FD15C04091620450916304609164040D
:1082100070916504841B950BA60BB70B80937604B5
:1082200090937704A0937804B09379048898809110
:108230007A0490917B04A0917C04B0917D04B7FDF9
:1082400015C0409162045091630460916404709180
:108250006504841B950BA60BB70B80937A0490934F
:108260007B04A0937C04B0937D048E9880917E045F
:1082700090917F04A0918004B0918104B7FD3AC031
:1082800040916204509163046091640470916504AC
:10829000841B950BA60BB70B80937E0490937F04F1
:1082A000A0938004B0938104809154048823E1F06A
:1082B0008091520482FF04C08091060287FD05C0B0
:1082C00080915104882309F496C7809152049091BB
:1082D000530493FF04C08091060287FD0BC0809178
:1082E0005004811107C005C080910B0188708093F4
:1082F00009014198E15041F08091840090918500FE
:1083000082179307C8F342CE809111029091120216
:10831000A0911302B0911402892B8A2B8B2B09F0A8
:1083200091C080919004882309F453C080909E04EA
:1083300090909F04A090A004B090A104C0908B04E2
:10834000D0908C04E0908D04F0908E0440918F04C6
:10835000C814D904EA04FB0480F480915B04909172
:108360005C0420915F04309160042817390728F4D9
:10837000415040938F04019714C08C149D04AE04A7
:10838000BF04E0F480915B0490915C0420915D0453
:1083900030915E048217930788F44F5F40938F04F7
:1083A000019690935C0480935B0440910D02509180
:1083B0000E0260910F02709110020EC08FEF9FEFBE
:1083C000DC0180930D0290930E02A0930F02B093F4
:1083D00010024FEF5FEFBA0180918F0487FD02C05A
:1083E000169A01C0169880918400909185004E964F
:1083F00020918F042223F1F0149A2091840030916F
:10840000850028173907C8F320918F0427FF02C081
:108410002F5F01C0215020938F04149820918F0466
:10842000222331F3209184003091850028173907E9
:10843000C8F3DDCF409311025093120260931302F0
:10844000709314028091A2049091A304A091A404BB
:10845000B091A504892B8A2B8B2B09F049C6A091DA
:108460001807B0911907109711F40C949C4A80904A
:108470009E0490909F04A090A004B090A10440910D
:108480009A0450919B0460919C0470919D04841601
:108490009506A606B706D8F010925A04109219074E
:1084A000109218079091B3098091B409981711F4AC
:1084B0000C949C4A8091B4098F5F8F708093B409AB
:1084C00040EDC42E47E0D42EE12CF12C1AC440918B
:1084D00096045091970460919804709199044815FE
:1084E00059056A057B0508F4AAC140919204509190
:1084F00093046091940470919504D6960D911D910A
:108500002D913C91D997401751076207730708F0E6
:1085100077C1411551056105710549F480905604F4
:1085200090905704A0905804B090590464C1E12C75
:10853000F980842E952F862F0A811B81FD81EE8183
:108540003F8128859C80E091EF17E89D912CFF27C3
:108550003091F017389D900CF11D1090F117189C78
:10856000F00DE99F900CF11D399FF00DE89FF00D83
:10857000092D1F2F099DE12D332722270F9FE00D85
:10858000311D2E1D199DE00D311D2E1D1F9F300D1B
:10859000211D032F122F099DF12C332722270F9F16
:1085A000F00C311D2E1D199DF00C311D2E1D1F9F2D
:1085B000300D211D032F122FEE278090560490912D
:1085C0005704809158040090B2040E2809F483C027
:1085D0003091AE04309FE1198E089E098E092091DA
:1085E000AF04209FE01981089E098E09F090B00425
:1085F000F09E801891098E09319FE01981089E092B
:108600008E09219F801891098E09F19E9019810988
:10861000099DF12C332722270F9FF00C311D2E1DB1
:10862000199DF00C311D2E1D1F9F300D211D032F94
:10863000122F3091AA04309FE10D8E1C9E1D8E1DBD
:108640002091AB04209FE00D811C9E1D8E1DF0909B
:10865000AC04F09E800C911D8E1D319FE00D811C9D
:108660009E1D8E1D219F800C911D8E1DF19E900DD3
:10867000811D099DF12C332722270F9FF00C311DFE
:108680002E1D199DF00C311D2E1D1F9F300D211D1B
:10869000032F122F3091A604309FE1198E089E09F6
:1086A0008E092091A704209FE01981089E098E0958
:1086B000F090A804F09E801891098E09319FE0196E
:1086C00081089E098E09219F801891098E09F19ECB
:1086D0009019810982C03091AE04309FE10D8E1C4B
:1086E0009E1D8E1D2091AF04209FE00D811C9E1DBC
:1086F0008E1DF090B004F09E800C911D8E1D319F58
:10870000E00D811C9E1D8E1D219F800C911D8E1DD4
:10871000F19E900D811D099DF12C332722270F9F7B
:10872000F00C311D2E1D199DF00C311D2E1D1F9FAB
:10873000300D211D032F122F3091AA04309FE11913
:108740008E089E098E092091AB04209FE0198108B4
:108750009E098E09F090AC04F09E801891098E0954
:10876000319FE01981089E098E09219F8018910987
:108770008E09F19E90198109099DF12C332722273A
:108780000F9FF00C311D2E1D199DF00C311D2E1D5B
:108790001F9F300D211D032F122F3091A604309FF3
:1087A000E10D8E1C9E1D8E1D2091A704209FE00DC3
:1087B000811C9E1D8E1DF090A804F09E800C911DC2
:1087C0008E1D319FE00D811C9E1D8E1D219F800CF2
:1087D000911D8E1DF19E900D811D11249C82F982A8
:1087E0000A831B83FD83EE833F832887912C992A7C
:1087F000A12CB12CA82A8BE395E121E0298B14C090
:10880000D2968D909D90AD90BC90D597F4CFB694B4
:10881000A79497948794D988DD0CD98A049625E18A
:108820008735920709F4EDC4FC0105911591259156
:108830003491081519052A053B0548F3E2C4409018
:108840008B0450908C0460908D0470908E044814BA
:1088500059046A047B0408F0C3C180918A04811121
:1088600021C0FD01EE5BFF4FE080F18002811381AA
:1088700078962081318142815381D2966D917D918C
:108880008D919C91D5970E9463C4DD24D394D0929E
:108890008A04E0911807F091190782A993A9A4A965
:1088A000B5A98EC1409186045091870460918804D7
:1088B00070918904DA960D911D912D913C91DD976F
:1088C000401751076207730708F073C1411551053E
:1088D0006105710549F48091560490915704A09167
:1088E0005804B09159046CC1F0E0E985842F352F0C
:1088F000262FAA857B856C855D85BE854F859889E9
:10890000B091EF17B89F612D55274091F017489F00
:10891000600D511D1090F117189E500DB39F600D02
:10892000511D439F500DB29F500DA62F752FA69F2E
:10893000B12D44279927A59FB00D411D9F1F769FFC
:10894000B00D411D9F1F759F400D911DA42F792FC4
:10895000A69FE12D44279927A59FE00D411D9F1F4C
:10896000769FE00D411D9F1F759F400D911DA42F07
:10897000792FBB27809156043091570420915804D9
:108980000090B2040F2A09F483C04091AE044A9FBC
:10899000B1198F0B3F0B2F0B9091AF049A9FB01919
:1089A00081093F0B2F0BE091B004EA9F8019310938
:1089B0002F0B479FB01981093F0B2F0B979F8019F1
:1089C00031092F0BE79F30192109A69FE12D44277C
:1089D0009927A59FE00D411D9F1F769FE00D411D2A
:1089E0009F1F759F400D911DA42F792F4091AA04C0
:1089F0004A9FB10D8F1F3F1F2F1F9091AB049A9F6D
:108A0000B00D811D3F1F2F1FE091AC04EA9F800D28
:108A1000311D2F1F479FB00D811D3F1F2F1F979F97
:108A2000800D311D2F1FE79F300D211DA69FE12DC9
:108A300044279927A59FE00D411D9F1F769FE00DBC
:108A4000411D9F1F759F400D911DA42F792F4091AF
:108A5000A6044A9FB1198F0B3F0B2F0B9091A704CF
:108A60009A9FB01981093F0B2F0BE091A804EA9F50
:108A7000801931092F0B479FB01981093F0B2F0B2C
:108A8000979F801931092F0BE79F3019210982C068
:108A90004091AE044A9FB10D8F1F3F1F2F1F909131
:108AA000AF049A9FB00D811D3F1F2F1FE091B004AE
:108AB000EA9F800D311D2F1F479FB00D811D3F1F65
:108AC0002F1F979F800D311D2F1FE79F300D211DF8
:108AD000A69FE12D44279927A59FE00D411D9F1FCB
:108AE000769FE00D411D9F1F759F400D911DA42F86
:108AF000792F4091AA044A9FB1198F0B3F0B2F0B7E
:108B00009091AB049A9FB01981093F0B2F0BE09114
:108B1000AC04EA9F801931092F0B479FB0198109D6
:108B20003F0B2F0B979F801931092F0BE79F3019AF
:108B30002109A69FE12D44279927A59FE00D411DFE
:108B40009F1F769FE00D411D9F1F759F400D911D3A
:108B5000A42F792F4091A6044A9FB10D8F1F3F1F6C
:108B60002F1F9091A7049A9FB00D811D3F1F2F1FAB
:108B7000E091A804EA9F800D311D2F1F479FB00D83
:108B8000811D3F1F2F1F979F800D311D2F1FE79FB6
:108B9000300D211D1124E987AA877B876C875D87AB
:108BA000BE874F87988B90E0932BA0E0B0E0A22B7C
:108BB00007C0A65ABF4F8D919D910D90BC91A02DDD
:108BC0002BE335E141E0498BF901459155916591E0
:108BD0007491481759076A077B0708F49CC3A9C317
:108BE00080918F048823E1F0FD01E85BFF4F408115
:108BF000518160E070E000910D0210910E02209111
:108C00000F0230911002401751076207730741F0BD
:108C1000109211021092120210921302109214027A
:108C20004091090250910A0260910B0270910C026E
:108C300077FF5FC0AE5ABF4FCD90DD90ED90FC90B6
:108C40008BE395E121E0FC0145915591659174918B
:108C50004C155D056E057F0550F4F694E794D794A6
:108C6000C794220F049675E18735970761F7209323
:108C7000910480E2C816D104E104F10428F470E202
:108C8000C72ED12CE12CF12C90E2C91AD108E108B1
:108C9000F108C114A8E0DA06E104F10408F405C4FF
:108CA000B4E0DB9EC0011124855C9E4EFC0132962F
:108CB00025913491EC2D6627E39FA001E29F410DA1
:108CC000561F0694461F561F112460E070E0FC01F9
:108CD00025913491C901A0E0B0E0841B950BA60B4F
:108CE000B70B8093090290930A02A0930B02B093F2
:108CF0000C02C0900902D0900A02E0900B02F090A2
:108D00000C028091180790911907892B09F0E8C18E
:108D10000E94E5C49093190780931807892B09F4E2
:108D2000DFC1E0911807F0911907808183FF3EC0F1
:108D300085899689A789B08D80938210909383103E
:108D4000A0938410B0938510818D928DA38DB48DE6
:108D50008093861090938710A0938810B093891009
:108D6000858D968DA78DB0A180938A1090938B10DE
:108D7000A0938C10B0938D1081A192A1A3A1B4A156
:108D800080938E1090938F10A0939010B0939110B9
:108D90009091B3098091B409981709F4B9CF8091E3
:108DA000B4098F5F8F708093B409B2CFC588D6881D
:108DB000E788F08C81E0C114D104E104F10409F4E6
:108DC00080E0018D128D238D348D01151105210553
:108DD000310509F08260458D568D678D70A1411572
:108DE00051056105710509F0846080935A04109261
:108DF00086041092870410928804109289041092BD
:108E0000920410929304109294041092950485A1F8
:108E100096A1A7A1B0A580939A0490939B04A093D8
:108E20009C04B0939D04882499245401881A990ABB
:108E3000AA0ABB0A8092820490928304A0928404BE
:108E4000B092850480927E0490927F04A092800468
:108E5000B092810480927A0490927B04A0927C0468
:108E6000B0927D048092760490927704A092780468
:108E7000B0927904CC0CDD1CEE1CFF1CC092660481
:108E8000D0926704E0926804F0926904000F111F09
:108E9000221F331F00936A0410936B0420936C0409
:108EA00030936D04440F551F661F771F40936E0467
:108EB00050936F04609370047093710441A152A1A8
:108EC00063A174A1440F551F661F771F409372045E
:108ED000509373046093740470937504880F991F02
:108EE000AA1FBB1F8093620490936304A093640441
:108EF000B093650410929E0410929F041092A004F7
:108F00001092A10482A593A5A4A5B5A5809396046B
:108F100090939704A0939804B093990486A597A57D
:108F2000A0A9B1A980938B0490938C04A0938D0485
:108F3000B0938E0481A580936104DF01A95BBF4FCC
:108F40009C9190939004992339F115962D913C9121
:108F500011973093600420935F0412972D913C91F8
:108F6000119730935E0420935D04109211021092C9
:108F70001202109213021092140212972D913C913A
:108F8000A90160E070E040930D0250930E026093DF
:108F90000F02709310020CC088248A94982C5401FC
:108FA00080920D0290920E02A0920F02B0921002D7
:108FB000EA5BFF4F90812091550492130AC02091E3
:108FC000080230E0482F082E000C550B42175307BB
:108FD00031F090935504809308020E94B5C48091AB
:108FE000370581110E94C5BD2FEF3FEFA9012093E6
:108FF000090230930A0240930B0250930C02E09155
:109000001807F0911907DF01DE96ED90FD900D91A4
:109010001C9122A933A944A955A9EA5AFF4F60819E
:109020007181828193810E9463C410928A04E091CD
:109030001807F0911907EA5AFF4F80809180A280AB
:10904000B3808BE395E121E0FC0145915591659159
:109050007491481559056A057B0558F4B694A79490
:1090600097948794220F0496A7E5B5E1A817B9074E
:1090700059F720939104B0E28B169104A104B10436
:1090800028F4B0E28B2E912CA12CB12C30E2831A63
:109090009108A108B108811448E09406A104B10424
:1090A00008F427C254E0959EC0011124855C9E4EB1
:1090B000FC01329625913491782D6627739FA0018B
:1090C000729F410D561F0694461F561F1124FC0126
:1090D000C590D490E12CF12CC41AD50AE108F1080E
:1090E000C092A204D092A304E092A404F092A5043A
:1090F0000091A2041091A3042091A4043091A5042E
:109100004091110250911202609113027091140269
:10911000F02E198BF22FE32F4017510762077307C8
:1091200020F4F42E598BF62FE72F8F2D9989AF2F2E
:10913000BE2F0097E1E0AE07B10520F08FEF9FEF63
:10914000A0E0B0E0081B190B2A0B3B0B0093A20414
:109150001093A3042093A4043093A5044F3FFFEF82
:109160005F076F077F0761F0481B590B6A0B7B0B8A
:1091700040931102509312026093130270931402F1
:10918000F8942091840030918500205F3F4F4A89F8
:1091900041504A8B442341F0280E391E22163306D3
:1091A00010F40C94603F01C01901309289002092A4
:1091B0008800789462960FB6F894DEBF0FBECDBFDC
:1091C000DF91CF911F910F91FF90EF90DF90CF90A3
:1091D000BF90AF909F908F907F906F905F904F90D7
:1091E0003F902F90089580910B0180958870809317
:1091F00009010C946C4080910B01887080930901E7
:1092000064C839893093910480E288169104A104DE
:10921000B10428F430E2832E912CA12CB12C30E241
:10922000831A9108A108B108811488E09806A10466
:10923000B10420F1E4E09E9EC0011124855C9E4EA5
:10924000FC01329625913491F82DEE27F39F7001A1
:10925000F29FE10CFE1E0694EE1EFE1E1124FC0180
:10926000C590D490860120E030E0480159018E1865
:109270009F08A108B1087501640122C0950184010D
:109280003695279517950795F801EC7FCF01855CFA
:10929000924FFC01C590D490FC01329625913491F7
:1092A000E82DE770E29FC001E39F900D112423E0B9
:1092B000969587952A95E1F7C81AD90AE12CF12CE1
:1092C0004C0D5D1D6E1D7F1D4093920450939304C1
:1092D00060939404709395049091900480918F040E
:1092E000992309F473C0882309F40BCDA85BBF4F01
:1092F0008D919C91A0E0B0E040910D0250910E0242
:1093000060910F027091100284179507A607B707A6
:1093100009F05FC0F6CCB695A79597958795D98843
:10932000DD0CD98A2C5F3F4F45E12735340709F022
:109330004BCC59895093910480329105A105B10518
:1093400020F480E290E0A0E0B0E08097A109B109AC
:10935000811558E09507A105B10508F443C074E0F4
:10936000979F90011124255C3E4EF901329645915C
:109370005491EE27859FB001849F610D7E1F069456
:109380006E1F7E1F1124F901C590D490E12CF12CA1
:10939000C61AD70AE108F1088091860490918704E3
:1093A000A0918804B09189048C0D9D1DAE1DBF1D38
:1093B0008093860490938704A0938804B0938904D3
:1093C00080919004811130C080918F04882309F42A
:1093D00098CC109211021092120210921302109265
:1093E00014028FCCAC01BD017695679557954795D2
:1093F000FA01EC7F9F01255C324FF901C590D490B2
:10940000F9013296459154918770849F9001859F10
:10941000300D1124F3E036952795FA95E1F7C21A3D
:10942000D30AE12CF12CB8CF8989480E511C611C5C
:10943000711C8091180790911907481459046A0407
:109440007B04D8F420918F04222309F45ACCFC0128
:10945000E85BFF4F20813181A90160E070E000915D
:109460000D0210910E0220910F0230911002401750
:1094700051076207730709F444CC1092110210924D
:1094800012021092130210921402FC01E85BFF4FCB
:1094900080819181A0E0B0E080930D0290930E0254
:1094A000A0930F02B09310022CCCD701C601B69541
:1094B000A79597958795FC01EC7FCF01855C924F2E
:1094C000FC0125913491FC013296459154916C2D0B
:1094D0006770649FC001659F900D112463E09695AD
:1094E00087956A95E1F7281B390BC901A0E0B0E028
:1094F000F8CBD501C401B695A79597958795FC0142
:10950000EC7FCF01855C924FFC01C590D490FC01AB
:10951000329625913491482D4770429FC001439F58
:10952000900D1124A3E096958795AA95E1F7C81AA6
:10953000D90AE12CF12CD4CD80EDC82E87E0D82EAD
:10954000E12CF12CE5CBCF92DF92EF92FF92CF93FB
:10955000DF936B017C01EA0121E338E040EA50EC43
:109560000E94AFEC87FD23C022E430E04CE553E4D9
:10957000C701B6010E943DE61816CCF0C880D9801C
:10958000EA80FB802FE632E143E85AEBC701B601DF
:109590000E94AFEC87FD0BC0C1E022E430E04CE557
:1095A00053E4C701B6010E943DE618160CF4C0E072
:1095B0008C2FDF91CF91FF90EF90DF90CF900895A7
:1095C0000F931F93CF93DF93FC01A685B7858D0181
:1095D00000581F4FE8018881998101968F7799275C
:1095E000AD014E575F4FEA012881398128173907AD
:1095F000D1F3E80128813981A20FB31F6C93A685AE
:10960000B785A058BF4F11969C938E93A689B789B2
:109610002C9181E090E0078C02C0880F991F0A947A
:10962000E2F7822B8C9381E081A30488F589E02DF9
:1096300080818064808381E090E0DF91CF911F91F1
:109640000F910895FC0181A1882329F0A489B5898F
:109650008C9186FFFBCF11A20895FC01A485B585EE
:10966000FD01E058FF4F2081318132968081918148
:109670002817390779F080819181A80FB91F8C9143
:10968000208131812F5F3F4F2F7733273183208314
:1096900090E008958FEF9FEF0895DC011C96ED9107
:1096A000FC911D97DF01A058BF4F2D913C91119760
:1096B00012968D919C9111972817390739F08D9149
:1096C0009C91E80FF91F808190E008958FEF9FEF44
:1096D0000895FC0124853585F901E058FF4F80810C
:1096E000918132962081318180589F4F821B930B4C
:1096F00060E870E00C9472ED0895089580E090E0C9
:109700000895CF92DF92EF92FF92C0903002D090F6
:109710003102E0903202F0903302FC0180819181AD
:10972000A281B3818093300290933102A0933202E0
:10973000B09333020E945CCAC0923002D0923102D0
:10974000E0923202F0923302FF90EF90DF90CF90E0
:1097500008958091961890919718981759F0E92FCD
:10976000F0E0EA5EF74E80819F5F9F7790939718B5
:1097700090E008958FEF9FEF08951F920F920FB61C
:109780000F9211240BB60F922F938F939F93EF9309
:10979000FF9320919718E091961881E08E0F8F77B4
:1097A0009091C600281729F0F0E0EA5EF74E90830A
:1097B000E82FE0939618FF91EF919F918F912F9151
:1097C0000F900BBE0F900FBE0F901F9018958091B9
:1097D000210490912204009731F04AE050E060E0CB
:1097E00070E00C9491E360E070E0CB010895EFDF4E
:1097F00097FD0AC0ECDF6F3F71058105910509F007
:109800002CF4E5DF862F089580E008958FEF08950A
:109810008091210490912204892B31F0E8DF91E0BE
:10982000811103C090E001C091E0892F08950F934A
:109830001F93CF938091210490912204009711F1FE
:10984000FC018F01C1912C2F2F7DA9F0C53411F09F
:10985000C536B9F7F801108260E070E0809121040C
:10986000909122040E943EE2F801C083562F472FB8
:10987000382F292F0BC060E070E0CF911F910F911E
:109880000C943EE250E040E030E020E0652F742F81
:10989000832F922FCF911F910F91089581548A3178
:1098A00008F042C0E82FF0E040910D1850910E18DA
:1098B00060910F187091101804C0769567955795B0
:1098C00047958A95D2F7842F817040FF2FC0ED50C5
:1098D000F84E9081992309F1E0917210F091731084
:1098E000E90FF11D908120ED290F2A3098F09E326A
:1098F00011F491810CC09D3211F09B3271F4918171
:1099000020ED290F2A3030F09E3239F492819053A5
:109910009A3018F42E2F9F2F02C020E090E0209361
:10992000210490932204089580E008950895B6DFFD
:10993000882341F081E02091210430912204232BDF
:1099400009F480E0089580E1E2E3F4E0AEEAB0E1FA
:1099500001900D928A95E1F708952F923F924F92D0
:109960005F926F927F928F929F92AF92BF92CF92AF
:10997000DF92EF92FF920F931F93CF93DF9300D06C
:109980001F921F92CDB7DEB77C018B016A011901CE
:109990008090320490903304A0903404B090350449
:1099A000A5019401FC0160817181828193810E94F3
:1099B0003DE6F1E0FD83811112C020913604309123
:1099C00037044091380450913904F8016081718165
:1099D000828193810E943DE6811101C01D82F601C2
:1099E0004080518062807380209115023091160270
:1099F0004091170250911802C301B2010E943DE646
:109A0000882309F453C040921502509216026092C6
:109A100017027092180220E030E040E450E46091B8
:109A2000FB067091FC068091FD069091FE060E9457
:109A300065EB69837A838B839C838092AE109092CE
:109A4000AF10A092B010B092B110809136049091F6
:109A50003704A0913804B09139048093B2109093E8
:109A6000B310A093B410B093B510F601808191812A
:109A7000A281B3818093B6109093B710A093B810D1
:109A8000B093B91080913E0490913F04A09140049E
:109A9000B09141048093BA109093BB10A093BC1076
:109AA000B093BD10CE0101962CDE4DDFFD81FF236A
:109AB00009F16090F7067090F8068090F906909092
:109AC000FA06A090F306B090F406C090F506D09088
:109AD000F6069501A601B301C4010E94AFEC181669
:109AE00014F05301640120E030E040E251E4B5019C
:109AF000C6010CC020E030E040EC5FE36091FF065F
:109B00007091000780910107909102070E9465EB18
:109B100069837A838B839C8320912004222349F0DC
:109B2000AB01BC018BE595E10E9437C58AE00E943C
:109B3000CC89F70180819181A281B3818093AE109D
:109B40009093AF10A093B010B093B110F801808142
:109B50009181A281B3818093B2109093B310A093AE
:109B6000B410B093B510F10120813181428153814D
:109B70006091BA107091BB108091BC109091BD1093
:109B80000E9489EA6093BA107093BB108093BC1056
:109B90009093BD10CE010196B4DDD5DE0F900F90ED
:109BA0000F900F900F90DF91CF911F910F91FF9029
:109BB000EF90DF90CF90BF90AF909F908F907F906D
:109BC0006F905F904F903F902F90089580E1EEEA64
:109BD000F0E1A2E3B4E001900D928A95E1F70895D7
:109BE0009C0197FD0EC08436910584F064E670E018
:109BF0000E9472EDCB016AE070E00E9472ED805D20
:109C000006C03195219531098DE201C080E2809333
:109C10002D042A30310564F0EAE0F0E0C901BF010B
:109C20000E9472EDCB01BF010E9472ED805D01C008
:109C300080E280932E04C9016AE070E00E9472ED18
:109C4000805D80932F048DE294E008958E36910517
:109C50001CF02EE680E002C0282F892F20934404B8
:109C6000809345040C94B6762F923F924F925F9268
:109C70006F927F928F929F92AF92BF92CF92DF921C
:109C8000EF92FF920F931F93CF93DF93CDB7DEB781
:109C9000C455D1090FB6F894DEBF0FBECDBFEAE1BF
:109CA000F8E184918F010F5F1F4F882321F00E94FC
:109CB000CC89F801F6CF0E9469B481110C94165832
:109CC00080E090E0A0E8BFE38093A6109093A710F7
:109CD000A093A810B093A91080E090E0A0ECB0E4AD
:109CE0008093AA109093AB10A093AC10B093AD10DA
:109CF0008DEC9CECACE4BEE38093A2109093A31097
:109D0000A093A410B093A51080E090E0A8ECB1E47B
:109D10008093240590932505A0932605B0932705ED
:109D20008CE390E0909323058093220588EC90E0EB
:109D3000909321058093200510921F058FE4F7DD95
:109D4000882311F074DD04C060E070E080E190E4ED
:109D50006BAF7CAF8DAF9EAF83E4E9DD882311F05C
:109D600057DD02C083E49ADD61968FAF61978BE483
:109D7000DEDD882311F04CDD02C08BE48FDD6096C0
:109D80008FAF609782E4D3DD8823E9F050DD0E9435
:109D9000CDEB70932305609322056115710599F051
:109DA000685271096536710570F0E5EEF7E184914E
:109DB0008F010F5F1F4F882311F40C9416580E94D7
:109DC000CC89F801F4CF8CE4B2DD882351F12FDD8A
:109DD0006B017C016093A2107093A3108093A41078
:109DE0009093A51020E030E0A9010E94AFEC87FD20
:109DF0000AC020E030E040E050E4C701B6010E9414
:109E00003DE6181674F4EDEBF7E184918F010F5FD6
:109E10001F4F882311F40C9416580E94CC89F80126
:109E2000F4CF81E53BDD882309F440C08091210413
:109E300090912204892B19F4E2E9F7E12BC0F7DCB9
:109E40006B017C016093AA107093AB108093AC10EF
:109E50009093AD102DEC3CEC4CE45DE30E94AFEC34
:109E600087FD0AC020E030E040E751E4C701B601B9
:109E70000E943DE61816D4F4E1E6F7E184918F01E3
:109E80000F5F1F4F882311F40C9416580E94CC8941
:109E9000F801F4CF84918F010F5F1F4F882311F4D5
:109EA0000C9416580E94CC89F801F4CF83E53FDD6D
:109EB000882319F1BCDC4B015C012DEC3CEC4CEC33
:109EC0005DE30E94AFEC87FD0AC020E030E040E88F
:109ED0005FE3C501B4010E943DE61816ACF4EAE365
:109EE000F7E184918F010F5F1F4F882311F40C94C9
:109EF00016580E94CC89F801F4CF5DEC852E5CECFD
:109F0000952EA92C5EE3B52E80E5C8DC882309F4E4
:109F100043C08091210490912204892B71F4E2E0E6
:109F2000F7E184918F010F5F1F4F882311F40C9488
:109F300016580E94CC89F801F4CF80911F058F5FDD
:109F400080931F0574DC6B017C0160932405709382
:109F50002505809326059093270520E030E0A90190
:109F60000E94AFEC87FD0AC020E030E048EC51E4ED
:109F7000C701B6010E943DE6181674F4EAEDF6E159
:109F800084918F010F5F1F4F882311F40C94165892
:109F90000E94CC89F801F4CF86E4C9DC882319F14A
:109FA00046DC6B017C0120E030E040E85FE30E948A
:109FB000AFEC87FD0AC020E030E040E850E4C70184
:109FC000B6010E943DE61816A4F4E1EBF6E1849197
:109FD0008F010F5F1F4F882311F40C9416580E94B5
:109FE000CC89F801F4CFC12CD12C40EEE42E4FE304
:109FF000F42EA7019601C701B6010E94A2E69B01BB
:10A00000AC0160E070E084E490E40E9465EB209194
:10A01000A6103091A7104091A8105091A9100E944D
:10A02000A2E62B013C01A5019401C501B4010E94E7
:10A03000A2E6A70196010E94A2E62CEE31E548EBCC
:10A040005DE30E9465EB9B01AC01C301B2010E947C
:10A05000A2E66093A6107093A7108093A810909327
:10A06000A91088E464DC8823C9F0E1DB0E94CDEB11
:10A070007093210560932005655A71096437710555
:10A0800068F0E3E8F6E184918F010F5F1F4F8823AA
:10A0900009F4CCC70E94CC89F801F5CF85E5FEDB39
:10A0A0008823E9F00E94FE5861157105810591052C
:10A0B00011F00E9435E28091210490912204892BB5
:10A0C00011F0B5DB04C060E070E088E492E46093D6
:10A0D0001B0570931C0580931D0590931E0582E55A
:10A0E000DDDB81110DC0EFE4F6E184918F010F5F9C
:10A0F0001F4F882309F49AC70E94CC89F801F5CF35
:10A100008091210490912204892BA9F060DB2F9685
:10A110007FAF6EAF2F97161617069CF0EBE1F6E1B6
:10A1200084918F010F5F1F4F882309F47FC70E941E
:10A13000CC89F801F5CF8AE190E02F969FAF8EAFE2
:10A140002F9788E5F4DB882361F071DB20911404FC
:10A150003091150440911604509117040E9488EA2A
:10A1600008C060913204709133048091340490915E
:10A170003504609317057093180580931905909323
:10A180001A0589E5D4DB882361F051DB209118049E
:10A190003091190440911A0450911B040E9488EADE
:10A1A00008C0609136047091370480913804909112
:10A1B00039046093130570931405809315059093EB
:10A1C00016056091170570911805809119059091F9
:10A1D0001A0543E155E0B7D981110DC0E1EFF5E172
:10A1E00084918F010F5F1F4F882309F41FC70E94BE
:10A1F000CC89F801F5CF84E451DB91E089270E94F6
:10A200002CAC20E030E040EA50E460913A047091D8
:10A210003B0480913C0490913D040E943DE687FF01
:10A2200014C0198A1A8A1B8A1C8A80E090E0A0EA6E
:10A23000B0E489839A83AB83BC83BE016F5E7F4F9A
:10A24000CE0101960E944BB4C1DCD8D76B017C01D2
:10A25000A8E8CA0EA3E1DA1EE11CF11C80912205D8
:10A2600090912305F3DC6091220570912305072E60
:10A27000000C880B990B0E9443E69B01AC01609196
:10A2800046047091470480914804909149040E94CB
:10A2900088EA4B015C0120E030E0A9010E94AFECAC
:10A2A00087FF04C0B7FAB094B7F8B09420E030E06C
:10A2B00040E450E4C501B4010E94AFEC1816F4F478
:10A2C0009DD7DC01CB018C199D09AE09BF09B7FDF3
:10A2D0000EC094D76B017C01B8E8CB0EB3E1DB1E56
:10A2E000E11CF11C0E94FC758AE00E94CC890E944E
:10A2F00002A18091961880939718B5CF8091200580
:10A30000909121050E94F3596091200570912105DB
:10A31000072E000C880B990B0E9443E69B01AC01B1
:10A3200060914C0470914D0480914E0490914F04C3
:10A330000E9488EA4B015C0120E030E0A9010E9404
:10A34000AFEC87FF04C0B7FAB094B7F8B09420E040
:10A3500030E040E450E4C501B4010E94AFEC1816AF
:10A36000F4F44CD7DC01CB018C199D09AE09BF096F
:10A37000B7FD0EC043D76B017C01E8E8CE0EE3E1E8
:10A38000DE1EE11CF11C0E94FC758AE00E94CC8953
:10A390000E9402A18091961880939718B5CF1092D1
:10A3A0003E0410923F0410924004109241040E9417
:10A3B0001AB380911F05882399F1C5DA20912405ED
:10A3C0003091250540912605509127056091BA10DE
:10A3D0007091BB108091BC109091BD100E9489EAD1
:10A3E0006093BA107093BB108093BC109093BD1013
:10A3F00020E030E040E751E46091FF0670910007F3
:10A4000080910107909102070E9465EB69837A832E
:10A410008B839C83CE01019674D995DA0E9427B173
:10A4200080E2E3EFF4E0DF01282F1D922A95E9F79F
:10A43000E3EDF4E0DF01282F1D922A95E9F7E3EB25
:10A44000F4E0DF011D928A95E9F77DDA8091A21090
:10A450009091A310A091A410B091A5108093B61074
:10A460009093B710A093B810B093B91019821A82C4
:10A470001B821C829E012F5F3F4F46EB50E162EB37
:10A4800070E18EEA90E169DA9E01255C3F4F46EB70
:10A4900050E162EB70E18EEA90E15FDA6196BFAD68
:10A4A0006197BB2329F066E374E082E394E004C083
:10A4B00063E175E087E195E00E948DD8298F3A8F9E
:10A4C0004B8F5C8F6D8F7E8F3FAF2D962FAF2D976B
:10A4D0002D96EFAD2D97E7FD81C4FFADF7FD7EC44E
:10A4E00024E0E202F0011124E350F64F4080518055
:10A4F000628073803FAD84E03802F0011124E7519F
:10A50000F64FD080C180328023808D2D9C2DA32DCD
:10A51000B22D8FAB98AFA9AFBAAFAE01495C5F4F18
:10A52000B201C30110D8882309F45CC420E030E0F4
:10A5300040EA50E4B201C3010E9489EAF62E072FD7
:10A54000182FE92E862F902FA12FBE2D8BAB9CAB01
:10A55000ADABBEAB8D2D9C2DA32DB22D8FA798AB8F
:10A56000A9ABBAAB2D969FAD2D97911152C0AFAD4F
:10A57000A11105C05F2D402F312F2E2D04C0542D69
:10A58000452D362D272D852F942FA32FB22F8BAB42
:10A590009CABADABBEABBFADB43034F4F42C052DE9
:10A5A000162DE72CBB2369F020E030E040EA50E4B0
:10A5B0006D2D7C2D832D922D0E9488EA362F272F1A
:10A5C00003C09601832D922D432F522FBC014FA71C
:10A5D00058AB69AB7AABEFADE4300CF0A7C020E02C
:10A5E00030E040EA50E46D2D7C2D832D922D0E94A9
:10A5F00089EA21966FAF219723967FAF23972596FF
:10A600008FAF259727969FAF2797FFADF11185C094
:10A6100099C02D962FAD2D9724300CF453C03FAD2B
:10A6200034305CF020E030E040EA50E4B201C30195
:10A630000E9488EA362F272F03C0342D252DC30111
:10A64000432F522FBC014BAB5CAB6DAB7EAB8FADE0
:10A650008111E3C420E030E040EA50E4B201C301DC
:10A660000E9488EAF62E072F182FE92E20E030E00E
:10A6700040EA50E46D2D7C2D832D922D0E9489EAB5
:10A680006FA778AB89AB9AAB9FAD992309F44EC005
:10A6900020E030E040EA50E46D2D7C2D832D922D9A
:10A6A0000E9488EA21966FAF219723967FAF239768
:10A6B00025968FAF259727969FAF2797AFADA430EC
:10A6C00064F140C0BFADB1110DC020E030E040EA00
:10A6D00050E4B201C3010E9488EAF62E072F182F1A
:10A6E000E92E0FC0EFADE430B4F120E030E040EAF5
:10A6F00050E4B201C3010E9488EA6BAB7CAB8DAB26
:10A700009EAB2196DFAE21972396CFAE2397259659
:10A710003FAE259727962FAE279732ED832E33E550
:10A72000932E3BE7A32E31E4B32E29C02196DFAE52
:10A7300021972396CFAE239725963FAE2597279650
:10A740002FAE279722ED822E23E5922E2BEFA22EFD
:10A7500020E4B22E14C02196DFAE21972396CFAE0F
:10A76000239725963FAE259727962FAE279792EDF4
:10A77000892E93E5992E9BEFA92E91E4B92E8BA9F2
:10A780009CA9ADA9BEA92C968CAF9DAFAEAFBFAFB3
:10A790002C979C01AD01B201C3010E9488EA698B2C
:10A7A0007A8B8B8B9C8B4FA458A869A87AA8A3019D
:10A7B00092016D2D7C2D832D922D0E9488EA6D8B48
:10A7C0007E8B8F8B988F2C962CAD3DAD4EAD5FADB3
:10A7D0002C976091320470913304809134049091ED
:10A7E00035040E9488EA2C966CAF7DAF8EAF9FAF88
:10A7F0002C97A301920160913604709137048091E7
:10A800003804909139040E9488EA2B013C018F2D75
:10A81000902FA12FBE2D89839A83AB83BC83219671
:10A820008FAD219723969FAD23972596AFAD2597A2
:10A830002796BFAD27978D839E83AF83B88780917E
:10A84000A2109091A310A091A410B091A510898797
:10A850009A87AB87BC872DEC3CEC4CEC5CE3C501E4
:10A86000B4010E94A2E62091A6103091A710409159
:10A87000A8105091A9100E94A2E620913E043091A8
:10A880003F0440914004509141040E9489EA6D8741
:10A890007E878F87988B2C962CAD3DAD4EAD5FADEE
:10A8A0002C97CA01B9010E94A2E66B017C01A301A9
:10A8B0009201C301B2010E94A2E69B01AC01C70153
:10A8C000B6010E9489EA20E030E040E050E40E94B6
:10A8D000AFEC18160CF046C00E9427B11BA21CA2B8
:10A8E0001DA21EA220E030E040E05FE360913A0448
:10A8F00070913B0480913C0490913D040E9489EA50
:10A900006F8F78A389A39AA39E012D5D3F4FAE015F
:10A91000415E5F4F66E374E082E394E01ED81BA2C1
:10A920001CA21DA21EA220E030E040E05FE3609187
:10A93000A2107091A3108091A4109091A5100E9474
:10A9400089EA6F8F78A389A39AA39E012D5D3F4F5B
:10A95000AE01415E5F4FBE01615D7F4FCE01C39688
:10A960000E94AD4C1F8E18A219A21AA29E01215E50
:10A970003F4F42EA50E1BE01615D7F4FCE01C39679
:10A980000E94AD4C0E9453B1409030025090310271
:10A990006090320270903302E090F706F090F80673
:10A9A0000091F9061091FA06A090F306B090F40613
:10A9B000C090F506D090F6069501A601B701C80132
:10A9C0000E94AFEC181614F47501860120E030E007
:10A9D00040E251E4B701C8010E9465EB6093300288
:10A9E00070933102809332029093330240E0BE01B3
:10A9F0006F5E7F4FCE0101960E94CEA4409230023E
:10AA00005092310260923202709233020E94A34C43
:10AA1000ADEFB9E02496BFAFAEAF249722961FAE3C
:10AA20001EAE229701E010E021960FAC219702C0E4
:10AA3000000F111F0A94E2F72296EEADFFAD2297A8
:10AA400031962296FFAFEEAF229721E030E02196BB
:10AA50000FAC219702C0220F331F0A94E2F76396CE
:10AA60003FAF2EAF639783EB282E84E0382E83EF21
:10AA700094E02A969FAF8EAF2A97A3EDB4E0289674
:10AA8000BFAFAEAF2897E9EEF9E02696FFAFEEAF85
:10AA900026972A962EAD3FAD2A9765963FAF2EAFEB
:10AAA0006597D9018D919C919C0120233123232B03
:10AAB00009F4ADC06396EEADFFAD63978E239F237F
:10AAC000892B09F4A4C02896AEADBFAD28978D910F
:10AAD0009C9180239123892B09F099C020E030E0DC
:10AAE00040E050E42496AEADBFAD24976D917D91CA
:10AAF0008D919C910E9489EA6B017C0120E030E0FD
:10AB000040E050E42496EEADFFAD2497648175815A
:10AB1000868197810E9488EA4B015C0120E030E049
:10AB200040E850ECC701B6010E943DE687FD70C1C8
:10AB300020E030E04BE553E4C701B6010E94AFECE2
:10AB4000181634F4C12CD12CBBE5EB2EB3E4FB2E4C
:10AB5000CBA6DCA6EDA6FEA62696AEADBFAD26978B
:10AB60004D905D906D907C9020E030E040E85FE398
:10AB7000C301B2010E943DE687FD51C120E030E0F3
:10AB80004BE553E4C301B2010E94AFEC181634F454
:10AB9000412C512CFBE56F2EF3E47F2E4F8E58A2F3
:10ABA00069A27AA24FA258A669A67AA620E030E050
:10ABB00040E850ECC501B4010E943DE687FD36C176
:10ABC00020E030E04BE553E4C501B4010E94AFEC56
:10ABD000181634F4812C912C7BE5A72E73E4B72E44
:10ABE0008BA29CA2ADA2BEA2AE01495D5F4FC70180
:10ABF000B6010E94A34A811120C12896EEADFFAD97
:10AC0000289780819181802B912B918380832A9634
:10AC10002EAD3FAD2A972E5F3F4F2A963FAF2EAF06
:10AC20002A976596AEADBFAD65978D919C918023B7
:10AC30009123892B09F4A6C0F90180819181802399
:10AC40009123892B09F49EC0F10180819181802399
:10AC50009123892B09F096C020E030E040E050E4D9
:10AC60002696AEADBFAD26976D917D918D919C914D
:10AC70000E9489EA2B013C0120E030E040E050E4F2
:10AC80002696EEADFFAD269764817581868197810A
:10AC90000E9488EA4B015C012496AEADBFAD2497BB
:10ACA000CD90DD90ED90FC9020E030E040E850EC5D
:10ACB000C701B6010E943DE687FDFFC020E030E0FD
:10ACC0004BE553E4C701B6010E94AFEC181634F40B
:10ACD000C12CD12C5BE5E52E53E4F52ECBA2DCA2F2
:10ACE000EDA2FEA2CBA6DCA6EDA6FEA620E030E0FB
:10ACF00040E85FE3C301B2010E943DE687FDE4C086
:10AD000020E030E04BE553E4C301B2010E94AFEC18
:10AD1000181634F4412C512C3BE5632E33E4732E8A
:10AD20004FA258A669A67AA620E030E040E85FE38B
:10AD3000C501B4010E943DE687FDCDC020E030E0B2
:10AD40004BE553E4C501B4010E94AFEC181634F48E
:10AD5000812C912C9BE5A92E93E4B92E8F8E98A27D
:10AD6000A9A2BAA2AE01495D5F4FC701B6010E9418
:10AD7000A34A8111B7C0F10180819181802B912B71
:10AD800091838083F2E02F0E311C28962EAD3FADCB
:10AD900028972E5F3F4F28963FAF2EAF28972696D5
:10ADA0008EAD9FAD2697049626969FAF8EAF2697C1
:10ADB0009DEB291694E0390609F06BCE2496AEADD2
:10ADC000BFAD249714962496BFAFAEAF24972296BA
:10ADD000EEADFFAD2297359709F024CE80919618FD
:10ADE000809397182F962EAD3FAD2F9721503109A4
:10ADF0002F963FAF2EAF2F97232B09F4B3C02D967C
:10AE00003FAD2D9737FDAEC08FAD87FF47CBAAC0B2
:10AE1000C12CD12CA0E8EA2EA0ECFA2E99CE412C20
:10AE2000512CE0E86E2EEFE37E2EB8CE812C912CD3
:10AE300060E8A62E60ECB62ED3CEAE01415E5F4F29
:10AE4000C501B4010E94A34A882309F4D6CE80919B
:10AE50002004882321F1B701A6018BEC95E10E9423
:10AE600037C54FA158A569A57AA585EC95E10E9443
:10AE700037C54BA15CA16DA17EA18BEB95E10E9432
:10AE800037C54F8D58A169A17AA185EB95E10E9444
:10AE900037C589E20E94CC898AE00E94CC899E0154
:10AEA000215E3F4FAE014D5D5F4FBE01695D7F4F3B
:10AEB000CE018B960E9483B1A0CEC12CD12C40E84C
:10AEC000E42E40ECF42E0ACF412C512C20E8622EC7
:10AED0002FE3722E25CF812C912C80E8A82E8FE3B2
:10AEE000B82E3CCFAE01415E5F4FC701B6010E9454
:10AEF000A34A882309F43FCF80912004882321F1BD
:10AF0000B701A60181E995E10E9437C54FA158A577
:10AF100069A57AA58BE895E10E9437C54BA15CA194
:10AF20006DA17EA181E895E10E9437C54F8D58A1A2
:10AF300069A17AA18BE795E10E9437C589E20E9459
:10AF4000CC898AE00E94CC899E01215E3F4FAE01F0
:10AF50004D5D5F4FBE01695D7F4FCE018B960E94B4
:10AF600083B109CF0E9427B180E090E0A0EAB0E46D
:10AF70008093B6109093B710A093B810B093B91007
:10AF800019821A821B821C829E012F5F3F4F46EB63
:10AF900050E162EB70E18EEA90E10E94AD4C80914D
:10AFA000170590911805A0911905B0911A05809385
:10AFB000AE109093AF10A093B010B093B1108091E9
:10AFC000130590911405A0911505B0911605809375
:10AFD000B2109093B310A093B410B093B51019822F
:10AFE0001A821B821C829E012F5F3F4F46EB50E16D
:10AFF00062EB70E18EEA90E10E94AD4C6096FFAD8D
:10B000006097F11113C010924504109244040E94FD
:10B01000B67680E090E0E7D109C02FADF42C052D85
:10B02000162DE72C24300CF033CB20CBCC5ADF4F3D
:10B030000FB6F894DEBF0FBECDBFDF91CF911F9149
:10B040000F91FF90EF90DF90CF90BF90AF909F90C7
:10B050008F907F906F905F904F903F902F900895CA
:10B060001F920F920FB60F9211240BB60F922F93CF
:10B070003F938F939F93EF93FF932091120F309103
:10B08000130F8091140F9091150F2817390731F481
:10B09000809131018F7D8093310114C0E091140FB4
:10B0A000F091150FEE56F14F20818091140F909181
:10B0B000150F01968F7799279093150F8093140F92
:10B0C00020933601FF91EF919F918F913F912F91A6
:10B0D0000F900BBE0F900FBE0F901F9018951F92F0
:10B0E0000F920FB60F9211240BB60F922F934F931E
:10B0F0005F938F939F93EF93FF938091300182FD35
:10B100001CC0209136018091960F9091970F40912D
:10B11000980F5091990F01968F77992748175907E3
:10B1200071F0E091960FF091970FEA5EF04F208357
:10B130009093970F8093960F02C080913601FF91F4
:10B14000EF919F918F915F914F912F910F900BBE37
:10B150000F900FBE0F901F901895CF92DF92EF9235
:10B16000FF920F931F93CF93DF936C017A018B01B2
:10B17000C0E0D0E0CE15DF0581F0D8016D918D01E2
:10B18000D601ED91FC910190F081E02DC601199559
:10B19000892B11F02196EECF7E01C701DF91CF916F
:10B1A0001F910F91FF90EF90DF90CF9008950E9434
:10B1B00099ED3FB7F8948091CF069091D006A09179
:10B1C000D106B091D20626B5A89B05C02F3F19F035
:10B1D0000196A11DB11D3FBFBA2FA92F982F882717
:10B1E000820F911DA11DB11DBC01CD0142E0660F72
:10B1F000771F881F991F4A95D1F708952FB7F894A4
:10B200006091CB067091CC068091CD069091CE06D0
:10B210002FBF08951F920F920FB60F9211242F93F4
:10B220003F938F939F93AF93BF938091CB06909161
:10B23000CC06A091CD06B091CE063091CA0623E08F
:10B24000230F2D3720F40196A11DB11D05C026E85E
:10B25000230F0296A11DB11D2093CA068093CB0631
:10B260009093CC06A093CD06B093CE068091CF06E6
:10B270009091D006A091D106B091D2060196A11D61
:10B28000B11D8093CF069093D006A093D106B093C2
:10B29000D206BF91AF919F918F913F912F910F90C7
:10B2A0000FBE0F901F9018951F920F920FB60F921E
:10B2B00011240BB60F922F933F934F935F936F938D
:10B2C0007F938F939F93AF93BF93EF93FF9380915F
:10B2D0002B0590912C05A0912D05B0912E05892B61
:10B2E0008A2B8B2B59F190912A05E0912805F0913A
:10B2F000290580818927808380912B0590912C05D9
:10B30000A0912D05B0912E05181619061A061B06D8
:10B310000CF056C080912B0590912C05A0912D0525
:10B32000B0912E050197A109B10980932B05909347
:10B330002C05A0932D05B0932E0542C080911902D3
:10B34000E7E4F8E1E4919FEF90931902E230C9F04D
:10B3500050F4EE2399F0E13081F590916F009D7FDC
:10B3600090936F002AC0E43019F1E0F0E53029F540
:10B37000909173009D7F909373001FC010926E0098
:10B380001CC0909170009D7F9093700091E090930D
:10B39000B0009091B100987F94609093B1001092AA
:10B3A000B3000BC0909171009D7F9093710005C018
:10B3B000909172009D7F9093720060E00E94DFB5D3
:10B3C000FF91EF91BF91AF919F918F917F916F917D
:10B3D0005F914F913F912F910F900BBE0F900FBE39
:10B3E0000F901F90189590934B0480934A0480E02F
:10B3F0000C9402772F923F924F925F926F927F92BE
:10B400008F929F92AF92BF92CF92DF92EF92FF9274
:10B410000F931F93CF93DF93CDB7DEB7C857D109F2
:10B420000FB6F894DEBF0FBECDBFE0914A07F09192
:10B430004B07EF2B11F00C94BA622896DFAECEAE1C
:10B4400028976E2C79016A015B01FC012081318112
:10B45000428153816C962CAF3DAF4EAF5FAF6C977E
:10B46000209192103091931040919410509195102A
:10B470006C966CAD7DAD8EAD9FAD6C970E94A2E6D3
:10B480000E94BAECE0966CAF7DAF8EAF9FAFE097B5
:10B49000D5018D919D910D90BC91A02DA0968CAF62
:10B4A0009DAFAEAFBFAFA09720919610309197108F
:10B4B0004091981050919910BC01CD010E94A2E6D4
:10B4C0000E94BAECE4966CAF7DAF8EAF9FAFE4976D
:10B4D000D6012D913D914D915C91A4962CAF3DAF3D
:10B4E0004EAF5FAFA49720919A1030919B1040917E
:10B4F0009C1050919D10A4966CAD7DAD8EAD9FAD0E
:10B50000A4970E94A2E60E94BAECE8966CAF7DAFC9
:10B510008EAF9FAFE897D7012D913D914D915C91F2
:10B5200022962CAF3DAF4EAF5FAF229720919E1079
:10B5300030919F104091A0105091A11022966CADB7
:10B540007DAD8EAD9FAD22970E94A2E60E94BAEC1F
:10B5500060966CAF7DAF8EAF9FAF60978091100704
:10B5600083FF1CC060962CAD3DAD4EAD5FAD6097C6
:10B570002093E5093093E6094093E7095093E809E1
:10B5800022968CAD9DADAEADBFAD22978093D5090F
:10B590009093D609A093D709B093D809D801BC914C
:10B5A000B9A7F801F181F9ABD8011296BC91BEABF5
:10B5B000F801F381FAAF8091B3099091B409891B26
:10B5C0008F708F3019F40E9402A1F5CF0091B3095A
:10B5D000E9960FAFE9978091B309082F10E01CA3FB
:10B5E0000BA38091D9099091DA09A091DB09B09160
:10B5F000DC09E0968CAC9DACAEACBFACE097881A91
:10B60000990AAA0ABB0A8091DD099091DE09A091EE
:10B61000DF09B091E009E4962CAC3DAC4EAC5FACD8
:10B62000E497281A390A4A0A5B0A8091E109909145
:10B63000E209A091E309B091E409E8962CAD3DAD93
:10B640004EAD5FADE897281B390B4A0B5B0B2DA362
:10B650003EA34FA358A78091E5099091E609A091D8
:10B66000E709B091E80960960CAD1DAD2EAD3FAD78
:10B670006097081B190B2A0B3B0B0DA71EA72FA7C2
:10B6800038AB012B022B032B09F4BCC080910F07B0
:10B6900081114BC060914C0470914D0480914E0417
:10B6A00090914F040E94CDEB20912502309126020B
:10B6B000621773070CF039C060962CAD3DAD4EADEE
:10B6C0005FAD60972093E5093093E6094093E70961
:10B6D0005093E80922968CAD9DADAEADBFAD2297DB
:10B6E0008093D5099093D609A093D709B093D80930
:10B6F000E4EEFDE184918F010F5F1F4F811103C0C4
:10B70000EBEBF9E104C00E94CC89F801F3CF8491FE
:10B710008F010F5F1F4F882321F00E94CC89F80111
:10B72000F6CF1DA61EA61FA618AA94E0699E80014A
:10B7300011240F5D1D4F6DA57EA58FA598A90E94B0
:10B7400043E6D8012D913D914D915C910E94A2E676
:10B750006B017C0120E030E0A9010E94AFEC87FF83
:10B7600004C0F7FAF094F7F8F09460919E1070918D
:10B770009F108091A0109091A1100E94CDEB9B0191
:10B78000AC01A8ECB0E00E9469EA0E9443E6A70180
:10B7900096010E943DE687FF39C060960CAD1DAD55
:10B7A0002EAD3FAD60970093E5091093E609209315
:10B7B000E7093093E80922962CAD3DAD4EAD5FAD63
:10B7C00022972093D5093093D6094093D7095093F7
:10B7D000D809E4EEFDE184918F010F5F1F4F8111C5
:10B7E00003C0ECE9F9E104C00E94CC89F801F3CF71
:10B7F00084918F010F5F1F4F882321F00E94CC8915
:10B80000F801F6CF1DA61EA61FA618AAD501C401D1
:10B810008827B7FD83959927AA27BB27782E57FE3F
:10B8200003C0382F3260732E8DA19EA1AFA1B8A5A1
:10B83000B7FF03C0972D9460792E0DA51EA52FA5E7
:10B8400038A937FF03C0172D1860712E24E0629EBF
:10B85000800111240F5D1D4F6DA57EA58FA598A9B0
:10B860000E9443E6D8012D913D914D915C910E943B
:10B87000A2E66B017C0120E030E0A9010E94AFEC60
:10B8800087FF04C0C701B601905802C0C701B601C6
:10B8900020E030E040E05FE30E9489EA0E94D2EBC2
:10B8A0006AAB7BAB8CAB9DAB88E60BA11CA1809FE8
:10B8B000F001819FF00D1124E159FE4E1082EA5BE8
:10B8C000FF4F7082B501A401B7FE07C0442755277A
:10B8D000BA01481959096A097B0988E60BA11CA11C
:10B8E000809FF001819FF00D1124E159FE4E458BA0
:10B8F000568B678B708F2C962CAE3DAE4EAE5FAEE6
:10B900002C9757FE0DC088279927DC0182199309CF
:10B91000A409B5092C968CAF9DAFAEAFBFAF2C97E5
:10B9200028E60BA11CA1209FF001219FF00D1124FE
:10B93000E159FE4E2C968CAD9DADAEADBFAD2C97B2
:10B94000818F928FA38FB48F0DA11EA12FA138A537
:10B9500037FF07C030952095109501951F4F2F4F49
:10B960003F4FE8E67E2EABA1BCA17A9EF0017B9E04
:10B97000F00D1124E159FE4E058F168F278F30A34D
:10B980008AA99BA9ACA9BDA981A392A3A3A3B4A38F
:10B9900023964FAF2397752EF62FE72F2C968CAD5D
:10B9A0009DADAEADBFAD2C97481759076A077B0711
:10B9B00078F429969FAD299723969FAF23972A96CF
:10B9C0007FAC2A972B96FFAD2B972C96EFAD2C973B
:10B9D00023968FAD2397972DAF2FBE2F80179107FA
:10B9E000A207B30710F4D901C8010AA91BA92CA901
:10B9F0003DA980179107A207B30710F4D901C80128
:10BA000028E60BA11CA1209FF001219FF00D11241D
:10BA1000E159FE4E85A396A3A7A3B0A70697A1055B
:10BA2000B10508F4A0C5DF01AE59BF4F80914204B3
:10BA3000909143048D939C9361A6452B462B472BF5
:10BA400009F05F9888E60BA11CA1809FF001819FFF
:10BA5000F00D1124E159FE4E818D928DA38DB48D90
:10BA6000892B8A2B8B2B11F08A98479888E60BA19B
:10BA70001CA1809FF001819FF00D1124E159FE4E21
:10BA8000858D968DA78DB0A1892B8A2B8B2B31F0BC
:10BA90008091080181708093060147982AA93BA9EB
:10BAA0004CA95DA9232B242B252B09F465C5809176
:10BAB0001507882319F0815080931507611004C081
:10BAC000129880E28093150760900B0770900C0726
:10BAD00000910D0710910E079301A80169A579A99E
:10BAE0008EA99AAD0E943DE687FF04C069A679AA97
:10BAF0000EAB1AAFC501B4010E9443E620915F115D
:10BB00003091601140916111509162110E94A2E642
:10BB100026966CAF7DAF8EAF9FAF2697698B7A8BE1
:10BB20008B8B9C8BC201B1010E9443E62091631173
:10BB30003091641140916511509166110E94A2E606
:10BB40002B013C016D8B7E8B8F8B988F6DA17EA11D
:10BB50008FA198A50E9443E620916711309168114A
:10BB60004091691150916A110E94A2E64B015C015B
:10BB7000698F7A8F8B8F9C8F20916B1130916C1114
:10BB800040916D1150916E11C701B6010E94A2E65D
:10BB90006B017C016D8F7E8F8F8F98A388E60BA140
:10BBA0001CA1809FF001819FF00D1124E159FE4EF0
:10BBB000258936894789508D2DA33EA34FA358A7C9
:10BBC000263031054105510508F4DFC42896AEAD95
:10BBD000BFAD2897CD90DD90ED90FC9020E030E057
:10BBE000A901C701B6010E943DE68111EDC4269668
:10BBF0002CAD3DAD4EAD5FAD2697CA01B9010E9497
:10BC0000A2E66B017C01A3019201C301B2010E9473
:10BC1000A2E69B01AC01C701B6010E9489EA6B0153
:10BC20007C01A5019401C501B4010E94A2E69B011B
:10BC3000AC01C701B6010E9489EA0E94F4EC28E633
:10BC40000BA11CA1209FF001219FF00D1124E159AF
:10BC5000FE4E658776878787908B88E60BA11CA1AF
:10BC6000809FF001819FF00D1124E159FE4E458423
:10BC7000568467847088A301920160E070E080E8D8
:10BC80009FE30E9465EB64966CAF7DAF8EAF9FAF74
:10BC9000649729A539A94EA95AAD0E94A2E64B0185
:10BCA0005C018091B3099091B109891B8F7027962F
:10BCB0008FAF2797A501940160E074E284E799E4CF
:10BCC0000E9465EB0E94BAEC6B017C0127968FAD58
:10BCD00027978250863008F486C4A5019401C301D9
:10BCE000B2010E94A2E69B01AC010E94A2E6689606
:10BCF0006CAF7DAF8EAF9FAF689788E6ABA1BCA15C
:10BD00008A9F80018B9F100D112401591E4E689649
:10BD10002CAD3DAD4EAD5FAD6897D80111962D931A
:10BD20003D934D935C93149795962D913D914D9134
:10BD30005C9198972EAB3FAB48AF59AFCA01B901A0
:10BD40000E9441E66AAF7BAF8CAF9DAF9B01AC0117
:10BD5000C501B4010E94A2E60E944FEB0E94D2EB03
:10BD6000A8966CAF7DAF8EAF9FAFA897F801EE5A43
:10BD7000FF4F60837183828393838E010F5E1F4F19
:10BD80002A961FAF0EAF2A970051110924961FAFB4
:10BD90000EAF249703EF16E0AC961FAF0EAFAC9733
:10BDA0008E010F5D1F4F1AA309A324960EAD1FAD80
:10BDB0002497AA961FAF0EAFAA97312C212C10E81A
:10BDC00019A70FE309AB2A96AEADBFAD2A972D9107
:10BDD0003D914D915D912A96BFAFAEAF2A97C501B7
:10BDE000B4010E94A2E66B017C01AA96EEADFFAD04
:10BDF000AA976193719381939193AA96FFAFEEAF47
:10BE0000AA9720E030E0A9010E94AFEC87FF04C0B0
:10BE1000F7FAF094F7F8F094AC96AEADBFADAC97EE
:10BE20004D905D906D907D90AC96BFAFAEAFAC97EE
:10BE3000A7019601C301B2010E943DE687FD0DC432
:10BE400009A11AA12A962EAD3FAD2A970217130712
:10BE500009F0B9CF20E030E040E85FE3632D722DB8
:10BE600089A599A90E943DE687FF58C07E0131E16E
:10BE7000E30EF11C24960EAD1FAD2497232D322D19
:10BE800049A559A9D8016D917D918D919C910E94F0
:10BE9000A2E6F80161937193819391938F01EE165D
:10BEA000FF0661F728E60BA11CA1209FC001219F7E
:10BEB000900D11249C0121593E4E790189010E5AA1
:10BEC0001F4FA8966CAD7DAD8EAD9FADA8970E941B
:10BED00041E6232D322D49A559A90E94A2E60E94D0
:10BEE000D2EBD8016D937D938D939C931397232D63
:10BEF000322D49A559A9632D722D89A599A90E94B2
:10BF0000A2E668962CAD3DAD4EAD5FAD68970E9440
:10BF1000A2E6F70161837283838394832AAD3BADEC
:10BF20004CAD5DAD64966CAD7DAD8EAD9FAD64974F
:10BF30000E94A2E669A77AA78BA79CA70DA11EA1C4
:10BF40002FA138A5012B022B032B09F09EC388E6F5
:10BF50002BA13CA1829F8001839F100D11240159C8
:10BF60001E4EF801818D928DA38DB48D892B8A2B65
:10BF70008B2B09F08AC3858D968DA78DB0A1892B57
:10BF80008A2B8B2B09F081C32091EF063091F006AC
:10BF90004091F1065091F20669A57AA58BA59CA562
:10BFA0000E94A2E60E944FEB0E94D2EB2B013C01C3
:10BFB000F801E95BFF4F108288E62BA13CA1829F2C
:10BFC0008001839F100D112401591E4EF801E25A81
:10BFD000FF4F4082518262827382C301B2010E948C
:10BFE00041E629A53AA54BA55CA50E9465EB6AAF81
:10BFF0007BAF8CAF9DAFD80151966D937D938D93A0
:10C000009C935497F801E95BFF4F8081882381F16D
:10C010007801B8E4EB0EF11C37962091E3063091DD
:10C02000E4064091E5065091E606608171818281C7
:10C0300093810E94A2E62AAD3BAD4CAD5DAD0E945E
:10C04000A2E620919E1030919F104091A010509137
:10C05000A1100E94A2E69B01AC0160E074E284EFB3
:10C0600099E40E9465EB0E94D2EBF7017183608333
:10C0700088E60BA11CA1809FF001819FF00D112487
:10C08000E159FE4E21813281438154812C962CAF9F
:10C090003DAF4EAF5FAF2C97CA01B9010E94F4ECDF
:10C0A000362E272E8C0143ED56E062965FAF4EAFE1
:10C0B00062973E0151E1650E711C83ED96E09FABE6
:10C0C0008EAB24964EAC5FAC24973DA62DA209A75B
:10C0D00019AB1AAAD201CD90DD90ED90FD902D0103
:10C0E00020E030E0A901C701B6010E94AFEC87FF54
:10C0F00004C0F7FAF094F7F8F094EEA9FFA9819044
:10C100009190A190B190FFABEEABA7019601C50154
:10C11000B4010E943DE687FDD8C564147504D1F6CC
:10C1200027965FAD2797552309F448C6C090B509F7
:10C13000D090B609E090B709F090B8092DEB37E33D
:10C1400046E855E3C701B6010E943DE687FD36C6C5
:10C15000C701B6010E94F4EC6B017C019B01AC01AC
:10C16000632D722DC8010E943DE687FD03C03C2C63
:10C170002D2C87019601A701632D722DC8010E9405
:10C1800065EB68966CAF7DAF8EAF9FAF689789EB1C
:10C1900099E028969FAF8EAF289720E030E040E8E6
:10C1A0005FE32AAB3BAB4CAB5DAB1EAA2896AEADB2
:10C1B000BFAD28972D913D914D915D912896BFAFD0
:10C1C000AEAF289768966CAD7DAD8EAD9FAD68978C
:10C1D0000E94A2E64B015C012496EEADFFAD2497D0
:10C1E000C190D190E190F1902496FFAFEEAF2497EB
:10C1F000FEA9FF2391F02AA93BA94CA95DA90E94A1
:10C20000A2E64B015C012AA93BA94CA95DA9C70183
:10C21000B6010E94A2E66B017C01A7019601C5014F
:10C22000B4010E94AFEC20E030E0A90118160CF038
:10C2300092C5C701B6010E94AFEC18160CF486C572
:10C2400020E030E0A901C501B4010E943DE687FD70
:10C250007DC52601370177FA709477F87094A301B1
:10C260009201C501B4010E94AFEC181614F4240128
:10C2700035016296AEADBFAD6297CD90DD90ED9089
:10C28000FD906296BFAFAEAF6297A3019201C70166
:10C29000B6010E943DE687FF15C0A3019201C701C8
:10C2A000B6010E9465EB9B01AC016AA97BA98CA930
:10C2B0009DA90E94A2E66AAB7BAB8CAB9DABBEA9ED
:10C2C000BF5FBEABE9ECF9E028962EAD3FAD2897F5
:10C2D000E217F30709F06ACF3EA9332361F02AA9D8
:10C2E0003BA94CA95DA9632D722DC8010E94A2E64D
:10C2F000362E272E8C0124EA30E74DE75FE3632DCD
:10C30000722DC8010E94A2E66B017C0120911107E9
:10C310003091120740911307509114070E943DE697
:10C3200087FD42C58DA59DA1A9A5B9A98093110737
:10C3300090931207A0931307B093140728E64BA11C
:10C340005CA1249FC001259F900D1124DC01A159FF
:10C35000BE4E7D01232D322DA801632D722DC80103
:10C360000E94A2E6F70161877287838794876AAD8E
:10C370007BAD8CAD9DAD90589B01AC010E9489EACC
:10C38000D7011D962D913D914D915C9150970E9442
:10C39000A2E69B01AC016BE077ED83E29BE30E9498
:10C3A00088EA9B01AC018BE097EDA3E2BBE3F701C8
:10C3B00085839683A783B08710812C966CAD7DAD65
:10C3C0008EAD9FAD2C970E943DE618160CF4FBC471
:10C3D00083E0182B88E62BA13CA1829FF001839F6C
:10C3E000F00D1124E159FE4E108380E1FE013196DB
:10C3F000A9EBB9E001900D928A95E1F72C968CADEE
:10C400009DADAEADBFAD2C978093B5099093B609A5
:10C41000A093B709B093B809E0960CAD1DAD2EAD51
:10C420003FADE0970093D9091093DA092093DB0917
:10C430003093DC09E4962CAD3DAD4EAD5FADE49795
:10C440002093DD093093DE094093DF095093E00922
:10C45000E8968CAD9DADAEADBFADE8978093E10998
:10C460009093E209A093E309B093E40960960CADC0
:10C470001DAD2EAD3FAD60970093E5091093E60921
:10C480002093E7093093E8096C962CAD3DAD4EAD95
:10C490005FAD6C972093C9093093CA094093CB09CB
:10C4A0005093CC09A0968CAD9DADAEADBFADA0971D
:10C4B0008093CD099093CE09A093CF09B093D00972
:10C4C000A4960CAD1DAD2EAD3FADA4970093D10940
:10C4D0001093D2092093D3093093D40922962CAD1E
:10C4E0003DAD4EAD5FAD22972093D5093093D6096F
:10C4F0004093D7095093D8099091B3098091B4091A
:10C50000981303C084E68093B009E9968FADE9974C
:10C510008F5F8F708093B3098091B3099091B209B6
:10C5200081508F70891351C41091B4091BA30091DD
:10C53000B3090DA728E61BA10DA51013D1C4812CAA
:10C54000912CA12CB12C1DA219A619AA1EAE212C2A
:10C55000312C00E010E02DA53BA12313CEC4211403
:10C56000310409F07FC580916F00826080936F0075
:10C5700081E0ECC680E0EAC660900707709008078B
:10C580000091090710910A07A7CA818D928DA38D8A
:10C59000B48D0697A105B10508F018CB858D968D51
:10C5A000A78DB0A10697A105B10508F00FCB20E03B
:10C5B00030E0A901C701B6010E94AFEC87FF04C0BB
:10C5C000F7FAF094F7F8F09488E60BA11CA1809F8D
:10C5D000F001819FF00D1124E159FE4EC586D686EB
:10C5E000E786F08A3ACB8091030790910407A091E7
:10C5F0000507B0910607C816D906EA06FB0608F03B
:10C600006CCB8C199D09AE09BF09BC01CD01660F29
:10C61000771F881F991F27964FAD2797042F10E08B
:10C6200020E030E0A90198010E942BEACA01B9017B
:10C630000E9441E60E94BAEC6C0D7D1D8E1D9F1D6F
:10C640000E9441E69B01AC0160E074E284E799E45A
:10C650000E9465EB4B015C0140CBA7019601C30131
:10C66000B2010E9465EB7B018C019B01AC01632D43
:10C67000722D89A599A90E94AFEC18160CF0E0CB99
:10C680003E2C2F2C09A719ABDBCB0AA91BA92CA97F
:10C690003DA9012B022B032B49F02091EB06309191
:10C6A000EC064091ED065091EE0608C02091E70699
:10C6B0003091E8064091E9065091EA0669A57AA50D
:10C6C0008BA59CA50E94A2E60E944FEB0E94D2EB94
:10C6D0002B013C012AA93BA94CA95DA9232B242BA2
:10C6E000252BC9F020E030E0A9016091E3067091AC
:10C6F000E4068091E5069091E6060E943DE68823D7
:10C7000051F081E00DA51EA52FA538A91016110620
:10C71000120613060CF080E098E62BA13CA1929F34
:10C720008001939F100D112401591E4E180137E40A
:10C73000230E311CD1018C93882309F4B3C02091BE
:10C74000C9093091CA094091CB095091CC096C9626
:10C750006CAD7DAD8EAD9FAD6C970E9488EA6DA7E4
:10C760007EA78FA798AB2091CD093091CE0940913B
:10C77000CF095091D009A0966CAD7DAD8EAD9FAD27
:10C78000A0970E9488EA4B015C012091D109309169
:10C79000D2094091D3095091D409A4966CAD7DADD6
:10C7A0008EAD9FADA4970E9488EA6B017C012DA5F8
:10C7B0003EA54FA558A9CA01B9010E94A2E66DA7DE
:10C7C0007EA78FA798ABA5019401C501B4010E9473
:10C7D000A2E69B01AC016DA57EA58FA598A90E943C
:10C7E00089EA4B015C01A7019601C701B6010E94CD
:10C7F000A2E69B01AC01C501B4010E9489EA0E9436
:10C80000F4EC6B017C012091D5093091D60940915F
:10C81000D7095091D80922966CAD7DAD8EAD9FADF4
:10C8200022970E9488EAA70196010E9465EB6B019E
:10C830007C01F801E25BFF4F608371838283938305
:10C8400020E030E040E450E40E94AFEC18161CF405
:10C85000F101108227C02091E3063091E406409157
:10C86000E5065091E606C701B6010E94A2E69B01CB
:10C87000AC016091DF067091E0068091E106909135
:10C88000E2060E9465EB29A53AA54BA55CA50E948E
:10C89000A2E60E94D2EB641575058605970510F493
:10C8A0002B013C0180913B1190913C11A0913D11D5
:10C8B000B0913E110EA91FA928AD39AD801791077F
:10C8C000A207B30708F4DFC02DA13EA14FA158A5D0
:10C8D000232B242B252B41F160913F1170914011A6
:10C8E0008091411190914211641575058605970557
:10C8F000D8F42EA93FA948AD59AD0E941CEA6B019E
:10C900007C012DA13EA14FA158A5C301B2010E94F7
:10C910001CEAC616D706E806F90630F4C701B601C8
:10C920000E942BEA29013A0188E60BA11CA1809FF5
:10C93000F001819FF00D1124E159FE4EC18CD28C83
:10C94000E38CF48CC114D104E104F10431F1609161
:10C9500043117091441180914511909146116415D5
:10C96000750586059705C8F42EA93FA948AD59ADB0
:10C970000E941CEA4B015C01A7019601C301B201B0
:10C980000E941CEA86169706A806B90630F4C5016F
:10C99000B4010E942BEA29013A0188E60BA11CA1EF
:10C9A000809FF001819FF00D1124E159FE4EC58C4E
:10C9B000D68CE78CF0A0C114D104E104F10431F16C
:10C9C00060914711709148118091491190914A11DD
:10C9D0006415750586059705C8F42EA93FA948ADCD
:10C9E00059AD0E941CEA4B015C01A7019601C301ED
:10C9F000B2010E941CEA86169706A806B90630F412
:10CA0000C501B4010E942BEA29013A0188E60BA175
:10CA10001CA1809FF001819FF00D1124E159FE4E71
:10CA2000C1A0D2A0E3A0F4A0C114D104E104F10498
:10CA300009F4C2CA60914B1170914C1180914D1153
:10CA400090914E11641575058605970508F0B4CAD6
:10CA50002EA93FA948AD59AD0E941CEA4B015C01CB
:10CA6000A7019601C301B2010E941CEA861697062F
:10CA7000A806B90608F0A0CAC501B4010E942BEAB5
:10CA800029013A0199CA2DA13EA14FA158A5232BF6
:10CA9000242B252BC9F160913F1170914011809199
:10CAA000411190914211641575058605970560F551
:10CAB0000E9441E62AAD3BAD4CAD5DAD0E94A2E6C1
:10CAC0006B017C016DA17EA18FA198A50E9441E61A
:10CAD0004B015C01C301B2010E9441E6A501940132
:10CAE0000E94A2E69B01AC01C701B6010E943DE68F
:10CAF00087FF0AC0A5019401C701B6010E9465EB3A
:10CB00000E94D2EB2B013C0188E60BA11CA1809F67
:10CB1000F001819FF00D1124E159FE4E818C928C21
:10CB2000A38CB48C81149104A104B104B9F1609177
:10CB300043117091441180914511909146116415F3
:10CB400075058605970550F50E9441E62AAD3BAD77
:10CB50004CAD5DAD0E94A2E66B017C01C501B40144
:10CB60000E9441E64B015C01C301B2010E9441E613
:10CB7000A50194010E94A2E69B01AC01C701B60188
:10CB80000E943DE687FF0AC0A5019401C701B601D6
:10CB90000E9465EB0E94D2EB2B013C0188E60BA1C1
:10CBA0001CA1809FF001819FF00D1124E159FE4EE0
:10CBB000858C968CA78CB0A081149104A104B1043B
:10CBC000B9F160914711709148118091491190918C
:10CBD0004A11641575058605970550F50E9441E6D2
:10CBE0002AAD3BAD4CAD5DAD0E94A2E66B017C0170
:10CBF000C501B4010E9441E64B015C01C301B201D1
:10CC00000E9441E6A50194010E94A2E69B01AC01AD
:10CC1000C701B6010E943DE687FF0AC0A501940145
:10CC2000C701B6010E9465EB0E94D2EB2B013C01CB
:10CC300088E60BA11CA1809FF001819FF00D1124BB
:10CC4000E159FE4EC1A0D2A0E3A0F4A0C114D104CA
:10CC5000E104F10409F4B0C960914B1170914C11D9
:10CC600080914D1190914E116415750586059705BB
:10CC700008F0A2C90E9441E62AAD3BAD4CAD5DADC6
:10CC80000E94A2E64B015C01C701B6010E9441E689
:10CC90006B017C01C301B2010E9441E6A70196012C
:10CCA0000E94A2E69B01AC01C501B4010E943DE6D1
:10CCB00087FF82C9A7019601C501B4010E9465EBF7
:10CCC0000E94D2EB2B013C0177C9FAA9FF2331F175
:10CCD000A5019401632D722DC8010E94A2E64B01AB
:10CCE0005C012DA53DA149A559A9C701B6010E9426
:10CCF000A2E69B01AC01C501B4010E943DE687FF9D
:10CD000022C0A7019601C501B4010E9465EB6DA781
:10CD10007DA389A799AB21E02AABFFC9A7019601A2
:10CD2000C501B4010E9465EB9B01AC016DA57DA11D
:10CD300089A599A90E94A2E66DA77DA389A799ABB1
:10CD400031E03AABEAC941E04AABE7C9A701960135
:10CD5000C501B40113C0C701B6010E943DE687FDBD
:10CD600009C020E030E0A901C501B4010E94AFEC88
:10CD700018164CF4A5019401C701B6010E9488EA77
:10CD80002B013C0176CA2401350177FA709477F8BB
:10CD90007094A3019201C701B6010E943DE687FD90
:10CDA00068CA2601370165CA2DA53DA149A559A923
:10CDB000C701B6010E943DE687FFB4CA3DA42DA07D
:10CDC00009A519A9AFCA81E004CBF090B3098FEF90
:10CDD0008F0D8F708BA3B090B2098091B309B816F4
:10CDE00009F454C0C12CD12C0BA10B1509F44EC071
:10CDF000602E712C28E6269D8001279D100D1124A0
:10CE000001591E4ED8018C9183FD2BC00EAF1AAB79
:10CE10000115110541F11996BC91BDA7F801F285E4
:10CE2000FDA3D8011B96BC91B9A7F801F485F9AB15
:10CE3000D80115962D903D904D905C901897A201C9
:10CE400091016DA57DA189A59F2F0E943DE68111CD
:10CE500086C1C114D10439F0F601808180FD7FC103
:10CE600002C0CEAEDAAA8BA181508F708BA38091C5
:10CE7000B2098B1103C0CEACDAA8B6CF0BA10B154B
:10CE800029F081E08B0D8F70B82EF1CF1091B2098F
:10CE90001BA3C12CD12C8091B3090BA1801709F4DD
:10CEA00043CB802E912C28E6289D8001299D100DD2
:10CEB000112401591E4ED8018C9183FD0AC05801DE
:10CEC000C114D10439F0C6010E94477F811102C00C
:10CED000C5C156018BA18F5F8F708BA36501DBCF1E
:10CEE000802F81508F70289FF0011124E159FE4E50
:10CEF000908193FF24CB8DA71ECB48E6439FC001B2
:10CF00001124DC01A159BE4E1D018C9183FD19C075
:10CF100015966D917D918D919C9118970E94F4ECDE
:10CF2000F62EE72ED82EC92E0115110509F48CC056
:10CF3000F801808180FD0AC0D1018C9180FD06C07E
:10CF400083C0FDA0E9A4D9A8CEAC83C0F80180813C
:10CF500081608083C8010E94477F811171C0F80100
:10CF600061817281838194810E94F4EC2B013C01E8
:10CF70009B01AC0160E070E080E89FE30E9465EBFC
:10CF80004B015C019B01AC016F2D7E2D8D2D9C2DE5
:10CF90000E94A2E669837A838B839C832DA139A5A5
:10CFA00049A95EADC501B4010E94A2E6698B7A8BE6
:10CFB0008B8B9C8BAE014F5F5F4FBE016F5E7F4FCF
:10CFC000C8010E944DB8F801E95BFF4F80818823BA
:10CFD000B9F12091E3063091E4064091E5065091C5
:10CFE000E606379660817181828193810E94A2E674
:10CFF00020919E1030919F104091A0105091A1104F
:10D000000E94A2E64B015C019B01AC01C301B2018D
:10D010000E94A2E60E94D2EBF801E65BFF4F71830B
:10D020006083A50194016F2D7E2D8D2D9C2D0E9476
:10D03000A2E60E94D2EBF801E45BFF4F71836083AC
:10D04000D8018C918E7F8C938F2C9E2CAD2CBC2C78
:10D0500081018BA18F5F8F708BA3FDA2E9A6D9AA56
:10D06000CEAE79CAF101808181608083C8010E94BF
:10D07000477F81116FC0D10111966D917D918D9186
:10D080009C9114970E94F4EC6B017C019B01AC0114
:10D0900060E070E080E89FE30E9465EB2B013C01BB
:10D0A0002DEC3CEC4CE45DE30E94A2E669837A83BC
:10D0B0008B839C839401A501C301B2010E94A2E667
:10D0C000698B7A8B8B8B9C8BAE014F5F5F4FBE0160
:10D0D0006F5E7F4FC1010E944DB8F101E95BFF4FC8
:10D0E00080818823B9F12091E3063091E4064091D4
:10D0F000E5065091E60637966081718182819381C1
:10D100000E94A2E620919E1030919F104091A010A5
:10D110005091A1100E94A2E64B015C019B01AC0161
:10D12000C701B6010E94A2E60E94D2EBF101E65BC4
:10D13000FF4F718360832DEC3CEC4CE45DE3C50153
:10D14000B4010E94A2E60E94D2EBF101E45BFF4F22
:10D1500071836083F10180818E7F808304CA28E619
:10D16000269DF001279DF00D1124E159FE4E80818E
:10D1700081FD43C0C114D10441F0D6011596CD9074
:10D18000DD90ED90FC90189708C08BE0C82E87EDDD
:10D19000D82E83E2E82E8BE3F82EB8E6B69DF00198
:10D1A000B79DF00D1124E159FE4E81899289A38922
:10D1B000B489BC01CD0190589B01AC010E9489EA61
:10D1C000F80125853685478550890E94A2E69B0196
:10D1D000AC01C701B6010E9488EAE62E872E982E80
:10D1E000A92E262F372F482F592F6DA57DA189A550
:10D1F00099A90E943DE687FF04C0EDA48DA099A4E3
:10D20000A9A82E2D382D492D5A2DC201B1010E94F9
:10D210003DE6882309F427CEF8E6F69DC001F79D88
:10D22000900D11249C0121593E4E6901D9018C9128
:10D2300081608C93C8010E94477F882329F0F60102
:10D2400080818E7F80830FCE8E2D982DA92DBA2DB3
:10D25000F60185839683A783B08705CED6018C918E
:10D2600081FD52C0D60115962D913D914D915C9155
:10D2700018972DA73EA74FA758AB1501B5E02B0E69
:10D28000311CF8014580568067807084A3019201AB
:10D290006DA57EA58FA598A90E943DE687FF34C0A5
:10D2A000F60181899289A389B489BC01CD01905886
:10D2B0009B01AC010E9489EAD6011D962D913D91FA
:10D2C0004D915C9150970E94A2E69B01AC016DA527
:10D2D0007EA58FA598A90E9488EA6B017C019B011D
:10D2E000AC01C301B2010E94AFEC18166CF4D80176
:10D2F0008C9181608C93C5010E94477F8823E1F067
:10D30000F80180818E7F808318E6189DF001199DB9
:10D31000F00D1124E159FE4E218532854385548557
:10D3200065817681878190850E943DE68111D2CD0D
:10D330000BA10093B209CECDD101CD92DD92ED9239
:10D34000FC9213970BA10093B209DECFC858DF4FB0
:10D350000FB6F894DEBF0FBECDBFDF91CF911F9106
:10D360000F91FF90EF90DF90CF90BF90AF909F9084
:10D370008F907F906F905F904F903F902F90089587
:10D380008091B3099091B409891B8F708F3019F483
:10D390000E9402A1F5CF8091B3098F5F8F70E09159
:10D3A000B30998E69E9FF0011124E159FE4EDF017A
:10D3B0001D929A95E9F798E090834091D909509190
:10D3C000DA096091DB097091DC09458B568B678B1C
:10D3D000708F4091DD095091DE096091DF097091F5
:10D3E000E009418F528F638F748F4091E109509112
:10D3F000E2096091E3097091E409458F568F678FC8
:10D4000070A34091E5095091E6096091E709709198
:10D41000E80941A352A363A374A32091B309909197
:10D42000B409291303C094E69093B0098093B3091B
:10D4300080916F00826080936F0008959091B3098E
:10D440008091B409981306C080914A0790914B07C8
:10D45000892B19F00E9402A1F1CF0895CF93DF9399
:10D460008B3D9240B1F0EFECFDE18491EF0121960C
:10D47000882321F00E94CC89FE01F7CFE6EDF9E187
:10D480008491EF012196882331F00E94CC89FE011E
:10D49000F7CF80E001C081E0DF91CF9108952F9216
:10D4A0003F924F925F926F927F928F929F92AF9234
:10D4B000BF92CF92DF92EF92FF920F931F93CF9381
:10D4C000DF93CDB7DEB7C757D1090FB6F894DEBFEB
:10D4D0000FBECDBF2DB63EB6A7961FAE1EAEA79708
:10D4E00084E690E0A9969FAF8EAFA99701E09E01D8
:10D4F0002B593F4F44E050E0BE01655A7F4FCE01AB
:10D5000089599F4F0E94F8CF9E012B593F4F42E00F
:10D5100050E0BE0167597F4FCE0189599F4F0E944D
:10D52000F8CF43E050E0BE01655A7F4F8FED92E0A7
:10D530000E94F4ED892B09F43FC06F968FAD6F9771
:10D54000882339F08FE36C968FAF6C976D961FAE82
:10D550006D97E4EEFDE184917F012FEFE21AF20A6C
:10D56000811103C0E9E9FAE104C00E94CC89F70106
:10D57000F2CF84917F013FEFE31AF30A882321F071
:10D580000E94CC89F701F5CFBE01655A7F4F80E933
:10D590009AE10E946DC5E2E8FAE184917F019FEF74
:10D5A000E91AF90A882321F00E94CC89F701F5CF06
:10D5B00081E08093160754C5EDB7FEB7E696FFAF3E
:10D5C000EEAFE6976B961CAE1DAE1EAE1FAE6B9710
:10D5D000A7961FAE1EAEA79701E09E012B593F4FA5
:10D5E00041E050E0BE0160597F4FCE0189599F4F05
:10D5F0000E94F8CF80E1EBE5F2E0DE019196019028
:10D600000D928A95E1F780E1EBE6F2E0DE015196BA
:10D6100001900D928A95E1F780E1EBE7F2E0DE01FF
:10D62000119601900D928A95E1F7E1964FADE19741
:10D6300050E04D5F5F4F440F551F440F551F2DB7EE
:10D640003EB7241B350B0FB6F8943EBF0FBE2DBF5F
:10D650008DB79EB701967C0100E09E012B593F4F8C
:10D66000BC01CE0189599F4F0E94F8CF9E012B59D2
:10D670003F4F44E050E063E077E0CE0189599F4F8F
:10D680000E94F8CFE1968FACE197912C93E0890E40
:10D69000911C880C991C880C991CEDB7FEB7E819F1
:10D6A000F9090FB6F894FEBF0FBEEDBF2DB73EB718
:10D6B0002F5F3F4F69018DB79EB7881999090FB643
:10D6C000F8949EBF0FBE8DBFEDB7FEB731965F01D8
:10D6D0009E012B593F4FA401B601CE0189599F4F9E
:10D6E0000E94F8CF9E012B593F4FA401B501CE01F6
:10D6F00089599F4F0E94F8CF10911707112309F401
:10D70000A7C000E09E012B593F4F44E050E06BEE74
:10D7100076E0CE0189599F4F0E94F8CF9E012B5988
:10D720003F4F44E050E06FEE76E0CE0189599F4FC5
:10D730000E94F8CF9E012B593F4F44E050E067EE26
:10D7400076E0CE0189599F4F0E94F8CF9E012B5958
:10D750003F4F44E050E06BE077E0CE0189599F4FA6
:10D760000E94F8CF9E012B593F4F44E050E067E004
:10D7700077E0CE0189599F4F0E94F8CF9E012B5927
:10D780003F4F40E150E063ED76E0CE0189599F4F75
:10D790000E94F8CF9E012B593F4F44E050E0BE015C
:10D7A000695A7F4FCE0189599F4F0E94F8CF9E0141
:10D7B0002B593F4F4CE050E068E375E0CE018959AA
:10D7C0009F4F0E94F8CF9E012B593F4F44E050E0FD
:10D7D00063E371E1CE0189599F4F0E94F8CF9E010A
:10D7E0002B593F4F44E050E0BE01695A7F4FCE01B4
:10D7F00089599F4F0E94F8CF01E09E012B593F4F5E
:10D8000041E050E0BE0161597F4FCE0189599F4FE1
:10D810000E94F8CF9E012B593F4F41E050E0BE01DE
:10D8200062597F4FCE0189599F4F0E94F8CF111145
:10D830008AC06B968CAD9DADAEADBFAD6B9780933E
:10D84000C2109093C310A093C410B093C5107BC0B6
:10D85000E1968FADE19790E0029623EF36E0E496F3
:10D860003FAF2EAFE497B501DE011196E2E98E2EAF
:10D87000E0E19E2EAE014F5E5F4FFFE4AF2EF1E17F
:10D88000BF2EE896FFAEEEAEE8977E0131E2E30EE2
:10D89000F11C20E030E0821793072CF0E896EEAD03
:10D8A000FFADE89701C0F70140805180628073802E
:10D8B000F50141925192619271925F018217930733
:10D8C00014F0F60101C0FA0140805180628073803B
:10D8D000F40141925192619271924F018217930724
:10D8E00034F0FB01408051806280738005C04D9010
:10D8F0005D906D907C901397E496EEADFFADE4974C
:10D900004192519261927192E496FFAFEEAFE4972B
:10D910002F5F3F4F6C5F7F4F1496F4E0CF0ED11C0A
:10D920004C5F5F4FE896EEADFFADE8973496E89612
:10D93000FFAFEEAFE897F4E0EF0EF11C24303105B5
:10D9400009F0A9CFDECEE0968FADE097853099F44F
:10D95000AF968FADAF97853071F400E09E012B59E3
:10D960003F4F44E650E066EC70E1CE0189599F4F8D
:10D970000E94F8CF24C0111102C00E94B5BDE096EC
:10D980008FADE097AF96CFACAF978C9D600111241F
:10D99000E12CF12CEC14FD0491F000E09E012B59D8
:10D9A0003F4F44E050E0BE01695A7F4FCE01895994
:10D9B0009F4F0E94F8CF2FEFE21AF20AEBCF00E060
:10D9C0009E012B593F4F44E050E0BE016D5A7F4FFE
:10D9D000CE0189599F4F0E94F8CF1AE0115079F07B
:10D9E00000E09E012B593F4F44E050E0BE01695AD0
:10D9F0007F4FCE0189599F4F0E94F8CFEFCF01E0B2
:10DA00009E012B593F4F41E050E0BE0163597F4FCB
:10DA1000CE0189599F4F0E94F8CF9E012B593F4F4D
:10DA200041E050E0BE0164597F4FCE0189599F4FBC
:10DA30000E94F8CF00E09E012B593F4F44E050E098
:10DA4000BE01635C7F4FCE0189599F4F0E94F8CF82
:10DA50009E012B593F4F44E050E0BE016F5C7F4F69
:10DA6000CE0189599F4F0E94F8CFAE968FADAE97E9
:10DA7000AD96CFACAD978C9D60011124E12CF12CBB
:10DA800000E09E012B593F4FCE14DF0471F044E0BB
:10DA900050E0BE01695A7F4FCE0189599F4F0E94C5
:10DAA000F8CF3FEFE31AF30AEBCF41E050E0BE01BD
:10DAB0006F587F4FCE0189599F4F0E94F8CF9E012A
:10DAC0002B593F4F41E050E0BE0165597F4FCE01D9
:10DAD00089599F4F0E94F8CF9E012B593F4F44E038
:10DAE00050E0BE01695A7F4FCE0189599F4F0E9475
:10DAF000F8CF9E012B593F4F44E050E0BE01695AD8
:10DB00007F4FCE0189599F4F0E94F8CF9E012B591C
:10DB10003F4F44E050E067E371E1CE0189599F4FE8
:10DB20000E94F8CF9E012B593F4F44E050E0BE01C8
:10DB3000615B7F4FCE0189599F4F0E94F8CF9E01B4
:10DB40002B593F4F44E050E0BE01655B7F4FCE0153
:10DB500089599F4F0E94F8CF9E012B593F4F44E0B7
:10DB600050E0BE01695B7F4FCE0189599F4F0E94F3
:10DB7000F8CF10E000E09E012B593F4F44E050E009
:10DB8000BE01695A7F4FCE0189599F4F0E94F8CF3D
:10DB9000111110C06B96CCACDDACEEACFFAC6B974A
:10DBA00020E030E84BE355E4C701B6010E943DE6B2
:10DBB000811103C054E0F52E33C080911707811105
:10DBC00008C0C0923C07D0923D07E0923E07F09219
:10DBD0003F0700E09E012B593F4F44E050E068E3CF
:10DBE00077E0CE0189599F4F0E94F8CF9E012B59B3
:10DBF0003F4F44E050E060E477E0CE0189599F4F09
:10DC00000E94F8CF9E012B593F4F44E050E0BE01E7
:10DC1000695A7F4FCE0189599F4F0E94F8CF12C099
:10DC2000FA94FF2079F000E09E012B593F4F44E029
:10DC300050E0BE01695A7F4FCE0189599F4F0E9423
:10DC4000F8CFEECF1F5F153009F094CF00E09E01B2
:10DC50002B593F4F42E050E0BE016D597F4FCE013E
:10DC600089599F4F0E94F8CF9E012B593F4F44E0A6
:10DC700050E0BE01695A7F4FCE0189599F4F0E94E3
:10DC8000F8CF6B96CCACDDACEEACFFAC6B9720E084
:10DC900030E84BE355E4C701B6010E943DE6882316
:10DCA00029F180911707811108C0C0923407D092E2
:10DCB0003507E0923607F092370700E09E012B59B6
:10DCC0003F4F44E050E060E377E0CE0189599F4F39
:10DCD0000E94F8CF9E012B593F4F44E050E06CE288
:10DCE00077E0CE0189599F4F0E94F8CF00E09E0156
:10DCF0002B593F4F42E050E0BE016F597F4FCE019C
:10DD000089599F4F0E94F8CF9E012B593F4F41E008
:10DD100050E0BE016F587F4FCE0189599F4F0E943E
:10DD2000F8CF19E0115000E09E012B593F4F11230D
:10DD300059F044E050E0BE01695A7F4FCE01895945
:10DD40009F4F0E94F8CFEECF41E050E06AE271E1D0
:10DD5000CE0189599F4F0E94F8CFF12C00E09E011F
:10DD60002B593F4F44E050E0BE01695A7F4FCE012E
:10DD700089599F4F0E94F8CF10911707111110C0B9
:10DD8000F1100EC06B968CAD9DADAEADBFAD6B9777
:10DD900080932F1190933011A0933111B0933211D1
:10DDA000F39485E0F812DACF111102C00E94B5C4D5
:10DDB0004CE0F42EFA94F11003C03CE0F32E0FC0B7
:10DDC00000E09E012B593F4F42E050E0BE01615AF6
:10DDD0007F4FCE0189599F4F0E94F8CFEBCFFA9425
:10DDE00000E09E012B593F4FFF2059F044E050E0E6
:10DDF000BE016D5B7F4FCE0189599F4F0E94F8CFC6
:10DE0000EECF46E050E0BE01635C7F4FCE01895902
:10DE10009F4F0E94F8CF9E012B593F4F44E050E0A6
:10DE200063EE76E0CE0189599F4F0E94F8CF9E01A4
:10DE30002B593F4F4CE050E0BE016F5C7F4FCE014D
:10DE400089599F4F0E94F8CF2CE1F22EFA94F110DD
:10DE500003C094E0F92E1DC000E09E012B593F4FF6
:10DE600044E050E0BE01695A7F4FCE0189599F4F6F
:10DE70000E94F8CFEBCF00E09E012B593F4F44E0CA
:10DE800050E0BE01695A7F4FCE0189599F4F0E94D1
:10DE9000F8CFFA94F110EFCF8BE0F82EFA94FF2030
:10DEA00079F000E09E012B593F4F44E050E0BE0165
:10DEB000695A7F4FCE0189599F4F0E94F8CFEECF0C
:10DEC000A9968EAD9FADA99784569109C7DA809324
:10DED0001607882309F1E4EEFDE184917F019FEFAD
:10DEE000E91AF90A882321F00E94CC89F701F5CFBD
:10DEF000A9966EAD7FADA997645671098AE79AE13C
:10DF00000E9454C56BED72E082E79AE10E9454C50D
:10DF10008AE00E94CC8999C0A7962EAD3FADA79705
:10DF2000AB968EAD9FADAB972817390709F44BC060
:10DF300081E080931607EFECFDE184917F012FEFE4
:10DF4000E21AF20A811103C0E2E5FAE104C00E947C
:10DF5000CC89F701F2CF84917F013FEFE31AF30AF6
:10DF6000882321F00E94CC89F701F5CFAB966EADE6
:10DF70007FADAB9780E090E04AE00E94EF8CEDE44B
:10DF8000FAE184917F019FEFE91AF90A882321F0D1
:10DF90000E94CC89F701F5CFA7966EAD7FADA7970C
:10DFA00080E090E04AE00E94EF8CEDE3FAE184919A
:10DFB0007F012FEFE21AF20A882309F446C00E947B
:10DFC000CC89F701F4CF111142C0E4EEFDE1849158
:10DFD0007F013FEFE31AF30A811103C00FED12E056
:10DFE00004C00E94CC89F701F2CFF80181918F0122
:10DFF000882319F00E94CC89F8CFA9966EAD7FAD29
:10E00000A9976456710980E29AE10E9454C5A796C7
:10E010004EAD5FADA79760E070E083E19AE10E94AA
:10E020001AC5E0E1FAE184917F012FEFE21AF20ACA
:10E03000811107C080911607811109C00E94B9D0D3
:10E0400006C00E94CC89F701EECF112399F3E69622
:10E050008EAD9FADE6970FB6F8949EBF0FBE8DBFF5
:10E0600080911707811102C00E9482BE909116070D
:10E0700081E089270FB6F8943EBE0FBE2DBEC95869
:10E08000DF4F0FB6F894DEBF0FBECDBFDF91CF914B
:10E090001F910F91FF90EF90DF90CF90BF90AF90C6
:10E0A0009F908F907F906F905F904F903F902F90B8
:10E0B000089581E080931707F2D910921707811114
:10E0C000EEC90E94F1C281E008958F929F92AF92B3
:10E0D000BF92CF92DF92EF92FF920F931F93CF9355
:10E0E000DF93CDB7DEB7CA5AD1090FB6F894DEBFB9
:10E0F0000FBECDBFE9961CAE1DAE1EAE1FAEE9979A
:10E100008091EC039091ED03A091EE03B091EF03A9
:10E11000ED968CAF9DAFAEAFBFAFED97C556DF4F5D
:10E1200019821882CB59D04084E690E0C356DF4F65
:10E1300099838883CD59D040109216079E012556A9
:10E140003F4F44E050E0BE0167587F4FCE018356F9
:10E150009F4F0E9445D0C356DF4F88819981CD598A
:10E16000D0400296C356DF4F99838883CD59D04063
:10E17000C556DF4F19821882CB59D04081E0CD556A
:10E18000DF4F8883C35AD0409E0125563F4F41E060
:10E1900050E0BE016D557F4FCE0183569F4F0E94C8
:10E1A00045D09E0125563F4F40E150E06FE471E1BC
:10E1B000CE0183569F4F0E9445D09E0125563F4F6A
:10E1C00044E050E063E077E0CE0183569F4F0E9429
:10E1D00045D09E0125563F4F40E150E062E970E195
:10E1E000CE0183569F4F0E9445D09E0125563F4F3A
:10E1F00040E150E063EF76E0CE0183569F4F0E94EE
:10E2000045D09E0125563F4F44E050E06BEE76E04E
:10E21000CE0183569F4F0E9445D09E0125563F4F09
:10E2200044E050E06FEE76E0CE0183569F4F0E94AF
:10E2300045D09E0125563F4F44E050E067EE76E022
:10E24000CE0183569F4F0E9445D09E0125563F4FD9
:10E2500044E050E06BE077E0CE0183569F4F0E9490
:10E2600045D09E0125563F4F44E050E067E077E0FF
:10E27000CE0183569F4F0E9445D09E0125563F4FA9
:10E2800040E150E063ED76E0CE0183569F4F0E945F
:10E2900045D08AE097EDA3EABCE3E9968CAF9DAF49
:10E2A000AEAFBFAFE9979E0125563F4F44E050E027
:10E2B000BE016B587F4FCE0183569F4F0E9445D0C1
:10E2C0009E0125563F4F4CE050E068E375E0CE01DB
:10E2D00083569F4F0E9445D080917D1090917E1073
:10E2E000A0917F10B0918010C358DF4F888399832D
:10E2F000AA83BB83CD57D0409E0125563F4F44E0B3
:10E3000050E0BE0163587F4FCE0183569F4F0E945D
:10E3100045D085E0CC55DF4F8883C45AD040CB55DB
:10E32000DF4F8883C55AD0409E0125563F4F44E0B9
:10E3300050E062EC70E1CE0183569F4F0E9445D0C1
:10E340009E0125563F4F41E050E0BE016C557F4F86
:10E35000CE0183569F4F0E9445D09E0125563F4FC8
:10E3600041E050E0BE016B557F4FCE0183569F4F79
:10E370000E9445D09E0125563F4F44E650E066EC92
:10E3800070E1CE0183569F4F0E9445D0CF57DF4F9B
:10E39000188219821A821B82C158D0409E012556CC
:10E3A0003F4F44E050E0BE016F577F4FCE01835690
:10E3B0009F4F0E9445D0E9961CAE1DAE1EAE1FAE0B
:10E3C000E9971AE0115071F09E0125563F4F44E045
:10E3D00050E0BE016B587F4FCE0183569F4F0E9485
:10E3E00045D0F0CF83E0CA55DF4F8883C65AD0406E
:10E3F000C955DF4F8883C75AD040CB57DF4F1882AB
:10E4000019821A821B82C558D040C757DF4F188225
:10E4100019821A821B82C958D040E9961CAE1DAEE3
:10E420001EAE1FAEE9979E0125563F4F41E050E0DA
:10E43000BE016A557F4FCE0183569F4F0E9445D043
:10E440009E0125563F4F41E050E0BE0169557F4F88
:10E45000CE0183569F4F0E9445D09E0125563F4FC7
:10E4600044E050E0BE0167577F4FCE0183569F4F77
:10E470000E9445D09E0125563F4F44E050E0BE012A
:10E480006B577F4FCE0183569F4F0E9445D00AE0C5
:10E4900010E00150110971F09E0125563F4F44E0F4
:10E4A00050E0BE016B587F4FCE0183569F4F0E94B4
:10E4B00045D0EFCFC855DF4F1882C85AD0408FEFF4
:10E4C000C755DF4F8883C95AD0409E0125563F4F1C
:10E4D00041E050E0BE0168557F4FCE0183569F4F0B
:10E4E0000E9445D09E0125563F4F41E050E0BE01BD
:10E4F00067557F4FCE0183569F4F0E9445D0E996C6
:10E500001CAE1DAE1EAE1FAEE9979E0125563F4FB5
:10E5100044E050E0BE016B587F4FCE0183569F4FC1
:10E520000E9445D09E0125563F4F44E050E0BE0179
:10E530006B587F4FCE0183569F4F0E9445D09E015E
:10E5400025563F4F44E050E067E371E1CE0183562A
:10E550009F4F0E9445D080918B0290918C02A09198
:10E560008D02B0918E02C357DF4F88839983AA83AF
:10E57000BB83CD58D04080918F0290919002A091A2
:10E580009102B0919202CF56DF4F88839983AA837C
:10E59000BB83C159D040CB56DF4F19821882C55971
:10E5A000D040C956DF4F19821882C759D0409E010A
:10E5B00025563F4F44E050E0BE0163577F4FCE01E8
:10E5C00083569F4F0E9445D09E0125563F4F44E001
:10E5D00050E0BE016F567F4FCE0183569F4F0E9481
:10E5E00045D09E0125563F4F44E050E0BE016B569A
:10E5F0007F4FCE0183569F4F0E9445D010E0C12C23
:10E6000080E8D82E8BE3E82E85E4F82E812C912C1F
:10E6100090E8A92E9FE3B92E111138C09E0125560E
:10E620003F4F44E050E06CE377E0CE0183569F4FCC
:10E630000E9445D09E0125563F4F44E050E068E3DC
:10E6400077E0CE0183569F4F0E9445D09E0125560C
:10E650003F4F44E050E060E477E0CE0183569F4FA7
:10E660000E9445D0E9968CAE9DAEAEAEBFAEE997A6
:10E670009E0125563F4F44E050E0BE016B587F4F4E
:10E68000CE0183569F4F0E9445D02AC0E996CCAE5A
:10E69000DDAEEEAEFFAEE9979E0125563F4F44E05A
:10E6A00050E0BE016B587F4FCE0183569F4F0E94B2
:10E6B00045D0E9961CAE1DAE1EAE1FAEE99704E034
:10E6C000015071F09E0125563F4F44E050E0BE01DD
:10E6D0006B587F4FCE0183569F4F0E9445D0F0CF9D
:10E6E0001F5F153009F098CF84E190E0C156DF4FED
:10E6F00099838883CF59D0409E0125563F4F42E0F1
:10E7000050E0BE0161567F4FCE0183569F4F0E945D
:10E7100045D09E0125563F4F44E050E064E377E04A
:10E72000CE0183569F4F0E9445D09E0125563F4FF4
:10E7300044E050E060E377E0CE0183569F4F0E94B3
:10E7400045D09E0125563F4F44E050E06CE277E013
:10E75000CE0183569F4F0E9445D080E290E0CF5576
:10E76000DF4F99838883C15AD0409E0125563F4F81
:10E7700042E050E0BE016F557F4FCE0183569F4F60
:10E780000E9445D0C655DF4F1882CA5AD04080E259
:10E79000E3E9F2E0DE019D9601900D928A95E1F7A2
:10E7A0009E0125563F4F41E050E0BE0166557F4F28
:10E7B000CE0183569F4F0E9445D09E0125563F4F64
:10E7C00040E250E0BE01635D7F4FCE0183569F4F14
:10E7D0000E9445D09E0125563F4F41E050E06AE23D
:10E7E00071E1CE0183569F4F0E9445D010E0111178
:10E7F0000EC080912F1190913011A0913111B091E4
:10E800003211E9968CAF9DAFAEAFBFAFE9979E01D5
:10E8100025563F4F44E050E0BE016B587F4FCE017C
:10E8200083569F4F0E9445D01F5F153001F7BE01F0
:10E83000635B7F4F86E1FB0111928A95E9F79E01A8
:10E8400025563F4F46E150E0CE0183569F4F0E9430
:10E8500045D08CE2E3EBF2E0DE01119601900D92DF
:10E860008A95E1F79E0125563F4F4CE250E0BE01EC
:10E870006F5F7F4FCE0183569F4F0E9445D0BE01F0
:10E8800061597F4F86E0FB0111928A95E9F79E015D
:10E8900025563F4F46E050E0CE0183569F4F0E94E1
:10E8A00045D09E0125563F4F44E050E063EE76E0B0
:10E8B000CE0183569F4F0E9445D0BE016D597F4FB8
:10E8C0008CE0FB0111928A95E9F79E0125563F4F96
:10E8D0004CE050E0CE0183569F4F0E9445D0E99610
:10E8E0001CAE1DAE1EAE1FAEE9971CE1115071F0BB
:10E8F0009E0125563F4F44E050E0BE016B587F4FCC
:10E90000CE0183569F4F0E9445D0F0CFE9961CAEB2
:10E910001DAE1EAE1FAEE99714E0115071F09E01BE
:10E9200025563F4F44E050E0BE016B587F4FCE016B
:10E9300083569F4F0E9445D0F0CFE9961CAE1DAE86
:10E940001EAE1FAEE9971BE0115071F09E012556D7
:10E950003F4F44E050E0BE016B587F4FCE018356DD
:10E960009F4F0E9445D0F0CF80911607811167C05C
:10E97000C356DF4FE880F980CD59D040F4E6EF1A56
:10E98000F108C556DF4F88819981CB59D040C756D1
:10E99000DF4F99838883C959D04084E690E0C356FD
:10E9A000DF4F99838883CD59D0409E0125563F4F34
:10E9B00044E050E06FED72E0CE0183569F4F0E941D
:10E9C00045D09E0125563F4F42E050E0BE016756BC
:10E9D0007F4FCE0183569F4F0E9445D0E4EEFDE16C
:10E9E00084918F010F5F1F4F882321F00E94CC89F3
:10E9F000F801F6CFB7018EEF99E10E9454C5C756D2
:10EA0000DF4F48815981C959D04060E070E081EF03
:10EA100099E10E941AC5EEEEF9E184918F010F5F32
:10EA20001F4F882321F00E94CC89F801F6CFC7013F
:10EA30000E942E6A90911607892B80931607909159
:10EA4000160781E08927C655DF4F0FB6F894DEBF61
:10EA50000FBECDBFDF91CF911F910F91FF90EF902F
:10EA6000DF90CF90BF90AF909F908F900895FF92CE
:10EA70000F931F93CF93DF938C01EB01F42E80E271
:10EA80000E94CC898FEFF81611F084E501C082E472
:10EA90000E94CC898AE30E94CC89F801608171814F
:10EAA0008281938142E00E94748D488159816A81FC
:10EAB0007B818DE49DE10E9437C562E070E080E0DB
:10EAC00090E0DF91CF911F910F91FF900C9410B7C0
:10EAD0008F929F92AF92BF92CF92DF92EF92FF926E
:10EAE0000F931F93CF93DF93F0E2FF2EE12CAE2D17
:10EAF000B0E0BD016F0D711D759567956E1511F034
:10EB0000F6120BC0E0E3FBE165917491072E000C57
:10EB1000880B990B0E9443E662C09B01215031098A
:10EB2000220F331F220F331FF901EE54F54E0591CA
:10EB30001491AB01440F551F440F551FFA01EE54B9
:10EB4000F54EC591D4918017910714F4F62ED1CFCC
:10EB5000C817D90714F4E62ECACFF901EC54F54EC4
:10EB6000E590F490FA01EC54F54EC590D490BC01B8
:10EB7000601B710B072E000C880B990B0E9443E65B
:10EB80004B015C01B6016E197F09072E000C880B42
:10EB9000990B0E9443E69B01AC01C501B4010E94A0
:10EBA000A2E64B015C01C01BD10BBE01DD0F880B3F
:10EBB000990B0E9443E69B01AC01C501B4010E9480
:10EBC00065EB4B015C01B701FF0C880B990B0E94B0
:10EBD00043E69B01AC01C501B4010E9489EADF91C3
:10EBE000CF911F910F91FF90EF90DF90CF90BF904A
:10EBF000AF909F908F9008950F931F93CF93DF93C3
:10EC0000CDB7DEB728970FB6F894DEBF0FBECDBFE5
:10EC100060914A0470914B04072E000C880B990BED
:10EC20000E9443E66D837E838F83988780914C0496
:10EC300090914D04A0914E04B0914F0489839A8322
:10EC4000AB83BC834DEFBE016B5F7F4FCE0101965E
:10EC50000EDF6091440470914504072E000C880B70
:10EC6000990B0E9443E66D837E838F839887809102
:10EC7000460490914704A0914804B09149048983C7
:10EC80009A83AB83BC834FEFBE016B5F7F4FCE0196
:10EC90000196EDDEE5E5FDE184918F010F5F1F4FE9
:10ECA000882321F00E94CC89F801F6CFE0914E072D
:10ECB000F0E0E45BF84F608170E080E090E00E945B
:10ECC0005A8DE0E5FDE184918F010F5F1F4F88238E
:10ECD00021F00E94CC89F801F6CF60914D0770E0D9
:10ECE00080E090E00E945A8D28960FB6F894DEBF1F
:10ECF0000FBECDBFDF91CF911F910F9108950F935C
:10ED00000FB70F9300916E000B7F00936E00789405
:10ED10000F930BB70F930CB70F921F922F933F9344
:10ED20004F935F936F937F938F939F93AF93BF9313
:10ED3000EF93FF931124EFD2FF91EF91BF91AF9129
:10ED40009F918F917F916F915F914F913F912F9103
:10ED50001F900F900CBF0F910BBF0F910460F894A0
:10ED600000936E000F910FBF0F911895CF92DF9215
:10ED7000EF92FF92C0904604D0904704E090480480
:10ED8000F090490460914404709145046650710903
:10ED9000072E000C880B990B0E9443E69B01AC01E7
:10EDA000C701B6010E943DE687FF1FC020E030E0AA
:10EDB00040E050E4C701B6010E9489EA0E94D2EB0C
:10EDC00070938607609385070E94FE58DC01CB0193
:10EDD000805A9541AF4FBF4F809381079093820730
:10EDE000A0938307B093840708C010928107109204
:10EDF00082071092830710928407FF90EF90DF90B4
:10EE0000CF900895CF92DF92EF92FF92C0904C0482
:10EE1000D0904D04E0904E04F0904F0460914A046D
:10EE200070914B0467507109072E000C880B990BE9
:10EE30000E9443E69B01AC01C701B6010E943DE67A
:10EE400087FF1FC020E030E040E450E4C701B60176
:10EE50000E9489EA0E94D2EB7093800760937F073B
:10EE60000E94FE58DC01CB01805A9541AF4FBF4F45
:10EE700080937B0790937C07A0937D07B0937E07D8
:10EE800008C010927B0710927C0710927D071092A9
:10EE90007E07FF90EF90DF90CF9008958F929F9222
:10EEA000AF92BF92CF92DF92EF92FF920F931F9398
:10EEB000CF93DF93F0E4FF2EE12CAE2DB0E0BD0147
:10EEC0006F0D711D759567956E1511F0F6120BC0DB
:10EED000E2EAFCE165917491072E000C880B990B16
:10EEE0000E9443E662C09B0121503109220F331F6B
:10EEF000220F331FF901EC55F44E05911491AB012B
:10EF0000440F551F440F551FFA01EC55F44EC5919F
:10EF1000D4918017910714F4F62ED1CFC817D907D2
:10EF200014F4E62ECACFF901EA55F44EE590F490B8
:10EF3000FA01EA55F44EC590D490BC01601B710BE8
:10EF4000072E000C880B990B0E9443E64B015C01D5
:10EF5000B6016E197F09072E000C880B990B0E94D1
:10EF600043E69B01AC01C501B4010E94A2E64B013E
:10EF70005C01C01BD10BBE01DD0F880B990B0E94F9
:10EF800043E69B01AC01C501B4010E9465EB4B0156
:10EF90005C01B701FF0C880B990B0E9443E69B01B3
:10EFA000AC01C501B4010E9489EADF91CF911F91A4
:10EFB0000F91FF90EF90DF90CF90BF90AF909F9018
:10EFC0008F90089560E0809191079091920780DD85
:10EFD00060934C0470934D0480934E0490934F04BF
:10EFE00080918F079091900759DF6093460470934A
:10EFF00047048093480490934904A89510924907C8
:10F0000008957F928F929F92AF92BF92CF92DF929C
:10F01000EF92FF920F931F93CF93DF9320E030E0A6
:10F0200048E452E460914C0470914D0480914E0488
:10F0300090914F040E94AFEC18164CF4E8E3FBE10A
:10F04000E491C1E001C0CC0FEA95EAF701C0C0E04D
:10F0500082E3E82E8BE1F82E08E31BE196E0A92E6F
:10F06000912CD0E0CC24C394D12CF7017490F801FA
:10F07000849077FC23C0892D90E0082C02C09595E0
:10F0800087950A94E2F780FD19C0BE01082C02C0E2
:10F09000759567950A94E2F76170B62EB1946B2D61
:10F0A000872D0E94DFB56B2D70E0872D0E9449B639
:10F0B000C60101C0880F8A94EAF7982AAA94FFEF44
:10F0C000EF1AFF0A0F5F1F4FA110CFCFDF91CF9133
:10F0D0001F910F91FF90EF90DF90CF90BF90AF9076
:10F0E0009F908F907F9008950F931F9380912B078F
:10F0F000813019F40E94FE5808C060912707709172
:10F1000028078091290790912A07009153071091B1
:10F1100054072091550730915607601B710B820BE5
:10F12000930B28EE33E040E050E00E942BEA809100
:10F130004F0790915007A0915107B0915207BC0121
:10F14000CD01620F731F841F951F1F910F910895AA
:10F1500010922B07109253071092540710925507E4
:10F16000109256071092270710922807109229072D
:10F1700010922A0710924F071092500710925107D1
:10F1800010925207089580912B078130E1F0823070
:10F1900051F4AADF60934F07709350078093510793
:10F1A0009093520701C0D4DF81E080932B070E9427
:10F1B000FE586093530770935407809355079093BC
:10F1C000560781E0089580E0089580912B078130F3
:10F1D00079F482E080932B070E94FE586093270702
:10F1E000709328078093290790932A0781E0089558
:10F1F00080E0089580912B078150823010F080E0EC
:10F20000089510922B070E94FE5860932707709371
:10F2100028078093290790932A0781E00895109288
:10F22000480780E090E00E94F35910924504109244
:10F2300044049CDDDFDF80E090E00E94F3591092EF
:10F240004C072C98109245041092440410924D07DC
:10F25000809102018072809300010895DF92EF9205
:10F26000FF920F931F93CF93DF93F82ED62EE72EA6
:10F270008A0180912702882309F439C0EFECFDE16F
:10F280008491EF012196882321F00E94CC89FE0110
:10F29000F7CFED2DFE2D8491EF012196882321F0EB
:10F2A0000E94CC89FE01F7CFE3E4FBE18491EF01FA
:10F2B0002196882321F00E94CC89FE01F7CFF7FC2C
:10F2C0000BC06F2DFF0C770B880B990B0E945A8D8A
:10F2D0008AE00E94CC890BC0EEE3FBE18491EF0150
:10F2E0002196882321F00E94CC89FE01F7CF8091DE
:10F2F0005707811108C01092270281E080935707B9
:10F30000C8010E94BBA0DF91CF911F910F91FF9088
:10F31000EF90DF9084CFEF92FF920F931F93CF93E4
:10F32000DF9380912A028F37A0F08F5790914C077E
:10F330009093A207992311F02C9A01C02C98209148
:10F340004D072093A10790910201222369F0909527
:10F350000BC09091A207891708F02C989091A107F3
:10F36000891728F0909102019072909300018F5FAD
:10F3700080932A029091A00781E089278093A007BB
:10F380008091290285301CF4C1E0C80F01C0C0E0A3
:10F39000823009F4B4C054F4882301F1813009F0BB
:10F3A000E3C088E080937B0085E4C0C0843009F42A
:10F3B000C5C00CF4B7C0853009F0D6C090919F0746
:10F3C000911102C080939F0780919F078150809385
:10F3D0009F07882309F4C8C0C5E0C6C080912802F1
:10F3E0008F5F80311CF480932802BEC010922802E7
:10F3F00080914907811113C08091950790919607DC
:10F40000909392078093910780919307909194072E
:10F410009093900780938F0781E0809349078AE05B
:10F42000E5E9F7E0DF011D928A95E9F7109294076C
:10F4300010929307009191071091920711950195F1
:10F44000110980914A0490914B04D1E018161906D5
:10F450002CF080914C07811101C0D0E080913205E1
:10F46000909133059195819591098017910734F416
:10F470004BED5CE16CEF7CE180E0F0DE80911C0202
:10F4800090911D029195819591090817190744F4EF
:10F49000DD2331F04EE05DE16FE27DE180E0DEDE14
:10F4A000809144049091450411E0181619062CF03F
:10F4B00080914D07811101C010E0E0908F07F0901E
:10F4C000900780913005909131058E159F0534F09D
:10F4D0004BEE5CE16CEF7CE18FEFC0DE80911A02B5
:10F4E00090911B02E816F9060CF43EC01123E1F1DD
:10F4F0004EE15DE16FE27DE18FEFB0DE35C08091DE
:10F500007A0086FD2EC0809178009091790020913C
:10F51000950730919607820F931F909396078093DB
:10F52000950722C088E080937B0086E480937C006E
:10F5300080917A00806480937A0016C080917A006E
:10F5400086FD11C0809178009091790020919307F9
:10F5500030919407820F931F9093940780939307A1
:10F5600003C0C2E001C0C4E0C09329028091370506
:10F5700081110E94C5BD80914A0790914B07009769
:10F58000A9F0019790934B0780934A07892B71F458
:10F5900081E49DE19093A4078093A307DF91CF912D
:10F5A0001F910F91FF90EF900C94F889DF91CF910C
:10F5B0001F910F91FF90EF9008952F923F924F92DD
:10F5C0005F926F927F928F929F92AF92BF92CF92F3
:10F5D000DF92EF92FF920F931F93CF93DF9300D0B0
:10F5E0001F92CDB7DEB75C017A8369834A011701A8
:10F5F00007FD07C0802F002E000C990B9C838B8386
:10F6000004C0E1E0F0E0FC83EB83F901408051802D
:10F61000628073808B819C81880F991F880F991F4E
:10F620009C838B838957984F7C01A3019201FC0135
:10F6300060817181828193810E943DE6882391F0EF
:10F64000F701408251826282738211E020E030E053
:10F65000A901C301B2010E94AFEC18160CF010E032
:10F66000F5011083F50180818230D1F0833009F4F7
:10F670005EC0813009F07CC0EB81FC81E957F84F16
:10F680002081318142815381F401608171818281C5
:10F6900093810E943DE687FD6BC082E0F501808387
:10F6A0008B819C818957984F9C838B83B60180E026
:10F6B00090E00E9441E69B01AC01EB81FC816081FE
:10F6C0007181828193810E9488EA9B01AC01F401DF
:10F6D00060817181828193810E94AFEC87FD14C0AB
:10F6E0000E94FE586B017C019101A8EEB3E00E94DC
:10F6F00079EAC60ED71EE81EF91EE981FA81C0829A
:10F70000D182E282F38234C00E94FE58E981FA81FC
:10F71000C080D180E280F380DC01CB018C199D098F
:10F72000AE09BF09B7FD24C083E0F50180830F3F18
:10F7300019F044EA5CE102C047EB5CE16BEC7CE170
:10F74000802F0F900F900F900F90DF91CF911F910E
:10F750000F91FF90EF90DF90CF90BF90AF909F9070
:10F760008F907F906F905F904F903F902F9076CDCD
:10F770000F900F900F900F90DF91CF911F910F91ED
:10F78000FF90EF90DF90CF90BF90AF909F908F90C1
:10F790007F906F905F904F903F902F9008954F9281
:10F7A0005F926F927F928F929F92AF92BF92CF9211
:10F7B000DF92EF92FF920F931F93CF93DF93CDB71A
:10F7C000DEB760970FB6F894DEBF0FBECDBF809155
:10F7D0004907811117C060960FB6F894DEBF0FBEBF
:10F7E000CDBFDF91CF911F910F91FF90EF90DF90F0
:10F7F000CF90BF90AF909F908F907F906F905F90D1
:10F800004F900895DFDB0E94FE584B015C01609130
:10F810004A0470914B04072E000C880B990B0E9430
:10F8200043E669837A838B839C8344E1C42ED12C85
:10F830005CE3E52EF12C00E09E012F5F3F4F4CE48E
:10F8400054E067E777E086E797E0B7DEC0904C04C6
:10F85000D0904D04E0904E04F0904F046091340538
:10F8600070913505072E000C880B990B0E9443E61A
:10F870009B01AC01C701B6010E94AFEC18160CF059
:10F8800009C160911E0270911F02072E000C880BA7
:10F89000990B0E9443E69B01AC01C701B6010E948F
:10F8A0003DE687FFF7C000914A0410914B04B80170
:10F8B000012E000C880B990B0E9443E6A7019601CC
:10F8C0000E9488EA2B013C0120ED3CEC4CE45DE316
:10F8D00060914007709141078091420790914307E2
:10F8E0000E94A2E66D837E838F83988720916D07A7
:10F8F00030916E0740916F0750917007C701B601B4
:10F900000E9488EA9B01AC016D817E818F81988580
:10F910000E94A2E66D837E838F83988723E333E37F
:10F9200043E75FE36091690770916A0780916B0715
:10F9300090916C070E94A2E69B01AC016D817E81D3
:10F940008F8198850E9489EA6D837E838F83988753
:10F950006093690770936A0780936B0790936C07B5
:10F96000C0926D07D0926E07E0926F07F092700719
:10F9700020E030E040E251E4C301B2010E94AFEC6C
:10F9800018160CF431C220E030E040E251ECC30123
:10F99000B2010E943DE687FD2FC2012B09F42CC263
:10F9A0008091680781112CC220916407309165070E
:10F9B000409166075091670729873A874B875C8794
:10F9C00020913C0730913D0740913E0750913F0701
:10F9D000C301B2010E94A2E66B017C01A301920166
:10F9E00069857A858B859C850E9489EA69877A87F3
:10F9F0008B879C8760936407709365078093660785
:10FA000090936707209138073091390740913A0762
:10FA100050913B070E94A2E6A70196010E9489EA45
:10FA20002D813E814F8158850E9488EA6B017C01BF
:10FA300020E030E04FE753E40E94AFEC20E030E0FC
:10FA4000A90118160CF4E3C1C701B6010E943DE6F6
:10FA500087FD07C0C701B6010E94CDEB759567957C
:10FA60001AC020E030E0A901C301B2010E943DE6C6
:10FA700087FF10C0A301920169857A858B859C85DB
:10FA80000E9488EA60936407709365078093660715
:10FA90009093670760E060934C0780917B0790919B
:10FAA0007C07A0917D07B0917E070097A105B10565
:10FAB00021F1A5019401281B390B4A0B5B0B57FD63
:10FAC0001CC060917F077091800780E090E00E94E9
:10FAD00041E69B01AC0160914C0470914D04809112
:10FAE0004E0490914F040E943DE687FF82C143E897
:10FAF0005BE165E97BE180E0B1DB809144079091B7
:10FB00004507A0914607B0914707A5019401281B1E
:10FB1000390B4A0B5B0B57FD0FC073DAD501C401DB
:10FB20008C53964FAF4FBF4F809344079093450738
:10FB3000A0934607B0934707809181079091820771
:10FB4000A0918307B09184070097A105B10511F139
:10FB5000881A990AAA0ABB0AB7FC1CC060918507DB
:10FB60007091860780E090E00E9441E69B01AC0125
:10FB70006091460470914704809148049091490433
:10FB80000E943DE687FF20C141E65BE164E77BE13F
:10FB90008FEF64DB6091440470914504072E000CE4
:10FBA000880B990B0E9443E669837A838B839C833D
:10FBB00095E0C92ED12C24E1E22EF12C0FEF9E010D
:10FBC0002F5F3F4F46E454E061E777E085E797E039
:10FBD000F4DCC0904604D0904704E0904804F090D4
:10FBE000490420E030E040EA50E4C701B6010E9439
:10FBF000AFEC87FDE5C020E030E04CED52E4C701FA
:10FC0000B6010E943DE618160CF4DAC06091440477
:10FC100070914504072E000C880B990B0E9443E657
:10FC2000A70196010E9488EA4B015C0120913407EC
:10FC30003091350740913607509137070E94A2E670
:10FC400069877A878B879C8720916007309161074D
:10FC50004091620750916307C501B4010E9489EA8F
:10FC60006D837E838F8398876093600770936107AD
:10FC7000809362079093630720913007309131079A
:10FC800040913207509133070E94A2E66D877E872C
:10FC90008F87988B20ED3CEC4CE45DE360912C0762
:10FCA00070912D0780912E0790912F070E94A2E658
:10FCB0002B013C0120915C0730915D0740915E076C
:10FCC00050915F07C701B6010E9488EA9B01AC0111
:10FCD000C301B2010E94A2E62B013C0123E333E3FE
:10FCE00043E75FE3609158077091590780915A0785
:10FCF00090915B070E94A2E69B01AC01C301B20197
:10FD00000E9489EA2B013C016093580770935907C0
:10FD100080935A0790935B07C0925C07D0925D076F
:10FD2000E0925E07F0925F072D853E854F855889EA
:10FD300069857A858B859C850E9489EAA301920159
:10FD40000E9488EA6B017C0120E030E04FE753E439
:10FD50000E94AFEC20E030E0A9011816C4F5C501FF
:10FD6000B4010E94AFEC181684F4A50194016D81D2
:10FD70007E818F8198850E9488EA609360077093E6
:10FD8000610780936207909363076FE71AC020E0D2
:10FD900030E0A901C501B4010E943DE687FF10C013
:10FDA000A50194016D817E818F8198850E9488EAEA
:10FDB0006093600770936107809362079093630775
:10FDC00060E060934D0707CD0E94B676E3CEC70191
:10FDD000B6010E943DE687FDDACFC701B6010E9459
:10FDE000CDEB75956795EDCF81E0809368076FE760
:10FDF00052CE80E007D881CE81E0809368074ACE5A
:10FE00001092680719861A861B861C86D9CDC301F5
:10FE1000B2010E94AFEC181654F7A3019201698554
:10FE20007A858B859C850E9488EA6093640770932D
:10FE3000650780936607909367076FE72CCE9091D4
:10FE40006F00292F227091FF05C090916F009D7F58
:10FE500090936F0034E0839FC0011124FC01EE57A2
:10FE6000FF4E4081518162817381FC01E55EF84F54
:10FE7000408351836283738381E080931A07222336
:10FE800029F080916F00826080936F000895BC011B
:10FE900020911807309119074091180750911907C0
:10FEA0002417350711F09A01F7CF81E0261737079D
:10FEB00009F080E008958F929F92AF92BF92CF9207
:10FEC000DF92EF92FF921F93CF93DF93C82F83EDC2
:10FED0009BE09093AF098093AE091092EF0B82E004
:10FEE00090E0A0E0B0E08093D80B9093D90BA09362
:10FEF000DA0BB093DB0B1092AD091092A9091092A6
:10FF0000AA091092AB091092AC098FEF9FEFDC01A8
:10FF10008093A5099093A609A093A709B093A80977
:10FF2000CC2379F1C53008F0F8C040E060E070E023
:10FF3000CB010E94A1D1882309F4EFC020E1C29F28
:10FF4000C00111248B56984FFC01E254FE4F2081D2
:10FF50002F7709F0E2C03C96408151816281738124
:10FF6000443651056105710508F4D7C03497C08047
:10FF7000D180E280F380C114D104E104F10421F4C2
:10FF8000CCC0C12CD12C760140E0C701B6010E9443
:10FF9000A1D1182F882309F4C0C08091B007909197
:10FFA000B1078115924009F0B8C0A091B507AA2306
:10FFB00009F4B3C06091B3077091B407611571057E
:10FFC00009F4ABC02091B207222309F4A6C0A09384
:10FFD000EA0B2093DC0B80E030E041E050E0C82FDA
:10FFE000FA01082E02C0EE0FFF1F0A94E2F72E1747
:10FFF0003F0739F08F5FC83091F789E08093E50BB8
:020000021000EC
:100000008CC08093E50B2091BB073091BC07211574
:10001000310519F040E050E008C02091C907309147
:10002000CA074091CB075091CC072093DD0B30934A
:10003000DE0B4093DF0B5093E00B46015701860E19
:10004000971EA11CB11C8092EB0B9092EC0BA0921E
:10005000ED0BB092EE0BE091B607F091B707F0937D
:10006000F10BE093F00BB0E00E9469EA860E971E58
:10007000A81EB91E8092F20B9092F30BA092F40B83
:10008000B092F50B85E0EE0FFF1F8A95E1F7E15086
:10009000FE4FEF2FFF27E6958E0E9F1EA11CB11C71
:1000A0008092E60B9092E70BA092E80BB092E90BDE
:1000B0002091B8073091B9072115310521F0A90128
:1000C00060E070E008C04091C5075091C60760919C
:1000D000C7077091C807D701C60188199909AA09ED
:1000E000BB09840F951FA61FB71F04C0B695A7951F
:1000F00097958795CA95D2F78093E10B9093E20B81
:10010000A093E30BB093E40B853F2FE09207A1058A
:10011000B10528F48CE08093EF0B10E01AC0853F06
:100120009F4FA105B10510F480E111C08091D10766
:100130009091D207A091D307B091D4078093F20B8E
:100140009093F30BA093F40BB093F50B80E28093A4
:10015000EF0B812FDF91CF911F91FF90EF90DF90F8
:10016000CF90BF90AF909F908F900895682F8AE9AD
:100170009FE00C94E04ACF92DF92EF92FF921F93A0
:10018000CF93DF931092320A8091650A882321F081
:1001900082E69AE00E94DF981092D70B1092D40B5F
:1001A00085E38093D30B0E94FE58EB01A89561E094
:1001B0008091D30B0E940DB683ED9BE00E94409A84
:1001C0002398229A219A209A289A85E08093D50B29
:1001D00082E58CBD1DBC1AE08FEF0E94459A11503C
:1001E000D9F720E030E0A90160E083ED9BE00E94B8
:1001F0004A9A182F8093D60B813049F00E94FE58FE
:100200006C1B7D0B613D774060F381E054C02AEAAE
:1002100031E040E050E068E083ED9BE00E944A9AC4
:1002200082FF03C01093D70B0EC014E00E94589FAA
:100230008093D60B1150D1F78A3A11F082E03BC07F
:1002400082E08093D70B8091D70B823021F0C12CB4
:10025000D12C760105C0C12CD12CE12C80E4F82EE4
:1002600020E030E0A90167E383ED9BE00E944A9A19
:10027000A701960169E283ED9BE00E944A9A809370
:10028000D60B882349F00E94FE586C1B7D0B613D04
:10029000774030F38AE00FC08091D70B823011F5A0
:1002A00020E030E0A9016AE383ED9BE00E944A9AD6
:1002B000882351F088E08093D40B83ED9BE00E946B
:1002C000409AE4EEFDE119C00E94589F807C803C7A
:1002D00019F483E08093D70B0E94589F0E94589F87
:1002E0000E94589F83ED9BE00E94409A1092D50B8C
:1002F00081E0E1DD811131C015C08491EF012196CB
:10030000882321F00E94CC89FE01F7CFE6EDFDE1C4
:100310008491EF012196882309F454C00E94CC896E
:10032000FE01F6CF80E0C7DD811117C0EFECFDE1E3
:100330008491EF012196882321F00E94CC89FE014F
:10034000F7CFEBEBFDE18491EF012196882309F4CF
:1003500039C00E94CC89FE01F6CF68ED7BE082E6D1
:100360009AE00E948C98811116C0EFECFDE1849117
:10037000EF012196882321F00E94CC89FE01F7CF5E
:10038000EAEAFDE18491EF0121968823D9F00E94E9
:10039000CC89FE01F7CF81E08093320AE4EEFDE1E3
:1003A0008491EF012196882319F0F6D7FE01F8CF4A
:1003B000EEE9FDE18491EF012196882319F0ECD755
:1003C000FE01F8CF8BE1E2E6FAE0A1E8BAE00190A5
:1003D0000D928A95E1F78091600A9091610A90935D
:1003E000800A80937F0ADF91CF911F91FF90EF9059
:1003F000DF90CF90089580913F0E823039F489E8E4
:100400009DE19093A4078093A307F2D70E94FE5822
:100410006093430E7093440E8093450E9093460E66
:100420008091320A882319F081E08093310A81E0BB
:1004300080933F0E0895CF93DF931092310A83E0AB
:1004400080933F0E80918C0E8823B1F0E1E8FDE1AE
:100450008491EF01882341F0082E000C990B86DE71
:100460002196FE018491F6CF8DE090E07FDE8AE058
:1004700090E0DF91CF917ACEE5E8FDE18491EF0144
:10048000882391F3082E000C990B70DE2196FE0153
:100490008491F6CF8F929F92AF92BF92CF92DF92CC
:1004A000EF92FF920F931F93CF93DF9300D01F9291
:1004B000CDB7DEB7FC018381813079F5818181FF81
:1004C0002CC081899289A389B489892B8A2B8B2B93
:1004D00009F448C07F0140E050E0BA01CF010E941A
:1004E000F5978823D1F0F70185889688A788B08C86
:1004F000C18CD28C82E090E0A0E0B0E0F601808375
:100500009183A283B3839E012F5F3F4FB501A40166
:10051000C6010E946AD2811102C080E03CC000E0A6
:1005200010E09801B501A401C6010E94D9D1882329
:10053000A1F389809A80AB80BC80F60187898031E5
:1005400041F4F8EF8F16FFEF9F06A104B10460F4A9
:10055000DACF88EF88168FEF9806A8068FE0B806E6
:1005600018F4D1CF81E017C0F701158A168A178ACF
:10057000108E118A128A138A148A8181806881837D
:10058000C7010E94B8D3882341F240E050E0BA018D
:10059000C7010E94F5970F900F900F900F90DF9179
:1005A000CF911F910F91FF90EF90DF90CF90BF9070
:1005B000AF909F908F9008951092340A1092310A54
:1005C0008091FD0B882321F08AEF9BE00C94DF984B
:1005D00008952F923F924F925F926F927F928F92E7
:1005E0009F92AF92BF92CF92DF92EF92FF920F93C2
:1005F0001F93CF93DF93CDB7DEB7C257D1090FB6A4
:10060000F894DEBF0FBECDBF8C013B014A014DB750
:100610005EB7E1965FAF4EAFE197AD961FAEAD9777
:100620001B0154E0250E311C7E018FE5E80EF11C04
:100630009DEE492E92E0592EE0E4F0E0EC0FFD1F14
:100640003496E396FFAFEEAFE397F30187818230F4
:1006500008F45AC184859585A685B7858F71992739
:10066000AA27BB27892B8A2B8B2B09F04DC110920F
:10067000420A42E45AE0BE016F5F7F4FC1010E940F
:1006800050D318160CF040C18C85982F987190317A
:1006900029F42091AF0C2150223078F429812223B3
:1006A00009F432C1253E89F22E3279F22091420AB4
:1006B0002E3259F28A7049F6B4C04DB75EB7AF9684
:1006C0005FAF4EAFAF97BE016F5F7F4FC7010E9414
:1006D0004BD10115110521F0F8018081811197C0DE
:1006E00021E081E090E0F70101900020E9F73197E7
:1006F000EE19FF098E0F9F1F02964DB75EB7481B7C
:10070000590B0FB6F8945EBF0FBE4DBF8DB79EB7A5
:1007100001965C01211102C0B80102C062E273E0DF
:10072000C5010E94EDEDB701C5010E94CEED62E268
:1007300073E0C5010E94CEED25961FAE2597289641
:100740001FAE289724961FAE1EAE249722965FAE4A
:100750004EAE229721E0A701B101E3968EAD9FAD89
:10076000E3970E946B9E811126C08091AF0C81118E
:1007700022C0E4EEFDE184916F019FEFC91AD90A0E
:10078000882319F009D6F601F6CFEDE6FDE1849154
:100790006F012FEFC21AD20A882319F0FDD5F60196
:1007A000F6CF6701F60181916F01882311F0F4D52E
:1007B000F9CF8AE0F1D58BE1FE01EC5BFF4FDE0162
:1007C000959601900D928A95E1F724968EAD9FAD96
:1007D00024979CA38BA35AA249A240E050E0BE01FB
:1007E0006F5D7F4FC501F5DECE0181960E9498A016
:1007F000CE01805C9F4F0E9498A0AF964EAD5FAD3A
:10080000AF970FB6F8945EBF0FBE4DBF1ECFF80175
:1008100001900020E9F73197CF01801B910B20E078
:1008200062CF81E0903109F080E08093330A90310B
:1008300041F08985873409F008CF8A858E3709F41D
:1008400004CF8091AF0C813029F08230B9F1811151
:10085000FCCE0AC08091B00C9091B10C019690939F
:10086000B10C8093B00CF1CEBE016F5F7F4F85E37A
:100870009AE00E944BD10115110529F485E3C82E99
:100880008AE0D82E08C06801F60181916F018823A3
:10089000A9F382D5F9CFF60181916F01882311F078
:1008A0007BD5F9CF80E278D56D8D7E8D8F8D98A127
:1008B0004AE00E94EF8C8AE06FD5C7CEBE016F5F21
:1008C0007F4F85E39AE00E944BD18114910441F05F
:1008D00065E37AE0C4010E94BBED892B69F414C082
:1008E000AD96FFADAD978F2F90E02091BC0F30916A
:1008F000BD0F8217930741F0AD962FADAD972F5FD7
:10090000AD962FAFAD97A1CEE1968EAD9FADE1979D
:100910000FB6F8949EBF0FBE8DBFCE58DF4F0FB6F7
:10092000F894DEBF0FBECDBFDF91CF911F910F9125
:10093000FF90EF90DF90CF90BF90AF909F908F90FF
:100940007F906F905F904F903F902F9008950F93FE
:100950001F93CF93DF93CDB7DEB76F970FB6F894A1
:10096000DEBF0FBECDBF8B0122E02093AF0C909372
:10097000BD0F8093BC0F81E89AE00E943C9A8BE106
:10098000E1E8FAE0DE01159601900D928A95E1F713
:1009900080917F0A9091800A9C838B838DEE92E0F8
:1009A0009A838983A801BE016F5F7F4F80E090E04A
:1009B00010DECE0101960E9498A06F960FB6F894B3
:1009C000DEBF0FBECDBFDF91CF911F910F91089574
:1009D0002F923F924F925F926F927F928F929F924F
:1009E000AF92BF92CF92DF92EF92FF920F931F933D
:1009F000CF93DF93CDB7DEB76F970FB6F894DEBF16
:100A00000FBECDBF6C012DB63EB61D8218861C826E
:100A10001B828DEE92E09A838983FB0180819E0187
:100A20002F5F3F4F39018F3241F08DE79AE0F60199
:100A300091838083F62E172F62C08EE59AE0F6012F
:100A4000918380838B010F5F1F4F0115110509F4FE
:100A500054C04DB65EB66FE270E0C8010E94D9ED99
:100A60004C010817190708F046C07C01E01AF10A8A
:100A7000FF24C70101962DB73EB7281B390B0FB6CF
:100A8000F8943EBF0FBE2DBF8DB79EB701965C0197
:100A9000A701B8010E9402EEF501EE0DFF1D1082C4
:100AA000F601608171816115710511F06C5F7F4FF6
:100AB00021E0A501CE0105960E946B9E81110FC019
:100AC000B50189E59DE10E946DC58EE265D48AE09D
:100AD00063D40FB6F8945EBE0FBE4DBE0EC0F601D5
:100AE0007182608284010F5F1F4F0FB6F8945EBE63
:100AF0000FBE4DBEAACFF02E02C0F12C10E0C301F4
:100B00000E9498A08F2D912F0FB6F8943EBE0FBE75
:100B10002DBE6F960FB6F894DEBF0FBECDBFDF912E
:100B2000CF911F910F91FF90EF90DF90CF90BF90EA
:100B3000AF909F908F907F906F905F904F903F907D
:100B40002F9008959091BF10E92FF0E0EC5BFA4FE1
:100B500080839F5F943018F49093BF1002C010926E
:100B6000BF108091C0108F5F8093C0100895CF9305
:100B7000FC0120812B33A1F02091C010243080F49F
:100B8000C62FBC018091BF10F0E68F9FC0011124D9
:100B9000875B9A4F0E94EDED8C2FD4DF81E001C07E
:100BA00080E0CF9108952F923F924F925F926F9283
:100BB0007F928F929F92AF92BF92CF92DF92EF92ED
:100BC000FF920F931F93CF93DF9300D000D0CDB748
:100BD000DEB79A8389830E94FE58E981FA81C68034
:100BE000D780E084F184C114D104E104F10409F058
:100BF000ACC22485222309F469C33285215024879D
:100C000021E0230F22874585241301C01286E98144
:100C1000FA8124E0329FE00DF11D1124C684D784AF
:100C2000E088F188E981FA81C282D382E482F58288
:100C3000DC01CB018C0D9D1DA11DB11D8683978309
:100C4000A087B18784819581892B09F43FC3FFB7C1
:100C5000FD83F894E981FA81228033802101612C9F
:100C6000712C04811581809119028F3121F08F3F01
:100C700009F068C205C0E7E4F8E124912E83DAC0E8
:100C80008FE180931902E7E4F8E184918E838F3F2E
:100C900009F458C2823009F469C030F5882309F498
:100CA0004CC0813009F0C6C01092800010928100C3
:100CB00080918100886080938100809181008160B3
:100CC00080938100EBE4F4E2E491F0E0EE0FFF1F8B
:100CD000E850FC4D85919491E1E9F4E2E491E093D0
:100CE000C10FE1E0EE8330C19E81943009F482C0EF
:100CF00008F460C0953009F09DC010922001109258
:100D0000210180912101886080932101809121013E
:100D1000816080932101EBE4F4E2E491F0E0EE0FD6
:100D2000FF1FE850FC4D85919491E1E9F4E2E491D4
:100D3000E093BE0F95E09E8307C114BC15BC84B53B
:100D4000826084BD85B5816085BDEBE4F4E2E49109
:100D5000F0E0EE0FFF1FE850FC4D85919491E1E922
:100D6000F4E2E491E093C20F1E82ABC21092B00095
:100D70001092B1008091B00082608093B0008091A9
:100D8000B10081608093B100EBE4F4E2E491F0E023
:100D9000EE0FFF1FE850FC4D85919491909329052B
:100DA00080932805E1E9F4E2E491E0932A05F2E07A
:100DB000FE8387C210929000109291008091910062
:100DC0008860809391008091910081608093910070
:100DD000EBE4F4E2E491F0E0EE0FFF1FE850FC4D8D
:100DE00085919491E1E9F4E2E491E093C00F23E06E
:100DF0002E83AAC01092A0001092A1008091A100A1
:100E000088608093A1008091A10081608093A100FF
:100E1000EBE4F4E2E491F0E0EE0FFF1FE850FC4D4C
:100E200085919491E1E9F4E2E491E093BF0F84E0CD
:100E30008E838AC0EE81E7FD85C161E08FE10E946B
:100E40000DB68E818D7F09F083C04801A12CB12C95
:100E500060E072E18AE790E0A50194010E944DEA0A
:100E600029833A834B835C8369017A01F1E0CF1ACD
:100E7000D108E108F1082FEFC216D104E104F10412
:100E800009F008F44EC060E472E48FE090E0A50140
:100E900094010E944DEA69017A0181E0C81AD108E3
:100EA000E108F1089E81923009F5EFEFCE16D104EA
:100EB000E104F10409F008F4CBC160E970ED83E0CE
:100EC00090E0A50194010E944DEA69017A01F1E0E8
:100ED000CF1AD108E108F1082FEFC216D104E104BE
:100EE000F10411F008F041C183E027C08FEFC8166C
:100EF000D104E104F104B9F0B0F068E478EE81E0E7
:100F000090E0A50194010E944DEA69017A0191E007
:100F1000C91AD108E108F108EE81EE2309F49AC15B
:100F200063C181E001C082E09E81911106C095B548
:100F3000987F892B85BD7AC085E09091B100987F1C
:100F4000892B8093B10072C061E08FE10E940DB6E1
:100F50004801A12CB12C60E072E18AE790E0A50184
:100F600094010E944DEA69017A01E1E0CE1AD108AC
:100F7000E108F108C114D104F1E0EF06F10488F0B2
:100F800068E478EE81E090E0A50194010E944DEACA
:100F900069017A0181E0C81AD108E108F10883E00B
:100FA00001C081E09E81913071F490918100987F21
:100FB000892B80938100452846284728D9F52FEFB3
:100FC0003FEFA90168C0EE81E33071F49091910088
:100FD000987F892B8093910045284628472851F512
:100FE0002FEF3FEFA90179C0FE81F43071F49091A9
:100FF000A100987F892B8093A10045284628472887
:10100000C9F42FEF3FEFA9017AC02E81253071F48A
:1010100090912101987F892B8093210145284628B2
:10102000472841F42FEF3FEFA9017BC04528462810
:10103000472869F0D801AA0FBB1F91010E9479EAE5
:1010400028EE33E040E050E00E942BEA03C02FEF8F
:101050003FEFA9018E81823081F12CF4882361F069
:101060008130C9F06FC09E81943009F448C0ACF162
:10107000953009F456C066C0C7BC2093D30F309397
:10108000D40F4093D50F5093D60F80916E0082609D
:1010900080936E0057C0D0928900C0928800209340
:1010A000CF0F3093D00F4093D10F5093D20F809138
:1010B0006F00826080936F0045C0C092B3002093A0
:1010C0002B0530932C0540932D0550932E058091D0
:1010D000700082608093700035C0D0929900C092F9
:1010E00098002093CB0F3093CC0F4093CD0F5093AB
:1010F000CE0F8091710082608093710023C0D092E6
:10110000A900C092A8002093C70F3093C80F409346
:10111000C90F5093CA0F8091720082608093720051
:1011200011C0D0922901C09228012093C30F30939F
:10113000C40F4093C50F5093C60F80917300826017
:1011400080937300ED81EFBFC1C0DC01CB018C192E
:101150009D09AE09BF09B7FDB9C04698E981FA817A
:101160001682178210861186B1C068E478EE81E09D
:1011700090E0A50194010E944DEA69017A01F1E035
:10118000CF1AD108E108F1082FEFC216D104E1040B
:10119000F10441F138F164E274EF80E090E0A501E0
:1011A00094010E944DEA69017A01F1E0CF1AD10859
:1011B000E108F1082FEFC216D104E104F10409F0AF
:1011C00008F4BACE62E17AE780E090E0A5019401EC
:1011D0000E944DEA69017A0181E0C81AD108E1084C
:1011E000F10819C084E0A9CE2FEFC216D104E104A2
:1011F000F10409F008F463C062E17AE780E090E06E
:10120000A50194010E944DEA69017A01F1E0CF1A2B
:10121000D108E108F1082FEFC216D104E104F1046E
:10122000A9F0A0F089819A81AB81BC812AE0B595B3
:10123000A795979587952A95D1F76C017D01F1E0E7
:10124000CF1AD108E108F10887E077CE86E075CEA5
:1012500082E073CEEFEFCE16D104E104F10469F120
:1012600060F162E17AE780E090E0A50194010E94DC
:101270004DEA69017A0181E0C81AD108E108F10854
:101280009FEFC916D104E104F104A9F0A0F089810F
:101290009A81AB81BC813AE0B595A79597958795E2
:1012A0003A95D1F76C017D01E1E0CE1AD108E10851
:1012B000F10885E03CCE84E03ACE83E038CE84E08D
:1012C00033CE61E08FE10E940DB6BFCD26960FB6FA
:1012D000F894DEBF0FBECDBFDF91CF911F910F916C
:1012E000FF90EF90DF90CF90BF90AF909F908F9046
:1012F0007F906F905F904F903F902F9008950F9345
:101300001F93CF93DF93CDB7DEB72C970FB6F8942A
:10131000DEBF0FBECDBFE2E3F4E080859185A285FC
:10132000B385448155816681778100811181228155
:10133000338109831A832B833C834D835E836F83C0
:10134000788789879A87AB87BC87AE01475F5F4FF5
:10135000BE016B5F7F4FCE0101960E94C8BC2EE399
:1013600034E0AE01475F5F4FBE016B5F7F4FCE0140
:1013700001960E9422C82C960FB6F894DEBF0FBECD
:10138000CDBFDF91CF911F910F910895FC01238173
:1013900021110C94DF9808959091C00095FFFCCF27
:1013A0008093C6000895EF92FF921F93CF93DF932F
:1013B0007C0160E0DCDB182F882399F0E4EEFDE18E
:1013C0008491EF012196882319F0E6DFFE01F8CF22
:1013D000B7018AEE9DE10E946DC582E2DDDF8AE001
:1013E000DBDF812FDF91CF911F91FF90EF90089568
:1013F000DF92EF92FF920F931F93CF93DF93CDB7BE
:10140000DEB76E970FB6F894DEBF0FBECDBF60910A
:10141000A3077091A4076115710541F14DE150E0FA
:10142000CE0101967C010E94E6E51E8EF7018F0138
:101430000E191F09D190DD2019F09AE0D912F7CFCB
:10144000F701E00FF11F1082C701ADDF882371F0B3
:10145000DD20A9F00F5F1F4F8091A3079091A40793
:10146000080F191F1093A4070093A30781E0209190
:10147000A3073091A407232B29F480E003C000E0E8
:1014800010E0F0CF6E960FB6F894DEBF0FBECDBF62
:10149000DF91CF911F910F91FF90EF90DF90089512
:1014A0003F924F925F926F927F928F929F92AF92F4
:1014B000BF92CF92DF92EF92FF920F931F93CF9341
:1014C000DF931F92CDB7DEB793DF811175C2809194
:1014D000C010843008F048C00E94A94BAC0197FFAF
:1014E0007CC142C08E3409F0D9C10115110509F43F
:1014F000D5C16DE17FE1C8010E94F5E57C01892B32
:1015000009F48EC16EE470E0C80104960E94D9ED22
:10151000009709F485C14AE050E060E070E0019670
:101520000E9491E36093D70F7093D80F8093D90FE7
:101530009093DA0F8090BE189090BF18A090C018BA
:10154000B090C1182FEF821A920AA20AB20A681547
:1015500079058A059B0509F465C1EF2809F062C188
:101560008AEE9EE10E942BD78091310A882309F4EC
:1015700023C28091C010811102C010923D10EE2450
:10158000E3944091AB0C5091AC0C6091AD0C709118
:10159000AE0C8091A70C9091A80CA091A90CB091D1
:1015A000AA0C481759076A077B0708F4E12C00E0EA
:1015B00010E09924939480E6882E92E2A92E9FE170
:1015C000B92E2DE8322E8091C010843008F0F4C17D
:1015D000E110F2C180913D108111EEC18091020CA9
:1015E0009091030CA091040CB091050C8093AB0C6E
:1015F0009093AC0CA093AD0CB093AE0C41E050E0D6
:10160000BE016F5F7F4F8AEF9BE00E945F9B019757
:1016100019F4898190E002C08FEF9FEFF82E40907F
:10162000AB0C5090AC0C6090AD0C7090AE0C409137
:10163000A70C5091A80C6091A90C7091AA0CEE24F3
:10164000E394441655066606770608F4E12C441622
:10165000550666067706B0F4019609F46AC08AE07A
:10166000F81609F489C09DE0F91609F485C023E253
:10167000F21619F08AE3F81296C080913C1081119D
:1016800092C06FC00E941E6A8AEF9BE00E94DF98A2
:101690008091150C882359F181508093150C389E48
:1016A000C001112441E061E0865E934F0E948BD51A
:1016B000E091150C94E0E99FF0011124EA5EF34FEC
:1016C00040815181628173814093AB0C5093AC0C8B
:1016D0006093AD0C7093AE0C8AEF9BE00E94F5977F
:1016E0008091320A8823A9F09092310A12C0109298
:1016F000310A0E94AAB70E94FA780E9474786D336A
:1017000071058105910528F0B092A407A092A30766
:101710006FDE8091310A811128C0E5E3FFE18491F9
:101720006F012FEFC21AD20A8823D9F035DEF601F5
:10173000F6CFEFECFDE184916F019FEFC91AD90A52
:10174000882319F029DEF601F6CFE6E2FFE1849165
:101750006F012FEFC21AD20A882319F01DDEF6019D
:10176000F6CF83E2F81208C005C023E2F21221C1CD
:1017700000E010E090923D1010923C100115110510
:1017800019F40E94CF7B0CC08091BF10889E000D81
:10179000111D1124F801E75BFA4F108280E0D2D9C5
:1017A00000E010E010CF0F35110508F00CCF9BE3DF
:1017B000F91202C090923C1080913C10811103CF2D
:1017C0008091BF10F801889EE00DF11D1124E75BA8
:1017D000FA4FF0820F5F1F4FF6CE982F2091BC1862
:1017E0003091BD188A3019F09D3009F0B0C01092C8
:1017F0003B102115310519F40E94CF7B68CEF90109
:10180000E552F04F10821092BD181092BC180BEDEB
:101810001FE0F8018191803209F064CE8F01F9CF89
:10182000C80179CE6AE270E0C8010E9411EE9C0105
:10183000009701F1982F901BF12C992339F09150CA
:10184000F801E90FF11D8081F826F7CF4AE050E05A
:1018500060E070E0C90101960E9491E3CF2CD12C89
:10186000E12CF12C6C157D058E059F0531F08BEC7C
:101870009EE178CE81EA9EE175CE8091D70F90915E
:10188000D80FA091D90FB091DA0F8093BE18909322
:10189000BF18A093C018B093C1180EC080912F0A32
:1018A000882351F060EF73E0C8010E94E4ED892BBA
:1018B00019F087E79EE156CE80912702811126C05C
:1018C00067E470E0C8010E94D9ED0097F9F04AE0A2
:1018D00050E060E070E001960E9491E397FD16C031
:1018E00064307105810591052CF065307105810525
:1018F000910561F4E0E0FEE184917F019FEFE91A38
:10190000F90A882319F048DDF701F6CF64EF73E098
:10191000C8010E94E4ED892B11F41092200269EFB6
:1019200073E0C8010E94E4ED892B21F487EF9DE16B
:101930000E94BBA06EEF73E0C8010E94E4ED892B0A
:1019400009F42AD261E08BED9FE011D9C0CD2F358B
:1019500031050CF0BCCD9C35C1F40E94A94B97FD1C
:10196000B6CD20913B102111B2CD2091BC18309101
:10197000BD18A9014F5F5F4F5093BD184093BC182D
:10198000F901E552F04F8083A2CD9B3319F481E039
:1019900080933B1080913B10811199CDC901019634
:1019A0009093BD188093BC18F901E552F04F408325
:1019B0008ECD10923C10E5CE0F90DF91CF911F910C
:1019C0000F91FF90EF90DF90CF90BF90AF909F90DE
:1019D0008F907F906F905F904F903F9008958F927F
:1019E0009F92AF92BF92EF92FF920F931F93CF936C
:1019F000DF93CDB7DEB7A0970FB6F894DEBF0FBE6A
:101A0000CDBF611571058105910589F100E0842E36
:101A1000912CA12CB12C102FEE24E394F12CEC0E80
:101A2000FD1EE00EF11C07FDFA94A50194010E9431
:101A30002BEAF7016083B901CA010F5F61157105D7
:101A40008105910541F71F3F21F1E1E0F0E0EC0F46
:101A5000FD1FE10FF11D17FDFA9580818A3010F00E
:101A600097E301C090E3890F97DC1150ECCF80E33E
:101A7000A0960FB6F894DEBF0FBECDBFDF91CF9119
:101A80001F910F91FF90EF90BF90AF909F908F901C
:101A900083CCA0960FB6F894DEBF0FBECDBFDF910A
:101AA000CF911F910F91FF90EF90BF90AF909F90BB
:101AB0008F900895CF92DF92EF92FF926B017C019D
:101AC00097FF0AC08DE268DCF094E094D094C09453
:101AD000C11CD11CE11CF11C4AE0C701B601FF90FA
:101AE000EF90DF90CF907BCF8F929F92AF92BF927B
:101AF000CF92DF92EF92FF92CF936B017C01B42ED5
:101B000020E030E0A9010E943DE687FF06C08DE29B
:101B100043DCF7FAF094F7F8F094C0E060E070E08E
:101B200080E09FE3CB1541F02DEC3CEC4CEC5DE309
:101B30000E94A2E6CF5FF6CF9B01AC01C701B601C0
:101B40000E9489EA6B017C010E94D2EB4B015C018F
:101B50004AE045DFCC2379F1C501B4010E9441E69A
:101B60009B01AC01C701B6010E9488EA6B017C01B0
:101B70008EE212DC20E030E040E251E4C701B60121
:101B80000E94A2E64B015C010E94CDEB6B01770F36
:101B9000EE08FF08C701B6018DDFC701B6010E943C
:101BA00043E69B01AC01C501B4010E9488EA6B01C8
:101BB0007C01C150F9F6CF91FF90EF90DF90CF906C
:101BC000BF90AF909F908F900895CF92DF92EF9249
:101BD000FF920F931F93CF93DF9388E50E944E4CA3
:101BE000D82E89E40E944E4CC82E882319F00E94FA
:101BF000E74B1CC0DD20C1F00E94174C20E030E014
:101C000040E251E40E9488EA20E030E048EC51E4F0
